:020000040000FA
:040000006FD00400B9
:101000006F00907E00000000000000009020002093
:10101000AA220020A9BDF9F56C23002000000000E1
:10102000000000006C230020902000200000000041
:101030000000000090200020000000009020002010
:101040000000000090200020902000209020002030
:101050009020002090200020582F00209424002071
:101060000000000090200020902000201E2400207E
:1010700090200020D22300209020002090200020EB
:101080009020002090200020902000209020002020
:101090009020002001A04111B7170040985F3AC688
:1010A000945F3247E39CE6FE3245410182800111A4
:1010B00013078008F337078093F787083EC20100C3
:1010C0000100B7170040930570052380B70413068D
:1010D00080FA2380C7040100010083C6B70493F699
:1010E000F60DA385D704238007049246F3A6068055
:1010F0000100010093760502D5CEF336078093F602
:10110000860836C4010001002380B7042380C70489
:1011100001000100B70614007D89558D88C70100C4
:1011200001000100010023800704A246F3A6068007
:101130000100010073370780137787083AC6010062
:1011400001002380B7042380C704010001000100CF
:1011500001003727004093061005A303D7802380A2
:101160000704B247F3A70780010001009307800836
:10117000F3B7078093F787083ECE01000100B71749
:101180000040130770052380E704130780FA2380CB
:10119000E7040100010003C7B70413670708A3852C
:1011A000E70423800704F247F3A70780010001004A
:1011B0000561828093760504BDC6F336078093F6F9
:1011C000860836C8010001002380B7042380C704C5
:1011D00001000100B7061400938606047D89558D31
:1011E00088C7010001000100010023800704C246F6
:1011F000F3A6068001000100733707801377870884
:101200003ACA010001002380B7042380C70401000B
:1012100001003727004093062005A303D7802380D1
:101220000704D24781B773370780137787083ACC12
:10123000010001002380B7042380C70401000100DE
:1012400098471367070C98C723800704E24719BF24
:101250000111814601468145114506CE97000000E7
:10126000E780605893078008F3B7078093F78708F3
:101270003EC601000100B717004013077005238028
:10128000E704130780FA2380E7040100010003C785
:101290006704136717002383E70423800704B2471A
:1012A000F3A7078001000100F2400561828041112F
:1012B000814601468145114597000000E780A05214
:1012C00013078008F337078093F787083EC40100AF
:1012D0000100B7170040130670052380C70493066A
:1012E00080FA2380D70401000100FD552396B70240
:1012F00023800704A245F3A5058001000100733790
:101300000780137787083AC6010001002380C704CD
:101310002380D7040100010003C767041367170087
:101320002383E70423800704B247F3A70780010063
:10133000010001A0BD473305F50201007D1575FDD3
:101340008280411122C426C206C6AA8401446317C2
:101350009400B24022449244410182800504130566
:10136000803E420497000000E78000FD4180C5B741
:101370009305000273A04580824573901534924016
:101380002242B2424243D2436244F2440255925551
:101390002256B2564257D2576258F25806499649D9
:1013A000264AB64A464BD64B664CF64C065D965DD1
:1013B000265EB65E465FD65F09617300203041113C
:1013C000B7170040985F3AC6945F3247E39CE6FE49
:1013D000324541018280B71700401307000323887C
:1013E000E702854717170000232EF74673002030C9
:1013F000411122C42D6426C24AC006C637190040D6
:101400001304A4AAB704002023208900976000E0F9
:10141000E78060719C408297976000E0E780A07051
:10142000E5B737370040834747009146BD8B639E41
:10143000D702B73600401306F00F973500009385AA
:10144000651E9737000083D7E72D03C7A6001377E3
:10145000F70F1DE3B7E70400BC4F09468945171590
:1014600000000345A5F7829731A099466394D70001
:10147000834757007300203003C786001377F70FA8
:10148000E365F6FC13851700AE9717380000231BA1
:10149000A8282380E70075B7B787004003C7670017
:1014A000098B6309071003C77700930600031377BE
:1014B0000703630DD708173800000348F87717367D
:1014C0000000130666740547B30606012380E60094
:1014D00083C577001737000013070775429793F508
:1014E000F50F2300B70003C58700973500009385EB
:1014F000A572C2951375F50F2380A5000347070059
:1015000089451377F703630CB70C63E7E50A6306B5
:10151000071A8545630CB7129737000083C7D77148
:101520003307F600034707001377F70F19CB85073A
:1015300093F7F70F3D476363F71A17370000A30DC2
:10154000F76EB787004009472383E700B78700405D
:1015500083C77700E207E18763DE0704973700005F
:1015600083C7976D173700001307076A3E978546B4
:101570002300D700173700001307076B3E97930629
:1015800000032300D700173700001307E7683E97D2
:10159000A14685072300D70093F7F70F3D47636403
:1015A000F71417370000A309F768B7870040094709
:1015B0002383E70073002030930610026300D70EE8
:1015C000930620026305D70693060002E316D7F4BC
:1015D00003C727021377C70F13672700D5A803C7D0
:1015E00067001377070465CB03C7A702173800000D
:1015F00013080843173500001305453A1347070839
:101600002385E70203C7A7021377370F1367870005
:101610002385E702814713070004B305F5008C41D9
:10162000B306F80091078CC2E399E7FEF5B503C74E
:10163000A702134707042385E70203C7A70213770E
:10164000C70F136727002385E702F9B503C76700B3
:101650001377070449C303C767021738000013084C
:10166000E82F1735000013052527134707082383A4
:10167000E70203C767021377370F136787002383D7
:10168000E702814713070004B305F5008C41B30658
:10169000F80091078CC2E399E7FEBDBD03C767025E
:1016A000134707042383E70203C767021377C70FB3
:1016B000136727002383E70285B503C76700137705
:1016C000070411CB03C727021377370F136787006F
:1016D0002381E70291B5238006003DBD97370000C6
:1016E000A38C0754B9BD97370000A387075475BD75
:1016F0002303048015472303E48001002302A48010
:10170000828083076480E3CE07FE23030480828007
:1017100083076480E3CE07FE03454480828083070D
:101720006480E3CE07FE2302A4808280411126C498
:101730004AC24EC006C61377F50BAD47AA892E895B
:101740009544630CF700194597000000E78080FA84
:1017500097000000E78020FB8D444E859700000035
:10176000E78040F9FD59FD1463983401B240A2446A
:101770001249824941018280135509011375F50F01
:1017800097000000E780E0F92209F1BF011126CCA3
:1017900006CEB704080097000000E780C0F61545A4
:1017A00097000000E78000F597000000E78080F6D2
:1017B00097000000E78000F62AC697000000E78047
:1017C00080F432459377150089EB13651500137586
:1017D000F50FF240E24405618280FD14E9F0014515
:1017E000CDBF397126DC4ADA4ED852D656D45AD2F9
:1017F0005ED006DE62CE66CCB7E700E07D5783AAF6
:10180000070022C603AA470023A0E71823A2E7186F
:10181000B7170040130770052380E704130780FA09
:101820002380E70483C74704930B75FFB684E20760
:1018300093FBFB0F8546AA892E8B32893724004003
:10184000E187015763FA76016308D50089461307DB
:1018500000026313D5000157D98F93F7F70FB71C18
:1018600000402382FC0411472303E4801305F00F9A
:1018700097000000E78000E8094C97000000E7802F
:1018800080E863657C15B7050700DA9537870700A0
:10189000795563FEE504B3879500636AF704370B57
:1018A0000800A94733EB65016395F90881E8814495
:1018B00097000000E78020E5268515A8DA85094510
:1018C00097000000E780C0E605090345F9FFFD1415
:1018D000050B97000000E780C0E481C49377FB0FFD
:1018E000E5F797000000E780A0EA69F17D55B7179A
:1018F0000040130770052380E704130780FA238054
:10190000E70403C74704418B2382E704F250B7E79B
:1019100000E023A0571123A24711E2543244525948
:10192000C259325AA25A125B825B724CE24C21615C
:101930008280A547639BF90685691309F00FB306FA
:101940009900B3742B01B6941349F9FFB37499004D
:10195000856B33796901416B9387F9FFB3F72701F1
:1019600099E363FC340193D94900C147E3E637FFAB
:101970003DBF0569C1697D19D9B71305800D63881D
:101980006901130500026384790113051008CA85F3
:1019900097000000E780C0D997000000E78040DF93
:1019A00031D54E99B38434416DBFDA852D4597000A
:1019B0000000E780E0D7CA94E30B99EE0509970091
:1019C0000000E78020D5A30FA9FEFDB79387F9FF9C
:1019D00093F7F70F636DFC0C83C71C0413073008E3
:1019E0006315F706370708006361EB06B3079B0032
:1019F000B706100063FBD704334BEB0089476399AC
:101A0000F9068980D549E38404EADA850945970017
:101A10000000E780E0D111090327C9FF9147232087
:101A2000E48003076480E34E07FE23033481FD173F
:101A3000EDFBFD14110B81C49377FB0FE9FF9700B9
:101A40000000E780E0D461F155B5B717004003C747
:101A50005704B70708001377070219E3B787070091
:101A60007955E376FBE833079B00E3F9E7F841B5E6
:101A70008547E380F9F0DA852D4597000000E7807F
:101A800020CB9389F4FFE38404E297000000E78011
:101A900060C893F7390091EB83260480032709007F
:101AA00093074900E396E6E03E89CE84D9BFB54767
:101AB0006399F9001305900B97000000E78080C33D
:101AC000FDB3B1471305B00AE388F9FE9947639760
:101AD000F904B7050800B365BB002D459700000069
:101AE000E78000C581448D4BA14997000000E78045
:101AF00060C263967401832704802320F900850463
:101B0000E39534FF8327048013172B0163550700E7
:101B10002312F90069BB2322F90051BB9D47639F43
:101B2000F90281451305B00497000000E78040C02A
:101B3000BD442320090023220900FD59970000001D
:101B4000E78040BD93F77400CA9703C70700FD14F0
:101B5000398D2380A700E39334FF91BBA14763979E
:101B6000F90697000000E780A0C28144630D0B00D6
:101B70008D479304C0036308FB00930400056304CE
:101B80008B01930440041375C507E30295D21945F0
:101B900097000000E78000B697000000E780A0B63D
:101BA000054597000000E780E0B426859700000017
:101BB000E78020B7094597000000E78080B69700CE
:101BC0000000E780E0BCE31405CE0DB39147639FAE
:101BD000F9001305600697000000E780A0B19700A8
:101BE0000000E78040B213059009F9B5E38109CC04
:101BF000F1547DB9BD660147173600001306063063
:101C0000938606A685458347060093F7F70F91C391
:101C100082800507E3F9E6FE973700002380B72EA0
:101C2000DDB77D166206618693178601E18763D46E
:101C3000070001458280931726003307F500AE9711
:101C400018439C4363E7E7007D16E37FF7FC7D556F
:101C5000828005458280FD15E205E18513978501A7
:101C6000618793F7F50F63480700FD15139725006B
:101C70002A97584365D713851700620561858280CE
:101C80003308B5021C4283A80600B335B502C297DB
:101C900033B50701AE98469585486367B5006394F0
:101CA000A50063E3070181480C43C6950CC388C2B5
:101CB0001CC2828081471397870161876343B70005
:101CC0008280139727002A97232007008507E5B70E
:101CD0008147014793968701E18663C5B6001335B6
:101CE0001700828093962700AA9694428507558F05
:101CF000D5B793D755408A07AA979C430545331516
:101D0000B5007D8D828017F3FFDFE702833D2A84D3
:101D100097000000E78060F405C5931725003E9406
:101D20000327C4FF814711EB7D1516053E9542053B
:101D3000418517F3FFDF6700033D05838507E5B79E
:101D40000145C5BF81471397870161876343C7007A
:101D5000828013972700B386E50094422A9785076F
:101D600014C3D5B77D1662066186014793178601B5
:101D7000E18763D50700133517008280931726008B
:101D8000B306F500AE9794429C437D16B58F5D8FE8
:101D9000F1BF8A05AA9501476363B500828083A6D7
:101DA000C5FFF11593D71600D98F9CC11397F60183
:101DB000E5B72A830148014701456343D700828084
:101DC000B387050183A80700B30706019C43C697A4
:101DD000AA976384F80033B517010507B308030118
:101DE000620723A0F80061871108C1BF2A83014759
:101DF0008147014563C3D70082803388E50083288B
:101E00000800330EE600032E0E003388A840330886
:101E1000C8416384080133B508018507B308E300AE
:101E2000E20723A00801E1871107E9B717F3FFDFF5
:101E3000E702232B0111B286B2842E86AA850A8579
:101E400097000000E780C0FA2A84A6850A859700DB
:101E50000000E78020E833348000060413351500C5
:101E6000018D056117F3FFDF6700E32917F3FFDF3B
:101E7000E702A3244111AA89AE8A328BB68402C23A
:101E800002C402C60144131C8401135C8C416349E3
:101E90009C02939B1400FD1B0549138CF4FFF15C1D
:101EA00033048901620461846340740792478E049D
:101EB000CE9423AEF4FE410117F3FFDF67006323E6
:101EC00013192400B30B2B01014A93172A00D6974C
:101ED00083A50B0088437800340050009700000071
:101EE000E78040DA050A93178A01E187F11BE35E78
:101EF000FCFC92474E9905042320F900A2473EC2FC
:101F0000B24702C63EC441B7131A8901135A8A4127
:101F1000131D240093178A01E18763CF970092472E
:101F20000A044E941CC0A24705091379F90F3EC25A
:101F3000B24702C63EC4ADB7B3079A0313152A00D1
:101F400056950841780034005000050AEA97DA9760
:101F50008C4397000000E780E0D26DBF197106C284
:101F600012C416C61AC81ECA22CC26CE2AD02ED219
:101F700032D436D63AD83EDA42DC46DECAC0CEC2C9
:101F8000D2C4D6C6DAC8DECAE2CCE6CEEAD0EED2F9
:101F9000F2D4F6D6FAD8FEDA971500009385058CB0
:101FA0008841E700050092402242B2424243D243B8
:101FB0006244F244025592552256B2564257D257C5
:101FC0006258F25806499649264AB64A464BD64BBD
:101FD000664CF64C065D965D265EB65E465FD65F45
:101FE0000961730020300000972100209381810156
:101FF000175100201301018117F5FFFF1305C500DC
:102000009705002093850500171600201306C6FDCE
:1020100063FAC5008322050023A055001105910530
:10202000E3EAC5FE170502001305C52E971500202B
:102030009385C5FB171600201306C66563FAC50015
:102040008322050023A0550011059105E3EAC5FE92
:102050001715002013050564974500209385053664
:102060006377B500232005001105E36DB5FEFD4241
:10207000739002BC8D4273904280B722000093821D
:10208000828873900230970200209382A2F793E235
:10209000320073905230975200009382E294739012
:1020A00012346FB0F47573002030397101436EC67D
:1020B00019A0397141536AC866CA62CC5ECE19A0B4
:1020C000397101535AD056D252D44ED64AD826DA54
:1020D00022DC06DE33016140828241114AC026C201
:1020E00022C406C68282B24D4101024D924C224C5E
:1020F000B24B4101024B924A224AB2494101024984
:1021000092442244B240410182803D432A87637356
:10211000C3029377F700BDEFADE5937606FF3D8AE6
:10212000BA960CC34CC30CC74CC74107E36BD7FE30
:1021300011E28280B306C3408A0697020000969699
:102140006780A6002307B700A306B7002306B700E1
:10215000A305B7002305B700A304B7002304B70005
:10216000A303B7002303B700A302B7002302B700FD
:10217000A301B7002301B700A300B7002300B700F5
:10218000828093F5F50F93968500D58D9396050182
:10219000D58D61B7939627009702000096968682A8
:1021A000E78086FA9680C1171D8F3E96E374C3F8C8
:1021B000A5B73367B500FD530D8B79E7B7877F7FF0
:1021C0009387F7F710419441B372F6003363F6003A
:1021D000BE92B3E262006397720C6318D606504158
:1021E000D441B372F6003363F600BE92B3E26200EC
:1021F0006398720A631BD60410459445B372F600C7
:102200003363F600BE92B3E262006391720A631E0A
:10221000D6025045D445B372F6003363F600BE9241
:10222000B3E26200639A72086311D60210499449BE
:10223000B372F6003363F600BE92B3E262006393BA
:1022400072085105D105E30FD6F6131706019397CF
:102250000601631CF7001357060193D706013305E7
:10226000F7409375F50F91E982804183C18333056F
:10227000F7409375F50F91E182801377F70F93F78D
:10228000F70F3305F74082800346050083C605003B
:10229000050585056313D60065FA3305D6408280AF
:1022A00011059105E312D6FE014582802105A105A5
:1022B000E31CD6FC014582803105B105E316D6FC4E
:1022C000014582804105C105E310D6FC01458280AD
:1022D000B717004003C777051377E70FA38BE70411
:1022E000130700F8A38DE7043D47238CE704130789
:1022F0005003A38CE70403C7A7051377D70F238DDB
:10230000E7048280B717004003C7E7020D89411137
:102310001377C70F498F93068008F3B6068093F6AC
:10232000860836C601000100930670052380D70495
:10233000930680FA2380D704010001002387E70277
:1023400023800704B247F3A7078001000100410181
:10235000828041112A83014E930E407E130F001993
:10236000930F400663E56E129308001913034006AD
:10237000B3781503854E0D4FA14F337365020D8958
:102380001335150063EFBE121308F6FF79467298F5
:102390004208135808013307C70213D61700BE07B7
:1023A00032976146B3F6C60213068070B386C60242
:1023B0003697A166F58F42075D8FB716004083C739
:1023C000F60293F70708A303F1000346710083C7E1
:1023D000F60293F70708E394C7FE83477100B71628
:1023E000004093F7F70F6388071293078008F3B74D
:1023F000078093F787083EC401000100B71700402B
:10240000930670052380D704930680FA2380D704AF
:102410000100010023AA070383C6170393E60608F9
:10242000A388D70223800704A247F3A707800100EF
:1024300001001166B71700407D16D45BC85F938515
:102440004703A98EF18EF5FA93068008F3B606804D
:1024500093F6860836C601000100930670052380B6
:10246000D704930680FA2380D7040100010098C1A5
:1024700003C7170313670704A388E7022380070431
:10248000B247F3A7078001000100410182807D135C
:102490003368E3039308E016630E08003368F30320
:1024A0009308D016630808009378330093B8180097
:1024B0009388D81633081E01131E0801135E0E01FF
:1024C00055B56393E5030548638608000148630337
:1024D00003002A8871087298FD15131E0801C205B1
:1024E000135E0E01C18179BD13F8150063F4BF00BE
:1024F0007908D5B713381800E5BF83C7F60293F7FC
:102500000708A303F1000346710083C7F60293F79F
:102510000708E394C7FE8347710093F7F70FF1DFD5
:10252000E9B531714AD966CB06DF22DD26DB4ED70D
:1025300052D556D35AD15ECF62CD6AC96EC7AA8C26
:1025400002D897100000E78020B12A8993078008FD
:10255000F3B7078093F787083EDA01000100B71749
:102560000040130770052380E704130780FA2380D7
:10257000E7040100010003C7F7021377770FA38771
:10258000E70203C7F70213678700A387E7022380E8
:102590000704D257F3A70780010001000545970003
:1025A0000000E78060D6130780C13347E902116A53
:1025B00093070AE893065002BD69930BA004814A71
:1025C000014B13048008930470057D1AB347F90288
:1025D0003307D7023EC0FD873ECC938709A69309F7
:1025E000803E3347F7023AC27D873AC43347390306
:1025F0008549B399990193D93940B306D702B30BF2
:102600007703B3C6F602B3CBFB0236C6FD8636C8E7
:1026100093D6FB4136CEB7460F0093860624334946
:10262000D9028566938606FAB3969601B389E902C4
:10263000130760553309D90293060010B389E902E4
:102640003349D902B3C9F9029316390036CA37198A
:102650000040FD8636D0930D090493D7F9413ED250
:10266000F336048093F6860836DC010001009307F8
:1026700070052380FD00930680FA2380DD000100B1
:1026800001008346390593F6860FA309D9048346D2
:10269000390593E61600A309D90423800D00E256FC
:1026A000F3A6068001000100130C80FA116DF336C9
:1026B000048093F6860836DE01000100930770055A
:1026C0002380FD0023808D01010001008346390530
:1026D000216693E60602A309D90483560905B3E6E9
:1026E000A6012318D90483560905D18E2318D904CD
:1026F00023800D00F256F3A60680010001008346F8
:10270000390593F606026381061A03463905218AC4
:102710006DDE081897100000E7800098733604807B
:1027200013768608B2C20100010023809D00238039
:102730008D0101000100B717004003C6370513766D
:10274000F60DA389C70403C6370513660602A389DD
:10275000C704835609052166B3E6A6012318D904E8
:1027600083560905D18E2318D90423800D0096467F
:10277000F3A60680010001008346390593F60602A0
:10278000638B061483463905A18AEDFE970000206D
:10279000E7806090AA8636D497000020E780A08F5B
:1027A000A256E30AD5FE835609054255B3E6A601B3
:1027B0002318D90497100000E780C08F834639059D
:1027C000A18AEDDE03560905834629058247337643
:1027D000CA00B306DA0293D5F641B296B388F64042
:1027E000E24733B8C6002E983308F840A247B3B684
:1027F00016013308D84063C70701631DF8009247EC
:1028000063FA1701C247634FF80E63950701B24799
:1028100063EAF80E894663E9660FF24693151800DD
:1028200013D3F8015E8613951800B365B30042D642
:1028300046D497C00100E78080113258050B137B06
:10284000FB0F63470001631A0838A25863870838F2
:1028500013081500B336A800B69513D6F5013298C3
:10286000B336C800AE9613581800FE06B3E606014C
:102870007336048013768608B2C6010001002380F7
:102880009D0023808D01010001000356C902B2960C
:10289000C206C1822316D90223800D00B646F3A6D4
:1028A00006800100010021B5F336048093F6860806
:1028B000B6C00100010023809D0023808D0101002E
:1028C00001008346390593E60602A309D904238053
:1028D0000D0086460DB5F336048093F68608B6C41F
:1028E0000100010023809D0023808D010100010073
:1028F0008346390593E60602A309D90423800D0017
:10290000A646BDB5E30B0BF0F336048093F68608BC
:10291000B6C801000100930680FA23809D00238041
:10292000DD00010001008346390593F5FC0F93F6A5
:10293000860FA309D90483463905CD8EA309D9048E
:1029400023800D00C646F3A6068001000100130592
:1029500080FA03463905930639051D8A631C9629BA
:102960007336048013768608B2CC0100010013068A
:1029700080FA23809D002380CD000100010003C662
:1029800006001376F60D2380C60003C60600136604
:1029900006022380C600835609051166D18E2318CE
:1029A000D904835609052166D18E2318D9042380C2
:1029B0000D00E646F3A6068001000100130680FA2A
:1029C0008346390593F60602638006268346390559
:1029D000130C3905A18AFDDA081897000000E7807A
:1029E000A06BF336048093F68608B6D00100010090
:1029F000930680FA23809D002380DD000100010002
:102A000083460C00116693F6F60D2300DC00834626
:102A10000C0093E606022300DC0083560905D18EE4
:102A20002318D904835609052166D18E2318D904A9
:102A300023800D008656F3A60680010001001306D0
:102A400080FA8346390593F60602638A0620834698
:102A50003905A18AEDFE97F0FF1FE780C0632A8C3D
:102A600097F0FF1FE7802063E30C85FF835609057D
:102A700011664255D18E2318D90497000000E780D3
:102A800060638346390513063905A18AFDDAF336FA
:102A9000048093F68608B6D401000100930680FAFC
:102AA00023809D002380DD00010001008346060095
:102AB00093F6F60D2300D60023800D00A656F3A64C
:102AC0000680010001008356090503462905D24707
:102AD000B376DA003306CA021305800C9355F6412B
:102AE0003696330DF6408257333CD6002E9C333653
:102AF000A601330CFC40330CCC40330885039256BE
:102B00004E86B335A5033305A503C29597C00100D2
:102B1000E780E0E363468001631E0C16630C0D162C
:102B2000130615003335A6002E959356F5013696FB
:102B3000B335D600AA959396F50105828585D18E89
:102B40006346B000639D051A638B061A0356C902DB
:102B500015823305D6003336C500B2956348B00000
:102B6000639105241306F00F637DA622894663F363
:102B7000561593078008F3B7078093F78708BED6EA
:102B80000100010037170040930770052300F70488
:102B9000930780FA2300F704010001008356C7025F
:102BA00089678117D58FC207C1832316F7022300D7
:102BB0000704B657F3A7078001000100FA506A54D2
:102BC000DA544A59BA592A5A9A5A0A5BFA4B6A4C49
:102BD000DA4C4A4DBA4D296182801308F5FF33352E
:102BE000A800FD152E951356F5013298B336C8008E
:102BF000AA9695B9F336048093F68608B6CA010002
:102C0000010023809D002380AD0001000100834668
:102C10003905CD8EA309D90423800D00D646F3A62D
:102C200006800100010035B3F336048093F6860870
:102C3000B6CE0100010023809D002380CD0001005D
:102C400001008346390593E60602A309D9042380CF
:102C50000D00F646F3A606800100010095B3F33699
:102C6000048093F68608B6D20100010023809D00FF
:102C70002380CD00010001008346390593E606025A
:102C8000A309D90423800D009656F3A606800100FF
:102C9000010045BB9306F5FF33B5A600FD152E9543
:102CA0009355F501AE96B3B5B600AA951396F50106
:102CB000858269B5F336048093F68608B6D801009C
:102CC0000100930680FA23809D002380DD0001002F
:102CD00001008356C9020566011693F6F60FD18EE0
:102CE000C206C1822316D90223800D00C656F3A660
:102CF000068001000100850A93FAFA0F95B233E6C7
:102D0000B60045C20356C9023305D0403338A0008F
:102D1000B305B040B385054115826345B000D1E1EC
:102D20006371A608894663F0560593078008F3B7D8
:102D3000078093F78708BEDA01000100B71700404B
:102D4000130770052380E704130780FA2380E70444
:102D50000100010003D7C7027D8B2396E702238081
:102D60000704D65781BDF336048093F68608B6DC97
:102D700001000100930680FA23809D002380DD007E
:102D8000010001008356C9020566011693F6F60F8D
:102D9000D18EC206C1822316D90223800D00E656C9
:102DA000B9B793078008F3B7078093F78708BEDEAB
:102DB0000100010037170040930770052300F70456
:102DC000930780FA2300F704010001000356C702AD
:102DD00093975600B297C207C1832316F7022300C8
:102DE0000704F657C1BB914763EEB70217D701003E
:102DF000130707548A05BA959C41BA978287B7177B
:102E0000004003A7470B1345F5FF698F23AAE70A84
:102E100003A7070B698F23A8E70A03A7070A798D81
:102E200023A0A70A8280B717004083A6470B134749
:102E3000F5FFF98E23AAD70A83A6070B558D23A881
:102E4000A70A83A6070A758F23A0E70A8280B7170F
:102E5000004003A7470B498F23AAE70A03A7070BE4
:102E60001345F5FF45BFB717004083A6470B13472F
:102E7000F5FF758F23AAE70A03A7070A598D4DB7F7
:102E8000B717004003A7470B498FEDB7914763EE93
:102E9000B70217D701001307E74A8A05BA959C4184
:102EA000BA978287B717004003A7470D1345F5FF70
:102EB000698F23AAE70C03A7070D698F23A8E70CE6
:102EC00003A7070C798D23A0A70C8280B7170040B9
:102ED00083A6470D1347F5FFF98E23AAD70C83A6C7
:102EE000070D558D23A8A70C83A6070C758F23A06B
:102EF000E70C8280B717004003A7470D498F23AA2C
:102F0000E70C03A7070D1345F5FF45BFB7170040B2
:102F100083A6470D1347F5FF758F23AAE70C03A778
:102F2000070C598D4DB7B717004003A7470D498FC0
:102F3000EDB7797122D43714004026D24AD0035914
:102F400024028354040206D64209C2044ECE52CC57
:102F500056CA13590901C1802DE11379F9F793F489
:102F6000F49F4209C20413590901C18093078008E4
:102F7000F3B7078093F787083EC401000100930769
:102F800070052300F404930780FA2300F404010081
:102F90000100231124032310940223000404A247F8
:102FA000F3A7078001000100B25022549254025945
:102FB000F249624AD24A45618280B7F507008146EC
:102FC0003000B105194597000020E7808081A247B5
:102FD00013972701E34A07FC1369090893E40440A7
:102FE00093098008F3B7098093F787083EC0010072
:102FF0000100930A700523005405130A80FA230088
:10300000440501000100231124032310940223002E
:1030100004048247F3A7078001000100294597F0C7
:10302000FF1FE7802031F3B9098093F989084EC268
:1030300001000100230054052300440501000100A4
:103040008357040293E707202310F40223000404AB
:103050009247B9B7B7170040884742054181937737
:10306000050491EB9377F5013755E80113050580C9
:103070003345F50282809377050C130700046397AC
:10308000E7009377F50137459C1CCDB72165130503
:1030900005D0828037E700E01C435443A183E20659
:1030A000D58F1CC1FD572320F7182322F7188280E3
:1030B00013178500B7E700E023A0E710618123A282
:1030C000A7108280B7F700E08847CC47828081470D
:1030D00037370040A14663C4C7003285828003456C
:1030E000B740E38EA6FE3385F5000345050085074E
:1030F0002304A740CDB797070020938727EF9C4371
:10310000173700201307872B3E95636EE5001737AE
:1031100000201307273F6368A70017070020232715
:10312000A7EC3E858280FD57EDBF8280411122C40D
:1031300006C62A8497000000E78000F22947B307FB
:10314000E502B2408D83B3D7870222449507B3D7F7
:10315000E70237370040C207C1832316F700410159
:103160008280411137150E0006C697000000E780E7
:1031700020FCB7370040130770F82381E7000D47A4
:10318000A381E70013070004A380E7000547238716
:10319000E700B24041018280373700408347270073
:1031A0001A0593F7F703C98F93F7F70F2301F70079
:1031B0008280B737004003C7170019C9D98DA38093
:1031C000B70003C70700136787002380E7008280EA
:1031D00093C5F5FFF98DA380B7008280AE872A875B
:1031E000B736004021463738004089E71703000012
:1031F0006700E3F383C8B600E30916FF05078348B9
:10320000F7FFFD17C20723041801C183F9BF41115D
:1032100022C406C62A8497000000E780E0E329471D
:10322000B307E502B2408D83B3D7870222449507E6
:10323000B3D7E70237370040C207C1832316F740F0
:1032400041018280716541111305052006C6970072
:103250000000E78000FCB7370040130770F82381B7
:10326000E7400D47A381E74013070004A380E74030
:1032700005472387E740B24041018280CC4141119C
:1032800006C6328503C6150083C5050022064D8E8D
:1032900042068D654186138875A2630C0611634B47
:1032A000C804138845A26300060D634AC8009385CD
:1032B00035A26301B6082390060029464DA0138865
:1032C00055A26305060D938565A2E316B6FE8D45EE
:1032D0001D4663E6E5081146198E63F3C7003E8676
:1032E000B7E704002390C600FC4797D501009385FB
:1032F000A5079DA0138895A263030611634E060DD2
:103300001388A5A263000613938505A5E315B6FAF5
:1033100099451D4663E5E504198E63F3C7003E86B3
:10332000B7E704002390C600FC479705002093856B
:1033300025D61DA09D451D4663E3E5022146198E55
:1033400063F3C7003E86B7E70400FC472390C6003E
:103350009705002093858534BA9582970146B2403F
:10336000328541018280AD451D46E3EAE5FE3146E6
:10337000198E63F3C7003E86B7E704002390C600AA
:10338000FC4797D501009385A500F9B7B1451D46C7
:10339000E3E7E5FC3546198E63F3C7003E86B7E7E1
:1033A00004002390C600FC4797D50100938545FF94
:1033B00065B78D451D46E3E4E5FA1146198E63F3C2
:1033C000C7003E86B7E704002390C600FC4797D5A8
:1033D0000100938525FA49B78D451D46E3E1E5F8DF
:1033E0001146198E63F3C7003E86B7E704002390A9
:1033F000C600FC4797D50100938545FCB1BFA545A4
:103400001D46E3EEE5F42946198E63F3C7003E86B8
:10341000B7E704002390C600FC4797D501009385C9
:1034200025F61DBFB5451D46E3EBE5F23946198E7D
:1034300063F3C7003E86B7E704002390C600FC474D
:1034400097D50100938545F101BFB7E7040003A3B9
:103450000713970600209386A6C24146A545170587
:1034600000201305E5B802832D455DE703C505007F
:103470000947631FE50803A84500411106C6034735
:10348000180032850346080022074168518F9308CF
:1034900028FE6307170563E9E800051863030703BF
:1034A00023900600294591A8130648FE630AC70425
:1034B0001518E31707FF15463E87637BF60015478F
:1034C00001A8130600023E876374F600130700028A
:1034D000B7E704002390E600FC471316070111A884
:1034E0003E8691C30546B7E70400FC472390C6001B
:1034F0004206CC45418282970145B240410182801B
:10350000130600083E87E375F6FC13070008C9B7E9
:103510002390060005458280828041677917630405
:10352000E504411122C406C685472A84639FF5003D
:10353000B7E7040022852244B24003A3871397050E
:1035400000209385E52F4101028389476399F500A7
:10355000B7E7040083A7070B8545829771D9B2406E
:103560002244410182808280797126D252CCAE847D
:103570002A8A97D50100938565E617D501001305C2
:1035800065E806D63AC622D44AD0368432894ECE71
:1035900097C00100E780E086A28517D501001305DA
:1035A00065E797C00100E780C085294597C0010005
:1035B000E780008A83C7840093F70702F9E383C991
:1035C00004008947054532476396F908D44083C70C
:1035D000160083C60600A207D58FC166138616FEA5
:1035E000638CC7028D16638FD7068D6693862690EF
:1035F00029456391D706B7E70400A286225403A3A6
:103600004714B250F2494A86A6850259925452850F
:10361000624A8547456102832D450DEF93070002FD
:10362000354563E98702B7E70400FC47C844130641
:103630000002CA8582978149970700209387072156
:103640009C43014581CB9C4391C74E852286CA8508
:1036500082970145B250225492540259F249624A6B
:10366000456182802D457DF79307700F3545E3E373
:1036700087FEB7E70400FC47C8442286CA858297C4
:1036800065BF2145C1BF411122C437E4040083272F
:10369000841326C2AA84416506C697050020938537
:1036A000251A7D1582978327C40A17050000130584
:1036B00005E78588829795C0032304132244B2400E
:1036C000924497060020938626AE4146C5451705CD
:1036D00000201305659C41010283B24022449244BC
:1036E00001454101828019C59707002023A0A71634
:1036F00001458280454582801147636AA70A97D6B3
:103700000100938666CC0A0536951841411106C61C
:103710003697AE87B2850287130700026145639D25
:10372000E700B7E70400FC47130600021705002076
:10373000130545F782970145B24041018280054754
:103740006145E39BE7FEB7E70400FC470546170524
:103750000020130525F7F9BF1307700F6145E39D9E
:10376000E7FCB7E70400FC471306700F17050020BD
:10377000130585F5C1B7130700086145E39EE7FA15
:10378000B7E70400FC4713060008170500201305DF
:1037900025034DB715476145E390E7FAB7E7040005
:1037A000FC471546170500201305C50961B70945F3
:1037B0008280411126C2B7E4040083A7C41322C447
:1037C0004AC006C62E8497050020938565072A897E
:1037D0008297058905C5970700209387E78B83D7D4
:1037E000A70BA28503A3440D2310F4002244B2408A
:1037F00092444A850249014641010283B240224473
:103800009244024949454101828097070020238163
:1038100007049707002023AF0702B717004003A74C
:10382000070CB706C0FFFD16758F23A0E70C03A792
:10383000070DB7064000558F23A8E70C03A7070C18
:103840003D9B23A0E70C03A7070D1367070123A8DF
:10385000E70C8280B717004003A5470C83A7470CED
:10386000598113451500C18B058999E3136525001E
:103870009707002083C7C7FD6380A7029707002032
:103880002388A7FC11C9970700209387A7FC03A3EF
:1038900007006303030002838280114517F3FFFFD3
:1038A000670063C8011122CC06CE3714004026CA37
:1038B0004AC84EC652C483447405034AB4058349BA
:1038C00084050349940597F0FFFFE780A0A0834794
:1038D000A40593F4F40F137AFA0F93E71700230D5E
:1038E000F40493F9F90F1379F90FB717004003C7E0
:1038F000A705058B6DFF03D5C705A38D4705238C51
:103900003705A38C2705A38B9704F2406244D24469
:103910004249B249224A05618280411193970501CB
:1039200022C406C626C2C1872E8463DC0700B7E422
:103930000400FC54829719C1BC5482972165218DE3
:1039400015A893F7150013C515008DE793F725000B
:103950009DC797000000E78020F0B7E70400BC4F48
:103960001306000A894517050020034525EF8297B5
:1039700013452400B240224492444101828093972F
:10398000250163D80702B7E4040083A7C41E829709
:1039900097000000E780A0F0BC4C375607001306E4
:1039A0000630896517050020034545EB82970965B8
:1039B00079B7939715010145E3DE07FA17D50100A2
:1039C000130545AD97B00100E780805BB7E70400C1
:1039D000BC4F13060064916517050020034505E8F8
:1039E00082971165A9BF1D71A2CC37E404005C5C0D
:1039F000485886CE494697D50100938525A58297DC
:103A000011E917D501001305A5A597B00100E780BE
:103A1000205701A0B7F600E0795798CAFD57DCCAD5
:103A20000567B7E700E023A0E7101306F00290C295
:103A300023A0E718010001003707002018471306EC
:103A4000000481459706002023A8E6E04157A38A99
:103A5000E7403C4408088297970700209387077C3B
:103A60003EC8856713870740938757D1231AE10023
:103A70002312F1021307B00F97F7FFFF9387C76474
:103A80002310E1023ED81547970700009387C7E14E
:103A9000B7F50700A30FE1003EDC054797070000DC
:103AA0009387E7DF81463000E10519452301E102F4
:103AB0003EDE97F0FF1FE780C0D218088147994685
:103AC00030003E960346060085070507A30BC70096
:103AD000E398D7FEC24791C70357410185676373D7
:103AE000F70001A0B7E7040083A7470A08088297F8
:103AF000AA8511C917D501001305C59797B0010014
:103B0000E780203001A0F6406644256182804111A3
:103B100026C2B7E4040083A7040806C622C417051A
:103B200000001305C5DF829717040020130404D397
:103B30002300A40097000000E780800297000000A7
:103B4000E780E0CC03450400224403A38405B2408F
:103B5000924413060032896541010283797106D6C9
:103B600022D413078008F337078093F787083EC2F3
:103B700001000100B7170040930570052380B704CA
:103B8000130680FA2380C7040100010083C6F702F0
:103B900093F6A60FA387D702238007049246F3A6C5
:103BA00006800100010073370780137787083AC445
:103BB000010001002380B7042380C7040100010035
:103BC00003C7F70213672700A387E70223800704D0
:103BD000A247F3A7078001000100054597E0FFFF1A
:103BE000E780807297000000E78060CB0147814644
:103BF0008147054685451305407E97E0FFFFE78036
:103C0000807537E404003C44680051468145829742
:103C1000B707C0A83EC8B787E803938707D03ECA56
:103C200097E7FF1F9387A7793EC67C586800829765
:103C3000B250225445618280411197D5010093858D
:103C4000A5E717C501001305E57B06C697B001007F
:103C5000E780201B17D501001305C5FD97B00100B3
:103C6000E780201AB2402945410117B301006700DF
:103C7000231E411197D50100938545E517C5010025
:103C80001305457806C697B00100E780801717D561
:103C900001001305E5F897B00100E7808016B240F7
:103CA0002945410117B301006700831A411122C45D
:103CB00006C6834705002A849DC797D501009385D2
:103CC000A5E617C501001305E57397B00100E7806D
:103CD00040134C4017D501001305C50A97B00100E9
:103CE000E78020123DA058410DEF97D50100938544
:103CF000A5E317C501001305E57097B00100E78043
:103D0000401017D501001305650997B00100E78041
:103D1000400F2244B2402945410117B3010067001A
:103D20002313A1679386D7036313D70297D50100A6
:103D3000938585DF17C501001305C56C97B0010099
:103D4000E780200C17D50100130545067DBFED0760
:103D500097D50100938545DD17C501001305856AD8
:103D6000631BF70097B00100E780A00917D5010099
:103D70001305050559BF97B00100E78080084C4046
:103D800017D501001305C50591BF411197D5010055
:103D9000938505D517C501001305C56606C697B0FE
:103DA0000100E7800006B2402945410117B3010038
:103DB0006700030A797122D426D24AD02E842A8938
:103DC000B28481457146480006D697E0FFFFE78040
:103DD000003497F7FF1F9387275EDC4783D70700E0
:103DE000231421012313F10097500000E780C01C29
:103DF0008547A305F1009307401F2305A1003EC698
:103E00002686FD57A2854800230AF100975000003E
:103E1000E780601DB250225492540259456182805D
:103E2000411197270020239E078E97170020238794
:103E3000077E06C6170700200347C72E9307F00A20
:103E40006315F7029307F0F889451705002013055D
:103E5000652D170700202307F72C97070020A38361
:103E6000072C97600000E78060D697600000E7802D
:103E7000200397600000E780600481453705040057
:103E80009707002023A607289707002023810728EB
:103E9000970700202390072097070020239E071CE8
:103EA00097070020239307269707002023940726CF
:103EB00097300000E7802068014597600000E780A8
:103EC000E0D9D147170700202312F724B7E70400F1
:103ED000BC4F13060014894517050020034585983B
:103EE000829797D50100938525C217C50100130558
:103EF000655197B00100E780C0F09705002083D599
:103F0000E52017D501001305E5F397B00100E78020
:103F100040EFB2402945410117B30100670043F368
:103F20004111814617F6FF1F1306464685451705C2
:103F300000200355251406C697C00000E780205EC8
:103F400015C997D501009385E5BC17C50100130578
:103F5000654B97B00100E780C0EA17D50100130553
:103F600065DE97B00100E780C0E9294597B0010000
:103F7000E78000EE97D501009385C5B917C501000C
:103F80001305454897B00100E780A0E717D5010069
:103F9000130585DC97B00100E780A0E6294597B0BE
:103FA0000100E780E0EA97F7FF1F9387E740DC47CF
:103FB000054797D501009385E5B52390E70017C520
:103FC00001001305254497B00100E78080E317D571
:103FD00001001305A5D997B00100E78080E2B24047
:103FE0002945410117B30100670083E6011122CC86
:103FF00006CE26CA4AC84EC693F715002E84B5CB06
:1040000097000000E78000F2930710F817070020E0
:10401000230AF7109707002083D78705170700208A
:10402000A302F7109145A183170500201305850F02
:10403000170700202309F70E97070020A385070E16
:1040400097600000E78080B8B7E70400BC4F130614
:10405000001493050010170500200345A5808297E2
:1040600013451400F2406244D2444249B24905610A
:10407000828093F70510B1C3054597600000E78083
:10408000E0BD171500200355C56997600000E78063
:10409000608997200000E780603D9707002083C774
:1040A000B71789E797600000E78080DF976000001E
:1040B000E780C0E01345041075B793F72500E9CFFA
:1040C000170700200357870469C7AD64B71900407C
:1040D0009384A4AA23A09900970600209386460300
:1040E000944297D701009387A7D71706002003466D
:1040F0000602814517D50100130585D7977000008A
:10410000E780A05D23A0990097F7FF1F239AA71AC5
:104110002A8941C197D50100938585A617C501005D
:104120001305452E97B00100E780A0CDCA8517C5BD
:1041300001001305E54497B00100E78080CC2945D4
:1041400097B00100E780C0D097070020239007FCBC
:10415000930710F8170700202306F7FC97070020A5
:1041600083D707F117070020A30EF7FAA1831707DB
:104170000020230AF7FA91458D4717050020130503
:1041800065FA17070020A300F7FA97600000E780A0
:10419000E0A313452400F9B593F74500D1C397D5A3
:1041A00001009385E59D17C501001305A52597B06E
:1041B0000100E78000C517C501001305253E97B033
:1041C0000100E78000C4294597B00100E78040C89E
:1041D000930720F8170700202306F7F4970700201D
:1041E00083D747EB17070020A30EF7F2A183170729
:1041F0000020230AF7F2854717070020A305F7F2EE
:1042000097500000E78040F217050020130585F164
:10421000914597600000E780609B1345440099B585
:1042200093F78500A9C797D501009385659517C5B4
:1042300001001305251D97B00100E78080BC17C55C
:1042400001001305E53697B00100E78080BB2945E2
:1042500097B00100E780C0BF97070020239807EAC6
:1042600097700000E780405713458400E5BB93F743
:104270000501D1C38545170500200355A5E19760C9
:104280000100E780000D97D501009385658F17C564
:1042900001001305251797B00100E78080B617C508
:1042A00001001305253297B00100E78080B529454C
:1042B00097B00100E780C0B9930730F817070020D6
:1042C0002302F7E69707002083D7C7DC17070020F3
:1042D000A30AF7E4170500201305C5E4A1838D4563
:1042E000170700202301F7E497600000E780008EA5
:1042F0001345040185BB93F70502D1C797D501008B
:104300009385058817C501001305C50F97B00100F7
:10431000E78020AF17C501001305052D97B00100F8
:10432000E78020AE294597B00100E78060B293078F
:1043300040F8170700202307F7DE9707002083D7F0
:10434000A7D317070020A30FF7DCA18317070020CE
:10435000230BF7DC854717070020A306F7DC970738
:104360000020239B07D097500000E780E0DB170573
:104370000020130525DB914597600000E78000854C
:1043800013450402C5B193F70504FDC397C50100A9
:104390009385057F17C501001305C50697B0010079
:1043A000E78020A617C501001305852597B00100F9
:1043B000E78020A5294597B00100E78060A997070D
:1043C000002083C727D61307700A6386E706130702
:1043D000800A638CE7081307600A6393E704930776
:1043E00060F817070020230FF7D29707002083D724
:1043F000C7D117070020A307F7D2A1831707002012
:104400002303F7D2854717070020A302F7D2B1454F
:1044100017050020130505D197500000E780007BA9
:1044200097500000E78040D0134504049707002010
:10443000239D07CC05B9930770F8170700202303C5
:10444000F7CE9707002083D747CC17070020A30B90
:10445000F7CCA183170700202307F7CC8547170760
:104460000020A303F7CC994565B7930780F8F1B70F
:1044700093F705080145E38707BE97C501009385BB
:10448000257017C501001305E5F797B00100E78017
:10449000409717C501001305251897B00100E78064
:1044A0004096294597B00100E780809A9307A0F8CD
:1044B000170700202308F7C69707002083D787C572
:1044C00017070020A300F7C6A18317070020230CBD
:1044D000F7C4854717070020A307F7C497070020F4
:1044E000239A07C297500000E78000C417050020F8
:1044F000130545C3914597500000E780206D134593
:1045000004088DB6411122C497C501009385056347
:104510002A8417C501001305E5EE06C697B0010011
:10452000E780208E4C4017C501001305257F97B00A
:104530000100E780008D294597B00100E780409198
:10454000034704009307F00F631FF70297C50100AC
:104550009385C55E17C501001305C5EA97B0010034
:10456000E780208A4C4017C501001305257C97B0D1
:104570000100E78000892244B2402945410117B378
:1045800001006700E38CB240224441018280411166
:1045900022C426C22A84AE8417C50100130585E60D
:1045A00097C501009385455506C697B00100E78081
:1045B000408517D501001305658797B00100E78096
:1045C0004084294597B00100E780808897C50100A5
:1045D0009385855297070020239E87A817C5010061
:1045E000130545E2054497070020239397A89707F2
:1045F0000020239087A8971700202394971297B044
:104600000100E78000809715002083D5851117D51C
:1046100001001305258297A00100E780807E2945CF
:1046200097B00100E780C08297170020238887FE9B
:1046300097F7FF1F938747D8DC4717F5FF1F034500
:10464000652203D70700C167FD17631EF700B7E7B0
:10465000040003A387051306000A85452244B240DF
:10466000924441010283B7E7040003A387051306C0
:10467000001493050010DDB7B1C1411122C417C564
:104680000100130525D82E8497C5010093850546A2
:1046900006C697A00100E780C076A28517C5010075
:1046A0001305057897A00100E780A0752244B24069
:1046B0002945410117A30100670083798280011118
:1046C00022CC37E404005C5C06CE26CA354697C58A
:1046D00001009385655717D5010013056529829759
:1046E00011E917C501001305A5D797B00100E780B0
:1046F000208901A097F7FF1F938787173EC4B7F55E
:104700000700856793870780814617F6FF1F13060A
:10471000A615E10519453EC697E0FF1FE780600C2E
:104720007C44194697F5FF1F938505141705002053
:10473000130585968297340017F6FF1F1306C612DD
:1047400097D501009385059B17D501001305059C9E
:1047500097700000E78060CDAA8421C197C5010051
:104760009385054117C501001305C5C997A0010030
:10477000E7802069A68517C501001305E54D97A0C0
:104780000100E7800068294597A00100E780406CA0
:10479000F2406244D2440561828097E00000E780E5
:1047A000403317C501001305254297600000E780DC
:1047B00080C197B00000E780808797600100E780A4
:1047C00000EC17F5FF1F1305A5BB97600100E780FC
:1047D000A0D417C501001305254097600100E780AC
:1047E00080ECAA8497600000E780C0279710010042
:1047F000E780E0C397800100E780005D97800000BC
:10480000E780A08397700000E780C09D974001007B
:10481000E780408597C501009385853517C5010060
:10482000130545BE99C897A00100E780805DA68565
:1048300017C501001305854499B797A00100E780CB
:10484000405C17C501001305A54597A00100E7804E
:10485000405B294597A00100E780805F9730010009
:10486000E780206197F00000E780E07F6DC5854517
:104870003705040097300000E780E0CB97C50100C2
:104880009385052F17C501001305C5B797A0010033
:10489000E780205717C501001305054297A00100C6
:1048A000E7802056294597A00100E780605A97F7D6
:1048B000FF1F9387E79F83D7070017170020231256
:1048C000F7E6854717170020230AF7D497F7FF1F4D
:1048D000938787AEDC4703D70700C167FD176316D0
:1048E000F70097F0FFFFE780E06397700000E78034
:1048F000E0FE8567938707E33E9597700000E780A9
:10490000A0FE97200000E78060B617150020035531
:1049100045E197500000E780E00005459750000012
:10492000E780C03397500000E780405997C50100E9
:104930009385052417C501001305C5AC97A0010098
:10494000E780204C17C501001305053C97A0010026
:10495000E780204B0DBDD14797C5010093854521C8
:1049600017C50100130505AA17F7FF1F2310F77AD3
:1049700097A00100E780E04817D601001306468A99
:1049800097F5FF1F83D5857817C5010013050535F9
:1049900097A00100E780E046294597A00100E78045
:1049A000204B3C4C1306000A894517F5FF1F0345B1
:1049B00065EB8297014597500000E780202ABDB73C
:1049C000411122C437E404008327041A06C68297E3
:1049D00097500000E780C0F88327040817F5FFFF11
:1049E00013050561829797F7FF1F238DA7E617F53B
:1049F000FF1F1305659C97500000E780A0A9224483
:104A0000B2404101170300006700A3CBB7E70400E1
:104A1000FC471171A2DDCAD986DFA6DBCED72E8472
:104A200032892E86AA8517F5FF1F1305A56F829779
:104A300017F7FF1F1307076F8347070093068002CE
:104A40009387E70793F7F70FE3ECF610BA898A0725
:104A500017C70100130747A4BA979C43BA978287E8
:104A60008D4797C501009385E51217C50100130511
:104A70006599630FF40097A00100E780803817C59F
:104A800001001305E5CF97A00100E7808037BDA4A2
:104A900097A00100E780E03617C501001305C5CFD8
:104AA00097A00100E780E035294597A00100E78045
:104AB000203A930720F8114697F5FF1F93858566E6
:104AC0004A8517F7FF1F230FF76497F7FF1FA38C83
:104AD000076497F0FFFFE780202E2A841DC997C541
:104AE00001009385250B17C501001305A59197A01B
:104AF0000100E7800031A28517C50100130585CDAF
:104B000097A00100E780E02F294597A00100E780EA
:104B1000203497C501009385E50717C501001305EB
:104B2000658E97A00100E780C02D17C50100130511
:104B3000A5CB97A00100E780C02C294597A00100D4
:104B4000E78000314165930730FA054697F5FF1F6E
:104B50009385455D7D1517F7FF1F2305F75C97F0DB
:104B6000FFFFE78060252A841DC997C50100938552
:104B7000650217C501001305E58897A00100E780CD
:104B80004028A28517C501001305C5C497A00100E0
:104B9000E7802027294597A00100E780602BB7E731
:104BA0000400BC4F0566130606C8A14517F5FF1F94
:104BB000034545CB8297FE506E54DE544E59BE5984
:104BC0001161828091476303F40297C501009385C8
:104BD00065FC17C501001305E58297A00100E78079
:104BE000402217C50100130565C371BDB7E7040076
:104BF000FC4F914517F5FF1F0345C5C6829797C522
:104C00000100938525F917B501001305A57F97A02D
:104C10000100E780001F17C501001305E5C197A03B
:104C20000100E780001E294597A00100E78040228F
:104C300097400000E780404F914535A485476303C6
:104C4000F40297C501009385E5F417B5010013053B
:104C5000657B97A00100E780C01A17C50100130506
:104C600025BF15B597F7FF1F23962743B7E7040025
:104C70000566BC4F130606C8C1450DBF8D476303CB
:104C8000F40297C501009385E5F017B501001305FF
:104C9000657797A00100E780C01617C501001305CE
:104CA000E5BCD5B3930740F8114697F5FF1F9385F0
:104CB00065474A8517F7FF1F2306F74697F7FF1F3B
:104CC000A383074697F0FFFFE780000F2A84E304E1
:104CD00005EE97C501009385E5EB17B501001305B7
:104CE000657297A00100E780C011A28517C5010079
:104CF000130545AE97A00100E780A010294597A0B5
:104D00000100E780E01445BD9147E31CF4F6B7E7E6
:104D10000400FC4F9305000217F5FF1F034585B4FF
:104D2000829797C501009385E5E617B50100130545
:104D3000656D97A00100E780C00C17C50100130541
:104D400065B4F1BD894763E3870297C50100938588
:104D500065E417B501001305E56A97A00100E78037
:104D6000400A17C50100130525B331BB97F4FF1F97
:104D700083C4643B97F7FF1F83C7D73A97C50100E9
:104D8000938545E1A20417B501001305A567DD8CE5
:104D900097A00100E780E006A28517C50100130572
:104DA000E5B097A00100E780C005C204294597A09F
:104DB0000100E780E009C1849305D4FF93960401C4
:104DC000C1824A8693F5F50F17F5FF1F1305B53518
:104DD00097200000E780E079E35F90DC930750F8CC
:104DE00017F7FF1F2300F73483C73900228697F592
:104DF000FF1F9385253385074A8517F7FF1FA304F7
:104E0000F73297F0FFFFE78020FB2A84E30505DAFD
:104E100097C50100938505D817B501001305855E78
:104E200097A00100E780E0FDA28517C501001305EA
:104E300025FEC9B5894763E3870297C501009385BD
:104E400065D517B501001305E55B97A00100E78064
:104E500040FB17C50100130525A735B19740000099
:104E6000E780802CA28517F5FF1F1305A52B97500F
:104E70000000E780A0D581B38D476303F40297C596
:104E80000100938525D117B501001305A55797A0FB
:104E90000100E78000F717C501001305A5A4E5B6DA
:104EA000B76602000146B7750200054597E0FF1F8F
:104EB000E7802093930760F817F7FF1F2304F72676
:104EC00097F7FF1FA38107269307000617F7FF1F19
:104ED000230CF724894717F7FF1FA307F72497F739
:104EE000FF1F2384072497F7FF1FA3800724C147D0
:104EF00017F7FF1F230CF722930720F917F7FF1F5F
:104F0000A306F722314697F7FF1FA382A72297F542
:104F1000FF1F938525214A8597F7FF1F23890720C7
:104F200097F0FFFFE78040E92A84E30605C897C5AC
:104F30000100938525C617B501001305A54C97A060
:104F40000100E78000ECA28517C501001305059B51
:104F500055B3B1476303F40297C50100938585C338
:104F600017B501001305054A97A00100E78060E925
:104F700017C501001305459A39B6B7E70400FC4F81
:104F80009305000417F5FF1F0345C58D82979740D1
:104F90000000E7806019B145F9B5914763E38702E6
:104FA00097C50100938505BF17B501001305854519
:104FB00097A00100E780E0E417C50100130585977D
:104FC000D9B497F4FF1F83C4241697F7FF1F83C734
:104FD0009715A204DD8C8E04B77702006D14BE9481
:104FE0002286A68517C501001305059697A0010026
:104FF000E78020E1B7E70400FC47228697F5FF1F12
:10500000938595122800829793160401C18230007F
:10501000A685094597D0FF1FE780A07C2A8409C98F
:1050200017C501001305059497A00100E78040F51E
:10503000930770F8194697F5FF1F9385A50E4A85CB
:1050400017F7FF1F2300F70E97F7FF1FA38E870C9C
:1050500097F0FFFFE78040D62A84E30E05B497C59A
:105060000100938525B317B501001305A53997A055
:105070000100E78000D9A28517C501001305858FBF
:1050800095B99947630BF41297C50100938585B0D4
:1050900017B501001305053797A00100E78060D61A
:1050A00017C501001305858EF9BA914763E387029E
:1050B00097C50100938505AE17B50100130585342A
:1050C00097A00100E780E0D317C501001305858D87
:1050D0005DBA97F4FF1F83C4240597F7FF1F83C7AA
:1050E0009704A204DD8C8E04B77702006D14BE9481
:1050F0002286A68517C501001305058C97A001001F
:10510000E78020D0B7E70400FC47228697F5FF1F11
:10511000938595012800829793160401C18230007F
:10512000A6850D4597D0FF1FE780A06B2A8409C98B
:1051300017C501001305058A97A00100E78040E428
:10514000930780F8194697F5FF1F9385A5FD4A85BB
:1051500017F7FF1F2308F7FC97F7FF1FA38687FCAD
:1051600097F0FFFFE78040C52A84E30605A497C5B2
:105170000100938525A217B501001305A52897A066
:105180000100E78000C8A28517C501001305C58589
:1051900095B699476303F40297C501009385859FEF
:1051A00017B501001305052697A00100E78060C52B
:1051B00017C501001305C584F9B0B7E70400FC4F1B
:1051C0009305000417E5FF1F0345C56982979740C3
:1051D0000000E78060F5994579B18D476303F402DB
:1051E00097C501009385059B17B50100130585211F
:1051F00097A00100E780E0C017C501001305C58135
:1052000059B017C501001305258297A00100E7805A
:1052100020D71305C01297D0FF1FE78080120145E9
:1052200097E0FFFFE78040E70D4597100000E7801B
:10523000A09E294597D0FF1FE780A01097D0FF1FA1
:10524000E78000018DBA99476303F40297C5010016
:105250009385459417B501001305C51A97A0010061
:10526000E78020BA17B501001305C57C29B817F7E8
:10527000FF1F034777EB97F7FF1F83C7E7EA220774
:105280005D8F9166BA96C2061166C1821306F6EF6B
:105290008D476365D60297E7FF1F9387E7119C4B05
:1052A00017F6FF1F034636E89386C7002DC203D6C4
:1052B000070069CA8907E39CD7FE89471307A0F84E
:1052C000114697F5FF1F9385E5E54A8597F6FF1F81
:1052D000238AE6E417F7FF1FA307F7E497F0FFFF21
:1052E000E78080AD2A84E308058C97C5010093858B
:1052F000658A17B501001305E51097A00100E78046
:1053000040B0A28517B5010013050574E5B203D6B8
:105310000700630EE60A8907E39BF6FE8D4779BF17
:1053200091476304F40297C501009385A58617B5DC
:1053300001001305250D97A00100E78080AC17B58B
:1053400001001305E5716FF00FF4B7E70400FC4F9F
:105350009305000817E5FF1F0345C5508297C9B89C
:1053600097C501009385058317B5010013058509CD
:1053700097A00100E780E0A817B501001305C56FED
:105380006FF06FF02390E70017E5FF1F1305C502CC
:1053900097300100E78060D397B501009385857F42
:1053A00017B501001305050697A00100E78060A569
:1053B00017B501001305456D97A00100E78060A4B3
:1053C000294597A00100E780A0A88147C5BD23908B
:1053D000070017E5FF1F130525FE97300100E78042
:1053E000C0CE97B501009385E57A17B50100130586
:1053F000650197A00100E780C0A017B50100130563
:10540000256A5DBF011122CC06CE26CA4AC8834751
:1054100005002A849DC797B501009385657317B56C
:105420000100130525FE97A00100E780809D4C40F8
:1054300017C501001305C5A497A00100E780609C73
:10544000D1A05841B707CF009387777D631BF7063C
:105450000359C500854704450356E50063FA270351
:1054600083C7040003C71400A207D98FC20771774E
:10547000C1871307C755639DE7006244F240CA85A0
:1054800026854249D244056117230000670043BCCA
:105490009707002083D7E728638AC700CA85268537
:1054A00032C697E0FFFFE780A0D332466244F24065
:1054B000CA8526854249D244056117F3FFFF67007C
:1054C0002355B707CC009387777D6317F70497B50B
:1054D00001009385E56717B501001305A5F297A0B4
:1054E0000100E78000921C448356E4008355C40009
:1054F00003C6070017C501001305059A97A0010010
:10550000E78020906244F240D24442492945056137
:1055100017A301006700C393B707CE009387777D79
:105520006304F70297B501009385856217B5010002
:10553000130545ED97A00100E780A08C4C4017C5EE
:1055400001001305E589CDBDF2406244D2444249D1
:1055500005618280B7E70400FC4741112E8606C62C
:1055600022C426C24AC02E842A89AA8517F5FF1FA5
:10557000130545BB829797B501009385656317B501
:105580000100130525E897A00100E780808797F5C3
:10559000FF1F83C525B917B501001305650997A03D
:1055A0000100E7800086294597A00100E780408A36
:1055B00097F4FF1F938404B783C704004147938780
:1055C000070693F7F70F6369F75A17B70100130738
:1055D000E7F68A07BA979C43BA9782879D47630785
:1055E000F40297B501009385A55C17B5010013057A
:1055F00065E197A00100E780C08017B501001305A1
:10560000A50397900100E780C07FA1AC97F7FF1F2B
:1056100083C757B1DDCB17F7FF1F0347D7B097F705
:10562000FF1F83C747B022075D8F97F7FF1F83C710
:10563000A7AFC2075D8F97F7FF1F83C7F7AEE207DB
:10564000D98F17F7FF1F2325F7AC83C7640097B5E1
:1056500001009385E55517B501001305A5DA17F785
:10566000FF1F2306F7AA97900100E780807997F73C
:10567000FF1F9387E7A98C4317F6FF1F034626A950
:1056800017B50100130505FD97900100E7806077CD
:10569000294597900100E780A07B97F7FF1FA38320
:1056A00007A82244B24092440249930700F817F732
:1056B000FF1F2309F7A69D4517F5FF1F130585A6B4
:1056C0004101174300006700635097600000E780C6
:1056D000202097F7FF1F2388A7A49357850017F76B
:1056E000FF1FA302F7A4935705012A8417F7FF1F92
:1056F000230CF7A293578501014517F7FF1FA30558
:10570000F7A297600000E780002197F7FF1F238E24
:10571000A7A097B501009385A54917B5010013050A
:1057200065CE97900100E780C06D17F6FF1F034616
:10573000C69FA28517B50100130545F3B1B7CD4744
:105740006303F40297B501009385854617B5010000
:10575000130545CB97900100E780A06A17B50100BB
:10576000130545F279BD97F7FF1F83C7C79CA207B2
:1057700017F7FF1F0347179CD98FC207C1876357CD
:10578000F00217F7FF1F2313F798B7E7040003A3EE
:1057900087051306000A89452244B2409244024913
:1057A00017E5FF1F0345050C41010283D147D1BF17
:1057B0008D476303F40297B501009385653F17B5E4
:1057C0000100130525C497900100E780806317B599
:1057D00001001305E5FA35B517F4FF1F0344A4943F
:1057E00097F7FF1F83C7179497B501009385453C32
:1057F000220417B501001305E5C05D8C97900100E8
:10580000E7802060A28517B50100130525E9979070
:105810000100E780005F294597900100E780406321
:105820000D4697F5FF1F9385E58F228597E0FFFFD3
:10583000E7808058AA8421C197B501009385453738
:1058400017B50100130505BC97900100E780605B68
:10585000A68517B501001305A5E597900100E7801F
:10586000405A2244B24092440249294541011793CB
:1058700001006700E35D97F7FF1F239D8780B7E76F
:105880000400116603A38705130606E8914529B7AE
:105890008D476303F40297B501009385653117B511
:1058A0000100130525B697900100E780805517B5D4
:1058B00001001305A5FBB1B317F4FF1F0344A48631
:1058C00097F7FF1F83C7178697B501009385452E6D
:1058D000220417B501001305E5B25D8C9790010015
:1058E000E7802052A28517B501001305A5DD97902A
:1058F0000100E7800051294597900100E78040555D
:105900000D4697F5FF1F9385E581228597E0FFFF00
:10591000E780804AAA841DC197B501009385452977
:1059200017B50100130505AE97900100E780604DA3
:10593000A68517B50100130525DA05B797E7FF1F00
:10594000239C8772B7E70400116603A3870513063B
:1059500006E89305000289B5894763E3870297B596
:1059600001009385E52417B501001305A5A99790BB
:105970000100E780004917B501001305E5F151B1B9
:1059800097E4FF1F83C4247A97E7FF1F83C79779A3
:1059900097B501009385C521A20417B50100130531
:1059A00065A6DD8C97900100E780A045A68517B518
:1059B00001001305E5D397900100E7808044294555
:1059C00097900100E780C048228697E5FF1F9385E6
:1059D0006575268597E0FFFFE780003E2A84630E09
:1059E000051A97B501009385A51C17B5010013058D
:1059F00065A197900100E780C040A28517B501001E
:105A0000130545D099BD854763F98718834519006B
:105A10002244B24092440249B335B00097E7FF1FD9
:105A20002384B76817B50100130505CF410117930B
:105A300001006700033DA2852244B24092444A859A
:105A4000024941011703000067004323994763039C
:105A5000F40297B501009385A51517B5010013054C
:105A6000659A97900100E780C03917B501001305CA
:105A700065FC41BE17E4FF1F0344E46A97E7FF1F7C
:105A800083C7576A97B5010093858512220417B51D
:105A90000100130525975D8C97900100E780603623
:105AA000A28517B501001305A5C897900100E780EE
:105AB0004035294597900100E7808039194697E5E0
:105AC000FF1F93852566228597E0FFFFE780C02EA4
:105AD000AA841DC197B501009385850D17B50100F6
:105AE0001305459297900100E780A031A68517B570
:105AF00001001305E5C495B397E7FF1F239C87605A
:105B0000B7E70400116603A38705130606E89305AB
:105B1000000859B1854797B501009385650917B508
:105B200001001305258E630BF40097900100E780B8
:105B3000402D17B501001305E5C1E1B497900100B0
:105B4000E780202C17B50100130545C2979001008E
:105B5000E780202B294597900100E780602F2244A1
:105B6000B2409244024997E7FF1F2391075A41012F
:105B700017630000670043C697B50100938545038E
:105B800017B501001305058897900100E78060278D
:105B900017B50100130545EEADB4B240224492445E
:105BA000024941018280411106C622C426C239C180
:105BB0002A8497E00000E780004BAA8411EDB7E744
:105BC0000400BC474146814522858297B240224469
:105BD000268592444101828041657D1597E0000051
:105BE000E7804049B7E7040001E9BC4741468145E9
:105BF000228582978144D9BF0347E501FC4793057D
:105C0000900819E393050003AA95414622858297DF
:105C100085446DBF411122C491462A8417E6FF1FB7
:105C20001306465E9D652D4506C697D0FF1FE7808B
:105C300040BBB7F7070003C70701A5476313F70089
:105C400001A09306001001469D65254597D0FF1FD2
:105C5000E78020B997E7FF1F2386875A2244B24086
:105C6000914617E6FF1F1306E6599D652945410138
:105C700017D3FF1F6700E3B61171CED7B7E9040051
:105C800083A7C904CAD917E9FF1F1309A949A2DDCF
:105C90002E8686DFA6DB2E84AA854A85829797E723
:105CA000FF1F83C727481307700A6385E710636DDA
:105CB000F7001307600A6385E704FE506E54DE5454
:105CC0004E59BE59116182801307800A6385E71619
:105CD0001307900AE393E7FE8D476306F41C97B51C
:105CE00001009385E52617A501001305A57197907E
:105CF0000100E780001117B501001305A52225A0BA
:105D00008D47630CF40297B501009385652417A5B0
:105D100001001305256F97900100E780800E17B5ED
:105D200001001305651997900100E780800D294552
:105D300097900100E780C01149B7854717B501006A
:105D40001305451917E7FF1F2300F7369790010049
:105D5000E7800023B7750200B766020001460545DB
:105D600097D0FF1FE780E0A7930760F817E7FF1FB2
:105D7000230AF73A97E7FF1FA387073A93070026FE
:105D800017E7FF1F2322F73AE5779387072117E7E5
:105D9000FF1F231DF738B14597E7FF1F23890738F9
:105DA00097E7FF1FA385A7384A8597000000E78083
:105DB000E01621B7914763E3870297B50100938509
:105DC000251917A501001305E56397900100E780E9
:105DD000400317B501001305E511B1B797E4FF1FA4
:105DE00083C4843497E7FF1F83C7F733A204DD8C95
:105DF00083A7C9046D14228697E5FF1F9385D532CA
:105E0000280082978E0493160401B7750200C182A0
:105E10003000A695094597D0FF1FE780809C930727
:105E200070F817E7FF1F230FF72E994597E7FF1F1D
:105E3000A38CA72E95BF914763E3870297B5010016
:105E40009385051117A501001305C55B9790010007
:105E5000E78020FB17B501001305450BE9B597E472
:105E6000FF1F83C4642C97E7FF1F83C7D72BA204AF
:105E7000DD8C83A7C9046D14228697E5FF1F9385E7
:105E8000B52A280082978E0493160401B775020084
:105E9000C1823000A6950D4597D0FF1FE780609422
:105EA000930780F8BDBF17B501001305E50897906B
:105EB0000100E780E00C930790F82304F10083478A
:105EC00019008D452800A304F1008347290023050C
:105ED000F10097000000E78060041305C01297C02E
:105EE000FF1FE7800046014597D0FFFFE780C01AFB
:105EF0000D4597000000E78020D2294597C0FF1F7D
:105F0000E780204497C0FF1FE78080347DB397E788
:105F1000FF1F23A1A730828097E7FF1F9387872F5A
:105F200003A3070063030300028317430000670015
:105F3000E3C941114AC097F6FF1F83D6867E328996
:105F400017D6FF1F0356664922C426C206C62A84F6
:105F5000AE8497000000E780A06629C921C8994750
:105F600063F697048347140003470400A207D98F00
:105F700013978700A183D98FC2073167C1831307A5
:105F8000C7556395E70297D7FF1F83D70745A3013E
:105F9000F400A1832302F40097F7FF1F83D76778EB
:105FA00091C7A302F400A1832303F400630D090247
:105FB00097F7FF1F83C787669DE797E7FF1F83C794
:105FC000A72595C38DC097E7FF1F83C7E70D81EF16
:105FD00022852244B2400249A685924441011743DA
:105FE00000006700A3BEB24022449244024941012E
:105FF0008280834755008345450017B5010013058E
:10600000E5F7A207DD8D17930100670083DF17B561
:1060100001001305A5F517930100670063F68D478E
:1060200063F6B708011126CA06CE22CC0344350018
:1060300097E4FF1F83C4541E97B50100938545F56F
:10604000B337800017E7FF1FA308F71C09C497B5F3
:1060500001009385A5F417B501001305A5F49790E9
:106060000100E78000DA97E7FF1F83C7F71A63860E
:10607000970097000000E780804397400000E7808A
:10608000E0E39967938757EE2316F1006800854790
:106090009145A30781002307F10097000000E780E6
:1060A000E0E7F2406244D244056182808280894701
:1060B00063F7B708011122CC06CE26CA8344250017
:1060C00085472A84639DF404914763F5B70403452B
:1060D00045008347340022055D8D97D7FF1F239E1F
:1060E000A72E97000000E78080569967938767EE98
:1060F0002314F1008347340023059100A305F10028
:1061000083474400954528002306F10097000000CE
:10611000E780C0E0F2406244D24405618280FDF82D
:106120009967938767EE2314F10097D7FF1F83D7F2
:10613000C72AA305F10023050100A183E1B78280EE
:106140000111996722CCD51717F4FF1F1304044DD2
:106150002314F1008347040026CA97F4FF1F938499
:10616000445C2305F10083D7040028009545A3056E
:10617000F100A18306CE2306F10097000000E7801E
:10618000E0D903D604008345040017B501001305C8
:1061900065E297900100E780C0C6F2406244D244B5
:1061A000056182809D677971D9172316F10097F7F1
:1061B000FF1F9387A74683C707001305F10006D684
:1061C0002307F10097000000E780209E09E9B7E768
:1061D0000400BC47414681451305F10082976800E1
:1061E000CD4597000000E78060D397F5FF1F83C57A
:1061F000E54217B501001305E5DE97900100E78041
:1062000040C0B25045618280630C0516011126CA58
:1062100006CE22CC4AC84EC697E7FF1F83C7D7FFDA
:1062200097F4FF1F83C4843F99C393E424002A8416
:1062300097100000E78020E193E9C40119E193E998
:10624000C40037E90400832789042285130620034C
:1062500081458297930750FA2300F4009307A00525
:10626000A300F4008D472301F4009147A301F4003B
:1062700093077004A302F40097F7FF1F83D7674AC0
:106280002304F400A183A304F40097D7FF1F83D74E
:10629000C7142305F4009304C400A183230204005F
:1062A00023033401A305F400268597000000E7804E
:1062B000C08F19E583278904414681452685829749
:1062C00097D7FF1F83D7070F230EF400A183A30ED8
:1062D000F40093070002230FF400930710FAA30FB2
:1062E000F4009D472300F402A3000402B7E7040072
:1062F000FC4713052402194697D5FF1F9385C55601
:10630000829797E7FF1F83D787DA2304F402A183DC
:10631000A304F40297E7FF1F83D727D92305F402CC
:10632000A183A305F40297E7FF1F938727D88397DC
:1063300007002285930500032306F402C207C183E8
:10634000A183A306F40297D7FF1F938767F783976C
:1063500007002307F402C207C183A183A307F40245
:1063600097000000E780C0212308A4022181A30830
:10637000A402F2406244D2444249B249056182809B
:1063800082805D71E17793C777FF1305E10086C6D0
:106390002316F10097000000E78040E768009305AE
:1063A000400397000000E78060B7B64061618280DB
:1063B0005DC9411122C426C206C6930750FA2300C4
:1063C000F5009307A005A300F50089472301F50018
:1063D0009147A301F50093077004A302F50097F716
:1063E000FF1F9387A72383C707009304C5002A8450
:1063F0002303F50097E7FF1F938717E283C7070082
:1064000023020500A303F50097F7FF1F83D7673129
:106410002304F500A183A304F50097D7FF1F83D7BA
:10642000C7FB2305F500A183A305F500268597F09A
:10643000FFFFE780807701E9B7E70400BC474146EA
:106440008145268582972285F14597000000E780E7
:106450002013230EA4002181A30EA400B2402244E5
:1064600092444101828082805D710A8586C6A2C401
:1064700097000000E78000F437E404007C448A853C
:106480000810794682973C441305E103094681458B
:106490008297101093050002014597D0FFFFE78017
:1064A000E025B6402644616182800111B7C7A55A34
:1064B00022CC9387C73317E4FF1F1304F4D53EC4DF
:1064C00083470400856601469965254506CE3EC68C
:1064D00097C0FF1FE780E0303000A146996529454D
:1064E00097C0FF1FE780E02F8345040017B5010028
:1064F0001305C5B997900100E780A090F24062446F
:10650000056182800111A146300099652D4522CC9C
:1065100006CE97C0FF1FE780C02CA24737C4A55AFC
:106520001304C43363958702B24517B50100130500
:10653000A5ADB335B00097E7FF1FA38FB7CC9790F9
:106540000100E780008CF240624405618280916521
:10655000A1463000938505F02D4597C0FF1FE780C9
:106560004028A247E38287FC97E7FF1FA38607CA5C
:10657000814517B50100130565ABD1B7C1676976D1
:106580008146FD1705061397060141836364B70032
:106590003E8582803307D50003470700B98F214726
:1065A00013F81700858363050800B18FC207C18304
:1065B0007D171377F70F6DF78506F1B741C5A5472E
:1065C000054763F2B70883471500034705003168A4
:1065D000A207D98F13978700A183D98FC207C183E0
:1065E0001308C855054763900707411106C622C422
:1065F00026C203442500914763F0870493075400A3
:1066000063ECF502A301C50021822302C5009304B7
:10661000340091C6A302D500A1822303D5002A84A9
:10662000A68597000000E780A0F526942300A4002B
:106630002181A300A4000147B240224492443A853C
:106640004101828005473A8582800111B7C7A55A6A
:1066500022CC9387E7342A842AC68566014695654D
:10666000254506CE3EC497C0FF1FE7808017300047
:10667000A1469565294597C0FF1FE7808016A28532
:1066800017B50100130585A297800100E7806077A8
:1066900097000000E78080DDF2406244056182805F
:1066A0000111A146300095652D4522CC06CE97C03C
:1066B000FF1FE7800013A24737C4A55A1304E43430
:1066C00063958702B24517B501001305259897D742
:1066D000FF1F2394B7D0C205C18197800100E780D6
:1066E0004072F2406244056182809165A1463000AB
:1066F000938505EE2D4597C0FF1FE780800EA247CA
:10670000E38287FCD14717D7FF1F2318F7CCD14569
:1067100017B5010013058595C9B721C1411126C2DE
:1067200006C622C4AE848DC52A8497100000E78077
:10673000209297E7FF1F83C727AE99CB228522447B
:10674000B240A68592444101173300006700034818
:10675000B2402244924441018280828001114EC69F
:1067600006CE22CC26CA4AC893F71500AE899DCB27
:10677000AD67371700409387A7AA1CC3B7E704008B
:10678000BC4F13060019854517D5FF1F0345C5C427
:10679000829713C51900F2406244D2444249B2497B
:1067A0000561828093F725000145F5D717F7FF1F94
:1067B000035707F7954763F9E70C014417F6FF1FE6
:1067C000130606E69306300513055004130810045B
:1067D0009308B00413039005930764006374F704EF
:1067E0003A847D5997F4FF1F83C484E397F7FF1F12
:1067F00083C717E3A204DD8CAD679387B755638B1E
:10680000F41463E3970AA9679387A755638EF4147A
:10681000A28517F5FF1F1305A5E097000000E7808C
:1068200000F0E9A0B307860083C50700639AD5048A
:1068300083C517006396A50483C5270063920505E9
:1068400083C53700639ED50283C54700639A15034D
:1068500083C757006396670222890DE897F5FF1FEB
:1068600083D505ECB3852541C20517F5FF1F130538
:1068700025DBC1814A9597000000E78040EAE1A04E
:1068800005044204418089BF3A847D598547E3EB82
:1068900087F45DC4854517F5FF1F130565D897007C
:1068A0000000E780C0E769A8B1679387C75563898F
:1068B000F404B5679387D755E39CF4F4A28517F5E4
:1068C000FF1F1305E5D597300000E780203089478A
:1068D000630EF4009305E4FFC205C18117F5FF1FA5
:1068E000130525D497000000E7808076A68517A5BC
:1068F00001001305657D97800100E780805089A025
:1069000097200000E780E02197000000E780A07357
:1069100011C9A28517F5FF1F130585D09700000048
:10692000E78000730546A28517F5FF1F130545CFC5
:1069300097F0FFFFE780206097200000E780601E4F
:10694000FD57E31DF9F097F7FF1F239B07DC13C5E5
:10695000290091B5A28517F5FF1F130565CC97F0A7
:10696000FFFFE780406959B7A28517F5FF1F1305A0
:1069700025CB97F0FFFFE780C0698DBF411122C48E
:1069800037E404005C5C06C6354697A50100938594
:10699000A52B17B501001305A5FD829711E917A5D1
:1069A00001001305A57397800100E780605D01A0D9
:1069B0008327041C82972A84054597C00000E7803E
:1069C000A01097700100E780C09597600100E780F4
:1069D000C06A97B00000E78020222285B24022449E
:1069E000410182804111054506C622C426C297C0D6
:1069F000FFFFE78040541305A00497B0FF1FE78016
:106A0000006B757585457D1597C0FFFFE780E03DFC
:106A10007D7585451305F53697C0FFFFE780404734
:106A2000371400408327840A8D451305002093E71F
:106A300007202324F40A97C0FFFFE780003BB7E458
:106A4000040097D0FFFFE7802080C858978001009E
:106A5000E780005317B50100130585F19780010009
:106A6000E78000528327840C8545414593E707085A
:106A70002324F40C97C0FFFFE78080418D45130568
:106A8000000897C0FFFFE780A04097C0FFFFE780A6
:106A9000806D37A507001305051297C0FFFFE7803B
:106AA0002069014597C0FFFFE780406F9545054588
:106AB000894717F7FF1F2307F7C697C0FFFFE78037
:106AC000806FB7E700E013070006238DE740370724
:106AD000000423A0E71097D0FFFFE78000F197D0D4
:106AE000FFFFE780000397000000E78060E9970060
:106AF0000000E78060A197000000E780A0BA97E05F
:106B0000FFFFE78020EC97000000E780A05597008A
:106B10000000E780801083A7040817050000130514
:106B200025C4829797D7FF1F2388A78ABC4C1306DA
:106B300000648545829797C0FF1FE780608B014501
:106B40008280AD67371700409387A7AA1CC3B7E7B9
:106B500000E03707400023A0E71801000100B7F765
:106B6000070003C70701A5476316F7009397450180
:106B700091C301A04111AE860146AA85254506C6EE
:106B800097C0FF1FE780E0C5B240B7E700E03707D6
:106B9000400023A0E710410182804111B2862E8679
:106BA000AA852D4506C697C0FF1FE78080C3B24067
:106BB0000145410182809307000463ECC7041D7105
:106BC000A2CC2A840808A6CACAC886CE32C6978034
:106BD0000100E780A017AD67371700409387A7AA89
:106BE0001CC3B7E400E03709400023A024190100CA
:106BF0000100B2461008A285294597C0FF1FE78013
:106C000040BEF640664423A02411D644464925617F
:106C100082803955828041110D658D4506C697C029
:106C2000FFFFE780801CB71700408D6623A6D70AB8
:106C300017F5FF1F130545AF1387C70A9387870A08
:106C40001CC15CC5856689675CC958C114C518C973
:106C5000B7E70400B24003A3871E410102838145C8
:106C6000B307B5008387070089E717230000670093
:106C7000E3F18505C205C181E5B7011106CE230701
:106C8000010001ED17A501001305056A970000003A
:106C9000E78020FDF240056182805800A947BA854F
:106CA00029462548B376C502FD1793F7F70F93865B
:106CB0000603A304D700B356C5026375A8007D1769
:106CC0003685EDF33385F500D1B797A7010093879B
:106CD000E7651357C5003E9703470700011106CE2D
:106CE0002304E100135785003D8B3E9703470700BF
:106CF00023060100A304E100135745003D8B3D89A5
:106D00003E97AA970347070083C70700280023057B
:106D1000E100A305F10097000000E78080F4F24055
:106D200005618280797117A501001305A55906D662
:106D300022D426D24AD04ECE97000000E78060F2DF
:106D400017F5FF1F0355E59D97000000E78020F829
:106D500097F7FF1F83C7878C17A5010013050554FC
:106D600089C717A501001305E55297000000E780C9
:106D700040EF17A501001305255597000000E78097
:106D800040EE17A501001305A55497000000E78009
:106D900040ED114597000000E78060EE17B5010057
:106DA000130505B197000000E780A0EB01459700AF
:106DB0000000E780C0EC17B50100130565AF970030
:106DC0000000E78000EA1305700497000000E780E8
:106DD00000EB97D7FF1F83C7374417A501001305A2
:106DE000654C89E717A501001305454C9700000085
:106DF000E78020E717A501001305054E9700000066
:106E0000E78020E637A5070013050512970000006C
:106E1000E780E0E617A501001305854C9700000008
:106E2000E78020E497F7FF1F83C7879117A501002C
:106E30001305454889E717A5010013052548970064
:106E40000000E78000E217A501001305254A97001E
:106E50000000E78000E117A501001305A549970090
:106E60000000E78000E017C5FF1F0355A5549700F9
:106E70000000E780C0E517A501001305E54797006E
:106E80000000E78000DE17C5FF1F0355055597007A
:106E90000000E780C0E317A50100130565469700D1
:106EA0000000E78000DC17D5FF1F03554520970041
:106EB0000000E780C0E117A501001305E544970035
:106EC0000000E78000DA17D5FF1F0355051E970065
:106ED0000000E780C0DF17A5010013056543970098
:106EE0000000E78000D817D5FF1F0355251C970029
:106EF0000000E780C0DD17A501001305A54197003C
:106F00000000E78000D617C5FF1F0355653B9700BB
:106F10000000E780C0DB17A501001305254097009E
:106F20000000E78000D4014497D9FF1F9389C993DB
:106F300097A401009384843F1949B307340183C7A0
:106F400007000A85050413D74700BD8B2697A6972F
:106F50000347070083C70700230101002300E10066
:106F6000A300F10097000000E780A0CFE31724FD05
:106F700017A501001305053B97000000E78060CED0
:106F80000A8597F0FFFFE78040C20A840408834720
:106F90000400034514000904A2075D8D970000005A
:106FA000E780E0D2E39584FEB25022549254025915
:106FB000F24945618280411126C2E97797F4FF1FAB
:106FC0009384048722C49387A7552E842381B40019
:106FD0002E86AA8517F5FF1F1305C58506C62390C3
:106FE000F400A381040097800100E78020D6930578
:106FF0002400C205C18117F5FF1F1305858397F093
:10700000FFFFE780E057B38784002382A700218138
:10701000A382A700930564002244B24026859244CF
:10702000C205C181410117230000670023B609C9C9
:107030009307000463E6B700170300006700E3F757
:10704000828017E5FF1F0345A56F828097E7FF1F2A
:1070500083C7C77D89E717230000670023B38280B9
:1070600097F7FF1F83C7278199EF411106C6972025
:107070000000E78080A9B240854717E7FF1F230C77
:10708000F77E4101828082806304054A6382054A5B
:107090001D71A2CCCAC886CEA6CACEC6D2C4D6C2DC
:1070A000DAC05EDE62DC66DA6AD86ED6B9472A8458
:1070B0002E8963F9B706394697A501009385C5085F
:1070C00097800100E78020C631ED8347E400130775
:1070D00010036394E702854717E7FF1F2308F7743F
:1070E00017A501001305450797E7FF1F239F0772A8
:1070F00097000000E780E0B671A01307000317A512
:10710000010013056508E395E7FE97E7FF1F238F4E
:10711000077097E7FF1F239A077017A50100130553
:107120002505F9B797E7FF1F83C7477063820724D8
:10713000BD6A396C014A17EBFF1F130BAB60938BD1
:10714000FA55938CFA66130DEC5505A8B307440164
:1071500083C6070097E7FF1F83D7276DB9E393071F
:10716000A005639BF600854717E7FF1F231FF76AFB
:1071700097E7FF1F2388D75C050A93170A01C1838D
:10718000E3E627FDF6406644D6444649B649264A1A
:10719000964A064BF25B625CD25C425DB25D256151
:1071A0008280854D639BB7039307500A639EF60068
:1071B000894717E7FF1F231AF766930750FA17E767
:1071C000FF1FA301F7584DBF9307A005E386F6FA0A
:1071D00097E7FF1F239B076445B7138717004207F4
:1071E000DA9741832380D70017E6FF1F231FE6624B
:1071F0008D47E3F3E7F897E4FF1F83C4D45497E780
:10720000FF1F83C74754A204DD8C9387F4FFC20796
:10721000C1839306F00DE3EDF6FA93876400C2078D
:10722000C183E31BF7F493852400C205C18117E5F0
:10723000FF1F1305455197F0FFFFE78060343307C8
:107240009B008347570003474700A207D98F17E7E2
:10725000FF1F231C075C6312F5108149638DB40185
:1072600097E9FF1F83C9494EA20997E7FF1F83C70C
:10727000B74DB3E9F90017050000130585DB97F05A
:10728000FFFFE78000C96385790963EF3B036388EB
:10729000A9059307EC656383F90697E7FF1F83C78A
:1072A000A74A05476380E70881CB1387A7051377B3
:1072B000F70F8D4663F9E6081307F0072300E10096
:1072C000A300F100894595A8638999059387FA770A
:1072D000E395F9FC97F0FFFFE780E00A11A8A68587
:1072E00017E5FF1F1305454697F0FFFFE78060D3C2
:1072F000014597F0FFFFE780C0C1BDBDA68517E53A
:10730000FF1F1305654497F0FFFFE78080DACDB7D4
:1073100097F0FFFFE78000E3E1BF97F0FFFFE78012
:10732000A0E8F9B7930710F8130511002300F10046
:1073300097F0FFFFE7800008FD450A8597000000F1
:10734000E780A0C775B7A68517E5FF1F1305C53FE2
:1073500097F0FFFFE780809261BF9307F0078945B0
:107360000A852310F10097000000E78000C529B5C9
:10737000BD4763FE2703414697A50100938505E3BA
:10738000228597800100E780009A0DE517A501008E
:10739000130505E397000000E780A08C970000002C
:1073A000E7808098179501001305856291B3014726
:1073B0006313F9023D4697A501009385A5E1228557
:1073C00097800100E7802096014711E517A501008D
:1073D000130545E1C1B7B7064000D945A506931985
:1073E000070193D9090163F12903B307E40083C7B7
:1073F0000700D91793F7F70F63E8F500B3D7F60046
:10740000858B13061700CDEFB3093941C20993D913
:107410000901A14763F8370BB304E400254697A59B
:107420000100938565DD268597800100E780A08FA8
:1074300051E9A547638DF90083C7940035476388F8
:10744000E70029476385E70093F7F70DA5EF17A538
:107450000100130525DB97000000E780808017A559
:107460000100130565DB97F0FFFFE780807F17A51C
:107470000100130525DB97F0FFFFE780807E1145B3
:1074800097F0FFFFE780A07F17A501001305454295
:1074900097F0FFFFE780E07C014597F0FFFFE78072
:1074A000007E17A501001305A54097F0FFFFE780B8
:1074B000407B1305700497F0FFFFE780407CDDB54B
:1074C000328731BFC14763FE2705414697A50100BA
:1074D0009385C5D5228597800100E780C08431E17E
:1074E0008347040113071003639CE700854717E7F0
:1074F000FF1F2307F72417A50100130565D4CDBE90
:107500001307000317A50100130585D6E392E7BE14
:1075100097E7FF1F2386072217A501001305C5D390
:10752000C1BECA85228597C0FFFFE78060CB99B9AD
:107530008280411126C2AE848D4522C406C62A84AB
:1075400097C0FFFFE780C094B717004099C803A514
:10755000C70C418D23A6A70CB2402244924441019E
:10756000828003A5870C418D23A4A70CF5B7834720
:10757000050003471500A207D98FC2076177C187AD
:1075800013072720639AE700834525003705040089
:1075900017030000670023FA828017E6FF1F130617
:1075A000E62D8147B2861303F00FA9483308F60091
:1075B0000348080013F7F70F6307A80C6306680079
:1075C0008507E39517FF2947B387E6002380A700C7
:1075D00097E7FF1F9387472B5DA8411113D76500DD
:1075E0001347170006C693F63500058B954791CAD9
:1075F000054699476387C60009469D476383C600D1
:10760000A14713F645003336C00093F685030506FF
:1076100085C2A145638BB604E145638AB604930530
:1076200080026388B604930580036393B600914695
:1076300097E5FF1F238FF54A97E5FF1F238AC54A69
:1076400097E5FF1FA386D54ABE8517A50100130540
:10765000E5D197700100E780C07AB240854717E70F
:10766000FF1FA308F748410182808546D1B78946AC
:10767000C1B78D4675BF17A501001305A5D11773B6
:1076800001006700037817E7FF1F1307E71FBA978A
:107690002380B700E147E302F5F493077002E30C9F
:1076A000F5FC82802A8723800500814717E5FF1FAC
:1076B0001305C51C1308F00F2946B306F50083C651
:1076C00006006396E60297E6FF1F9386E61BB697D1
:1076D00083C7070005452380F5009947636EF702CD
:1076E0009D4763FDE700E147630DF70082806385F6
:1076F00006018507E393C7FC0145C5B72380050054
:107700008280B737004003C7370083C7050093F76F
:107710000704D98F2380F50082805D7152DC56DA30
:107720005ED6716A97EBFF1F938BCB4D8D6AA6C215
:107730004EDE62D486C6A2C4CAC05AD866D26AD007
:107740006ECEC1495E8C97E4FF1F9384A414130A84
:107750000A20938A7ADC17E9FF1F0349A94DB387F2
:107760002B0183C7070093F7F70FC9EFB7870040D6
:1077700003C76700058BE310077C03C76700118B05
:10778000E30D077E83C75700918B99E36F102003A9
:1077900017E7FF1F0347274A85476304F7006F1069
:1077A000400197E7FF1FA386E73497E7FF1F238376
:1077B000071A97E7FF1F2381072697E7FF1F238FED
:1077C000073097E7FF1F238C073097E7FF1FA3833E
:1077D000071897E7FF1FA381072497E7FF1FA38FD1
:1077E000072E97E7FF1FA38C072E97E7FF1FA383A2
:1077F000073097E7FF1FA3800744B7870040114772
:107800006F0070779307190093F7F70F3D47636494
:10781000F70617E7FF1F230FF74097E7FF1F938730
:107820006740CA9783C707001307100293F7F7034F
:10783000638EE71E6366F70405446385871CE38C4B
:1078400007620947638EE71013070002E384E74EDF
:10785000B7E700E03707400023A0E7180100010068
:10786000629923000900FD1923A0E71093F9F90F8D
:10787000E39309EEE5BD97E7FF1F238D073A71BF3C
:10788000130730026388E70C63E8E716130740022A
:10789000638CE70A13070003E39CE7FA97E7FF1FEF
:1078A00093874737CA9703C70700A1471377F70F96
:1078B000E31BF71483C7640097E6FF1F2382F622B9
:1078C00097E7FF1F83C777FD91C7FD5797E6FF1F17
:1078D0002388F62097E5FF1F83C5D5FB97E7FF1F99
:1078E000A380B72097E7FF1F83C7C7FA13FB0708DA
:1078F0009306000493F70706639FD74C9307A009EC
:10790000638DF51663EAB7129307F0056386F54AAF
:10791000930750096384F52A014497E7FF1F83C743
:10792000371C1547E392E736B7E700E0370740001A
:1079300023A0E71801000100B786004023808602DB
:10794000130680FC6F00500EFD5717E7FF1F23083A
:10795000F718FDBDFD5717E7FF1F2301F718CDBD31
:1079600017A50100130585B497700100E7804061F9
:1079700097E7FF1F9387072ACA9703C40700014BA5
:1079800097ECFF1F938C8C091374F40F17AD010053
:10799000130D4DB263478B04294597700100E780B2
:1079A000204B854717E7FF1FA308F70617E7FF1FC0
:1079B0002305870617E7FF1F230EF71237E700E0BE
:1079C000B70640002320D718010001003786004089
:1079D0008347A60293F7370F2305F6022320D7101B
:1079E00085BDB3876C0183C507006A85050B977059
:1079F0000100E780004179BF854717E7FF1F230D8E
:107A0000F700B9B517E7FF1F1307C7204A970347C9
:107A1000070097E6FF1FA38FF6F297E6FF1F238C60
:107A2000E6F217E7FF1F2307F70C1DB5854717E799
:107A3000FF1F2301F7F229BD9307400A6389F5343C
:107A40009307200B6384F5369307100AE396F5EC51
:107A5000838724000144E3D207EC97E7FF1F83C725
:107A600097E393F63700638A061A0546638AC622AF
:107A700009466395C61A1D4755A217E5FF1F034522
:107A800085E1C94797ECFF1F83CCFCE097E5FF1F1A
:107A900083C585E017E4FF1F034414E06315F51068
:107AA000CD476392FC1093077008639CF50213079F
:107AB000300FB7170E006308E4001307900DB7B737
:107AC00004006314E40817E7FF1F2321F702BE85B3
:107AD00017A501001305859E97700100E7806032AD
:107AE00025BD93078008639DF500B307804013F41C
:107AF000F70FB7774600938787CDB3D78702E1B7F3
:107B000093079008639AF500B307804013F4F70FCA
:107B100091679387C766D5B79307A008639BF50065
:107B2000B307804013F4F70FB7173D009387079012
:107B3000E9B79307B008639AF500B307804013F4E0
:107B4000F70F9167938797D04DBF93F5F5078D4752
:107B5000639BF500B307804013F4F70FB7975B0002
:107B6000938707D859BF8947639BF500B3078040C7
:107B700013F4F70FB7770B009387071BBDBF85473B
:107B8000639AF500B307804013F4F70FDD6793871E
:107B900067E3A5B7D28785F9B307804093F7F70F5E
:107BA000B3D7FA020DB797000000E780409FA28587
:107BB000668597000000E780809EB9BB9305610051
:107BC00017E5FF1F034525CD17E4FF1F0344B4CC81
:107BD00097000000E78040AD930571002285970073
:107BE0000000E78060AC3C0017E7FF1F232AF70086
:107BF000834761002304F10083477100A304F1006F
:107C0000894717E7FF1F230DF7EC8357810017E71C
:107C1000FF1F2311F7C8094409B3154793F647001E
:107C2000B336D00093F78703850685C32146638B5F
:107C3000C7066146638AC706130680026388C706C3
:107C4000130680036393C700914717E6FF1F2301C4
:107C5000D6EA97E6FF1FA38DF6E897E7FF1F238A72
:107C6000E7E817E7FF1F034727C39376070497E763
:107C7000FF1F83C777C28DEE1377770C93067008CA
:107C8000630CD7021377F7078D466312D70CB3073F
:107C9000F040B7955B0093F7F70F938505D849A897
:107CA0001947ADBF854755B7894745B78D4771BF60
:107CB000930670086311D7021307300FB7150E0033
:107CC0006389E7021307900DB7B504006383E702E9
:107CD0001307700845BF9306800C6311D702B307E2
:107CE000F040B775460013F7F70F938785CDB3D5EE
:107CF000E70297E7FF1F23ABB7DED9BB9306900CD3
:107D0000631CD700B307F04093F5F70F9167938793
:107D1000C766B3D5B702F1BF9306A00C631DD700A9
:107D2000B307F040B7153D0093F7F70F9385059023
:107D3000B3D5F5027DBF9306B00CE315D7F4B307B6
:107D4000F04093F5F70F9167938797D0D9B789469D
:107D5000631BD700B307F040B7750B0093F7F70F1D
:107D60009385051BF1B78546631AD700B307F0402A
:107D7000DD6593F7F70F938565E35DBFD28535FB2E
:107D8000B305F04093F5F50FB3D5BA029DB783C79D
:107D90002400C18B99C7854717E7FF1F2305F7D438
:107DA000A5BE97E7FF1F238007D4BDB6854717E719
:107DB000FF1FA300F7D48DB63C0017E7FF1F232158
:107DC000F7E40947930700032314F10097E6FF1F28
:107DD0002388E6D02DBD63940756A94763E5B742D3
:107DE000179701001307C7558A05BA959C41BA97A2
:107DF000828717E4FF1F034414AA894C6306940D7D
:107E000063E68C0685476303F4089307F00F17E7D2
:107E1000FF1F0347E7CC63F6E70017E7FF1F2301C7
:107E2000F7CC97ECFF1F83CCACCB9307000413F483
:107E3000FC0F63F497011304000497E7FF1F938777
:107E400027DC03AD070022862685EA85B38C8C40AB
:107E5000229D97700100E78060EF97E7FF1F238165
:107E600097C997E7FF1F23ADA7D945BC8D47630C82
:107E7000F40A9947E31BF4F8979701009387C752D8
:107E800017E7FF1F232EF7D6A94751B717E7FF1FA4
:107E9000034767DA97E7FF1F938787C64946979599
:107EA00001009385655963068700979501009385C6
:107EB000A5543E8597700100E78040E917E7FF1F52
:107EC0002320A7D4C947A1B797E6FF1F83C6A6D62C
:107ED000054797E7FF1F9387A7C26394E6023E8595
:107EE00013067002979501009385855297700100E3
:107EF000E780C0E517E7FF1F2324A7D09307700290
:107F000039B73E8513063004979501009385854A5D
:107F100097700100E78080E317E7FF1F2322A7CEB9
:107F200093073004EDB597E5FF1F83C5C5961795F8
:107F300001001305E55997700100E78080EC054DBD
:107F400097EDFF1F83CD2DCF97E5FF1F83C5A59428
:107F5000179501001305C5576398AD0B9770010085
:107F6000E78020EA97E7FF1F83C7E792B5CBE36E70
:107F7000F4E81794010013046450638CB70117945C
:107F80000100130424506386970117940100130421
:107F9000E450228597700100E780C0FF1375F50F4C
:107FA00093071500860717E7FF1F230BF7B48D47CC
:107FB00017E7FF1FA306F7B497E7FF1F938747B4A0
:107FC0000147BE861376F70F89076365A60297E718
:107FD000FF1F23A7D7C297E7FF1F83C767B205BD5F
:107FE000979701009387874217E7FF1F232AF7C05F
:107FF000914731BD3306E40003460600A380070025
:1080000005072380C7007DBF97700100E78060DF10
:1080100097E7FF1F83C72788E1D7E368F4DE17944B
:1080200001001304A442638CA701179401001304F8
:108030006442638697011794010013042443228548
:1080400097700100E78000F51375F50F9307150091
:10805000860717E7FF1F2305F7AA8D4717E7FF1FBE
:10806000A300F7AA97E7FF1F938787A90147BE865A
:108070001376F70F8907E37CA6F43306E400034682
:108080000600A380070005072380C700D5B797E542
:10809000FF1F83C545801795010013052544977080
:1080A0000100E78000D697E7FF1F83C737A593E756
:1080B000470017E7FF1FA303F7A483C7240017E7B0
:1080C000FF1FA30BF7A289B81795010013054542BE
:1080D00097700100E780C0EA97E7FF1F9387C7A169
:1080E00083C7070017D7FF1F2306F77A17E4FF1F80
:1080F0000344049F333480000DB01795010013052D
:10810000654097700100E780A0E797E7FF1F83C7EE
:10811000F79E93E7070117E7FF1FA301F79E83C7A9
:10812000240017E7FF1F2309F79C6FF0EFFE179558
:1081300001001305653E97700100E78060E403C706
:1081400004007D8B51EFB787004003C767021377A8
:10815000C70B136727002383E70203C7A702137720
:10816000C70B136727002385E70203C7E7021377CE
:10817000C70B136727002387E70203C7270313777B
:10818000C70B136727002389E702854717D7FF1F0F
:108190002302F77C17E7FF1F2300F78817E7FF1F6D
:1081A000230EF79217E7FF1F230BF79297D7FF1FB6
:1081B000A382077A97E7FF1FA380078697E7FF1F31
:1081C000A38E079097E7FF1FA38B079097E7FF1FEA
:1081D000A382079297E7FF1FA38F07A46FF0CFF347
:1081E00089476312F70297D7FF1F83C7E76A914653
:1081F000638CD70863E0F604638EE70C6369F70AC3
:1082000005476380E70EFD5717E7FF1FA30AF78CAA
:1082100037074000B7E700E023A0E718010001009E
:10822000B78600401306F0FC2381C60223A0E710A6
:108230006FF00FE2130720086382E7086362F7021A
:1082400013071008E391E7FC378700408347670274
:1082500093F7C70B93E727002303F7026FF0CFEBE9
:10826000130730086389E70213074008E39DE7F826
:10827000378700408347270393F7C70B93E727000F
:108280002309F7026FF04FE9378700408347270340
:1082900093F73707F5B7378700408347E70293F72F
:1082A000C70B93E727002307F7026FF0EFE6378746
:1082B00000408347E70293F73707F5B73787004059
:1082C0008347A70293F7C70B93E727002305F7021D
:1082D0006FF08FE4378700408347A70293F7370793
:1082E000F5B7378700408347670293F73707ADB785
:1082F000179501001305452397700100E78040C8DA
:1083000097D7FF1F23880758D5B31795010013058A
:10831000A52297700100E780A0C697D7FF1F239B77
:10832000075697D7FF1F9387A77B03C4070089478A
:1083300063F3870009441374F40F6FF00FDE130723
:108340000002E392E7EC631B0B0A638FF5009307CF
:1083500020026383F50817950100130565219770C6
:108360000100E78000AA45B5179501001305851D9A
:1083700097700100E780C0C00144179D0100130DF4
:10838000AD1DA14CB387840083C507006A85050431
:1083900097700100E780E0A6E31694FF17850100BF
:1083A0001305056997700100E78080BD17D4FF1F92
:1083B0000344844E01E897D7FF1F238F074A014BE0
:1083C0006FF0AFD58947E310F4E4854717D7FF1F57
:1083D0002304F74A6FF04FD417D6FF1F0346B64B5E
:1083E00097D5FF1F83C5254B17950100130545172A
:1083F00097700100E780E0A06FF00FD26380F50670
:1084000093071002E399F5F497D5FF1F83C5C5487C
:10841000179501001305C51697700100E780609E4F
:1084200097D7FF1F23AE977C97D7FF1F9387076CC3
:10843000944383D7470017D7FF1F0347876B17D68F
:10844000FF1F2329D6441D4497D6FF1F2396F644C9
:1084500097D7FF1F2383E7446FF02FCC97D5FF1FDB
:1084600083C5854317950100130505139770010017
:10847000E780209997D7FF1F2380074097D7FF1FDA
:10848000239A07406FF02FF92547638FE7C8994675
:10849000378700406394D70223008702B7E700E0E4
:1084A000B706400023A0D71801000100130600FC06
:1084B0002301C70223A0D7106FF08FB99306100ACB
:1084C000639FD70023008702B7E700E0B7064000AC
:1084D00023A0D71801000100130680FCD1BF93062A
:1084E000A009E381D7FE9306400AE38DD7FC9306EB
:1084F0002002639DD700B7E700E0B706400023A045
:10850000D7180100010023008702F9B78546E384EC
:10851000D7FE93070008E300FBFEB7E700E0B706CD
:10852000400023A0D71801000100130620FC2300FF
:108530008702BDBF17D7FF1F0347975A6302F71E75
:1085400063E7E70295476300F7109947630AF7046A
:10855000B786004023800602B7E700E037074000F7
:1085600023A0E718010001001306A0FC75B99307CA
:10857000F005630AF700930750096306F7009307B5
:108580001002E317F7FCB7E700E03707400023A02D
:10859000E71801000100B7860040130620FC69B10E
:1085A00017DBFF1F034BCB53930700045A8D63F473
:1085B0006701130D000497D7FF1F9387676483AC8F
:1085C00007001374FD0F2286E6852685976001005B
:1085D000E780C077B3078B40669417D7FF1F23014E
:1085E000F75097D7FF1F23AD8760B7870040630C14
:1085F0000B022380A703B7E600E03706400023A064
:10860000C6180100010003C727021347070423818E
:10861000E70203C727021377C70F2381E70223A0CE
:10862000C6106FF0EFA22380070237E700E0B7061D
:1086300040002320D71801000100130620FC2381ED
:10864000C7026FF0AFB9378700408347370097D62E
:10865000FF1F83C6764A93F70708D58FA301F7005B
:10866000B7064000B7E700E023A0D71801000100DB
:108670001306A0FC35BD97D7FF1F9387A759CA974C
:1086800083C7070093F7F70FC1CF97D7FF1F83C7A3
:10869000875AD9E717D7FF1F03479744930700026C
:1086A0006310F70883AD040017DDFF1F034DCD1ED7
:1086B00097DCFF1F83CC5C1E17DBFF1F034BEB1DFA
:1086C000E6876A87DA866E8697D5FF1F83C5C51A47
:1086D000179501001305C5ED97600100E7806072F2
:1086E00097D7FF1F23A4B74197D7FF1F2382A74126
:1086F00097D7FF1FA38E973F97D7FF1F238B673F07
:1087000097D7FF1FA3898716B7E700E03707400018
:1087100023A0E71801000100B78600406FF04FA2C8
:10872000B7E700E03707400023A0E7180100010089
:10873000B786004015BD97D6FF1F83C6C64F0547B5
:10874000639CE60429472381E70209472383E70264
:108750002385E70297D7FF1FA38E073897D7FF1F00
:10876000A38B074CB7870040A381070017D7FF1FD3
:10877000A304073805472383E700B6402644964400
:108780000649F259625AD25A425BB25B225C925C51
:10879000025DF24D6161828029472381E70209472A
:1087A0002383E7022385E7022387E7022389E70281
:1087B00055B717D7FF1FA300F70C6FE01FFF8547C2
:1087C00017D7FF1F2308F71817D7FF1F2306F72413
:1087D00017D7FF1F2304F73017D7FF1F2301F730E8
:1087E0006FE0BFFE854717D7FF1F2305F71617D782
:1087F000FF1F2303F72217D7FF1F2301F72E17D7D9
:10880000FF1F230EF72C17D7FF1FA305071417D739
:10881000FF1FA303072017D7FF1FA301072C97D71C
:10882000FF1FA38E072A8280411106C69700000011
:10883000E78080FBB787004023800700130740FCD8
:108840002386E7001307C004A386E70017D7FF1F9E
:10885000130747042398E70017D7FF1F130787075D
:10886000239AE70017D7FF1F13070713239CE7007E
:1088700017D7FF1F1307871E239EE7002947238171
:10888000E70209472383E7022385E7022387E702FC
:108890002389E702A3810700930600F8A380D7008D
:1088A000930690022380D700FD562383D7002381AF
:1088B000E7009306000537E700E0230BD740B70633
:1088C00040002320D71003C7170013671700A380A9
:1088D000E700B24097D7FF1F239007224101828013
:1088E000411106C697000000E78000F0B7870040FE
:1088F00023800700130700FC2386E7003147A38687
:10890000E70017D7FF1F1307E7F82398E70017D7EB
:10891000FF1F130727FC239AE70017D7FF1F130732
:10892000A707239CE70029472381E7020947238300
:10893000E7022385E702A3810700930600F8A380DE
:10894000D700930690022380D700FD562383D700DB
:108950002381E7009306000537E700E0230BD740AB
:10896000B70640002320D71003C71700136717006E
:10897000A380E700B24097D7FF1F239F071641014E
:108980008280F1679387072017D7FF1F2320F716F0
:10899000854717D7FF1F231DF714A14717D7FF1FC0
:1089A0002309F71497D7FF1FA385071497D7FF1F35
:1089B0002382071497D7FF1F238007EC97D7FF1F49
:1089C000A38B07EA814717D5FF1F130525EBFD553C
:1089D00017D6FF1F130646EB2947B306F500238081
:1089E000B600B306F600238006008507E397E7FE8E
:1089F00097D7FF1FA387070E97D7FF1FA385070EE3
:108A000097D7FF1F2380070E97D7FF1F238B070CD5
:108A100097D7FF1F238A070C97D7FF1FA384070C44
:108A200097D7FF1F2381070C814717D6FF1F130617
:108A3000661D4147B306F600238006008507E39BC9
:108A4000E7FE828017D7FF1F0347E71E854763169F
:108A5000F700170300006700E3E817030000670052
:108A6000E3DC411122C406C617D7FF1F0347A71C2A
:108A700085472E8613F4F50FAA856317F70417D5DB
:108A8000FF1F130565F597600100E780202C97D73D
:108A9000FF1F238307F8B787004023848702B7E6C8
:108AA00000E03706400023A0C6180100010003C7FC
:108AB000A7021377C70F2385E702B240224423A001
:108AC000C61001454101828017D5FF1F130585E4BB
:108AD00097600100E780802797D7FF1F238C07E668
:108AE000B787004023828702B7E600E037064000E0
:108AF00023A0C6180100010003C767021377C70F40
:108B00002383E7025DBF411106C697000000E7809E
:108B100080E7B2404101170300006700E3F2411112
:108B200006C697F0FFFFE78080BF97D7FF1F83C778
:108B300077E2A1CB97D5FF1F83C5E5E189C917D59A
:108B4000FF1F130565E197E0FFFFE780205497D7EB
:108B5000FF1FA38107E097D7FF1F238D07F837E793
:108B600000E0B70640002320D71801000100378637
:108B700000408347660293F7370F2303F602232052
:108B8000D710B2404101828041C9D9C597D7FF1F94
:108B900083C787F6D1C3011122CC4AC84EC656C23C
:108BA0005AC006CE26CA52C42E89AA890144930A05
:108BB0000004371B030063772403B3078940C2070F
:108BC000C183BE8463F4FA0093040004C204C1802C
:108BD000130A1BD497D7FF1F83C7C7D79DE37D1AFE
:108BE000631C0A00F2406244D2444249B249224A1C
:108BF000924A024B0561828097F0FFFFE78020B226
:108C0000D1BF338589002694A685420497000000D1
:108C1000E78060E5418045B7828097D7FF1F938743
:108C2000E71318429C4383D645000345070083C5DC
:108C3000C700035646006396A50083D5E700638D01
:108C4000D502011106CE2386A7002397D700B705CA
:108C5000CF00DC4B9385757D05077D162EC2230062
:108C600001003AC42316C1002317D10099C30A8515
:108C70008297F240056182808280411122C417A44C
:108C8000FF1F1304E4775C4C06C691CBC84B01C9A7
:108C9000B7E70400BC5782975C4C23AA0700B24098
:108CA000224441018280DC4DDC4B81CFB7E70400D8
:108CB000904503A38705914517D5FF1F0345450A36
:108CC00002838280B7E7040003A30705A14517D5F7
:108CD000FF1F0345E50802836D713C083EC6B707D8
:108CE000E500232291103EC8AA843C083285232641
:108CF00011103ECA23248110232021112E89973080
:108D00000000E780605A2A84979501009385C58DFD
:108D1000177501001305056F97600100E780600E6D
:108D2000A285179501001305E59897600100E7807B
:108D3000400D294597600100E7808011B705CB0001
:108D40009385757D680097100000E780E05FA2853D
:108D5000680097300000E780804701478146700037
:108D6000CA85268597200000E780608305CD2A8488
:108D70009795010093854587177501001305856850
:108D800097600100E780E007A285179501001305B1
:108D9000259397600100E780C00629459760010090
:108DA000E780000B8320C11003248110832441102D
:108DB000032901105161828097D7FF1F938707FA1B
:108DC00018429C43797122D406D60348070083C811
:108DD00007012A8483D6450003554600639608019F
:108DE00083D82701638DD8022388070105072399BB
:108DF000D7003708CC00DC4B1308787D3ACC13073A
:108E0000F5FF42CA23080100231EE100231FD10001
:108E100099C7080832C62EC482973246A2452285D9
:108E200097000000E78080EBB250225445618280B9
:108E300079713146977501009385854D280006D6D6
:108E400097600100E78080F097A7FF1F83D7475BFB
:108E5000231B0100231C0100231D0100231E010010
:108E6000231F010099E3C167FD17231AF10097A79B
:108E7000FF1F83D7075991EB97D7FF1F938707EE03
:108E80009C439C43DC4783D7070097A6FF1F93862C
:108E90002657231BF100D84E83D74600231CF10030
:108EA0005C4B91CB97A7FF1F83C7F75581EB9700CA
:108EB0000000E780C0DCB25045618280FD1717A634
:108EC000FF1FA302F6540356070183C706014C4750
:108ED0002800230FF10097300000E780602C97D71F
:108EE000FF1F9387A7E79C4301479786010093865E
:108EF0002679884330004C0897100000E780206AEC
:108F00005DD975B799C9B7E7040003A30705A14563
:108F100017D5FF1F0345C5E4028382805C4EDC4BFE
:108F2000B9CFB1CD411122C4177501001305854D8C
:108F30002E84978501009385657006C697600100B1
:108F4000E78020ECA2851785010013056571976005
:108F50000100E78000EB294597600100E78040EFC2
:108F6000B7E704002244B24003A3870517D5FF1FCB
:108F7000034505DF130640069145410102838280C7
:108F8000411122C417A4FF1F130444451C4C06C6FC
:108F900089C7DC4399C34C488297584CB7E7040013
:108FA000BC57484B82975C4CB240224423AA07002E
:108FB0004101828017A7FF1F13074744834707001B
:108FC0009306F00B850793F7F70F63E9F60097A672
:108FD000FF1F2385F642034507008280930700F8B0
:108FE000FDB78357450099E37D558280011122CC5E
:108FF00017A4FF1F1304C4405C4C4AC84EC6DC4B88
:1090000052C406CE26CA56C2B2892E8A2A898DC774
:10901000B7E70400FC5F829797D7FF1F938707D2BB
:109020009C431307301FB307F54071556375F7066E
:1090300097000000E780A0C49307D00D7D5563EC36
:109040003705B7E4040093878900B858832AC40120
:10905000139507014181029723AAAA00484C584959
:1090600021E7978501009385655B1775010013055E
:10907000653997600100E780C0D8178501001305A6
:10908000E56697600100E780C0D729459760010039
:10909000E78000DC5D55F2406244D2444249B24967
:1090A000224A924A0561828013874900B705CF00A2
:1090B0002319E5009385757D310597100000E78041
:1090C000A028484C83456900310597300000E780AF
:1090D0000010484C4E86D285310597300000E7805D
:1090E000200C7146CA8517A5FF1F130565319760CF
:1090F0000100E780A0C5FC5C82970326C90097D7D2
:10910000FF1F23ADA7C211CABC4C854517D5FF1F51
:10911000034505C582970145BDBF97000000E78064
:1091200060D1D5BF411106C622C426C217D4FF1F85
:10913000130404C397000000E78060B4B7E40400A0
:10914000FC4C0345040085458297034504002244F6
:1091500003A3C405B2409244A145410102834111D9
:1091600026C297D4FF1F938464BF9C4006C622C4C6
:109170004AC0D5C3DC43C5C35CC12300B5002A8403
:10918000978501009385C544177501001305852750
:1091900097600100E780E0C6294597600100E780FD
:1091A00020CB9C4023A4070023A2070097A7FF1F02
:1091B0009387C722DC4FDC4B91C7295597000000ED
:1091C000E78040DC97A7FF1F93878723DC4FDC4BAA
:1091D00089C797000000E78020F537E9040083275E
:1091E000C905894517D5FF1F034585B78297832792
:1091F000C905914517D5FF1F034585B682979C4049
:1092000003A347016309030022852244B24092442C
:10921000024941010283B240224492440249410181
:1092200082800111328506CE22CC26CA2E84973048
:109230000000E7806007AA84978501009385853C3C
:10924000177501001305051C97600100E78060BBDE
:10925000030784000356640083554400A6861785DF
:1092600001001305654297600100E78080B9294538
:1092700097600100E780C0BD97A7FF1F83C76716EF
:10928000639D9700014597000000E780A0CF8145CE
:109290000A8597000000E780C0ECF2406244D244A7
:1092A000056182806D7123248110232611102322F1
:1092B000911093F745002E84638707143C083EC045
:1092C000B707E5003EC23C083EC42317010023183F
:1092D000010023190100231A0100231B010097A795
:1092E000FF1F83D7A70F99E3C167FD172316F1006E
:1092F00097A7FF1F83D7A70E91EB97D7FF1F9387E1
:10930000E7A59C439C43DC4783D7070017A7FF1FB3
:109310001307C70C2317F100544F83574700231836
:10932000F100DC4AA1E7978501009385E5311775C7
:1093300001001305250D97600100E78080AC1785BB
:1093400001001305254197600100E78080AB2945A6
:1093500097600100E780C0AF134544008320C1102F
:1093600003248110832441105161828097A7FF1F3D
:1093700083C737072555D9C3FD1717A6FF1FA302BB
:10938000F60603D6060183470701CC460A85230B60
:10939000F10097300000E780A0E097D7FF1F938788
:1093A000E79B9C4317A7FF1F1307470397860100FE
:1093B0009386862A88430A866C0097100000E7800F
:1093C000001EAA8451D9978501009385E52717755A
:1093D00001001305250397600100E78080A2A685A0
:1093E000178501001305C53797600100E78060A16C
:1093F000294597600100E780A0A526859700000019
:10940000E78040B891BF93F725009DC7B7E70400F8
:10941000BC474146814528088297255597000000A2
:10942000E78040B628089305F00F97000000E7801A
:1094300040D3134524001DB793F7150081CB970047
:109440000000E780209F1345140009BF93F78500B3
:10945000014589D717A7FF1F0347F7FA97A7FF1FF3
:10946000938707FA0DC3D84F584B11CF37E7040045
:10947000384F9047854517D5FF1F0345658E0297E6
:1094800013458400E1BD97F0FFFFE780407FCDBF2B
:109490005C4D411106C688C317D7FF1F2320F78CE8
:1094A000B7E7040083A70708170500001305C5DF09
:1094B0008297B24097D7FF1F2384A78A01454101B5
:1094C000828001113335A000A307A100B7E7040093
:1094D00083A7471706CE1306F100854513055030C4
:1094E0008297F240056182808280411122C406C6C3
:1094F00097B7FF1F83C757D2054489EF97C7FF1F50
:1095000083C7C711014499E717B4FF1F0344C4D0B0
:1095100013441400228597000000E780C0FA1785E5
:1095200001001305A52A09E4178501001305052B81
:109530002244B2404101176301006700838C7971B6
:1095400022D4A30F010037E404008327841726D216
:109550004AD006D6AA842E89130550309305F1010E
:1095600032C6829732468347F10193150601C181C5
:1095700085CB01452EC697000000E780C0F4832705
:109580004417B2454A862685829705459700000014
:10959000E78060F3B25022549254025945618280B0
:1095A000832744174A8626858297EDB74111939702
:1095B000050122C406C626C2C1872E8463D40702D1
:1095C000B7E40400FC5417A5FF1F034565E6829726
:1095D00019C1BC5482972165218DB2402244924426
:1095E0004101828093F715008DC7B7E7040083A778
:1095F000471A17A6FF1F1306A6E297C5FF1F9385FC
:10960000E57617A5FF1F0345A5E2829713451400D1
:10961000E9B793F725000145E9D397C7FF1F83C733
:10962000677685E7B7E7040003A8871A1307401F8A
:1096300097A7FF1F83C7C7DF8146130640069945DA
:1096400017C5FF1F0355857302981345240071B792
:1096500097C7FF1F83D787726398A70217C7FF1F9B
:10966000231FB77017C7FF1F231CC77017C7FF1F23
:109670002319D7702E86178501001305A51CBE85FA
:10968000175301006700E377178501001305051DD7
:10969000176301006700C38E0357450097C7FF1F7C
:1096A00083D7C76D6318F702C167F91717C7FF1F84
:1096B0002326F76C97C7FF1F23A4076C97C7FF1FCC
:1096C000238C076A97C7FF1F238E076A17030000C2
:1096D0006700E3E1178501001305451817630100D2
:1096E0006700038A7D15954763E2A71C1787010071
:1096F0001307470C0A053A951C41011122CC06CEEE
:10970000BA972E848287178501001305A5159760E7
:109710000100E780E086A1A203C7250099476311F5
:10972000F7022E8597000000E78040F7834564002C
:10973000178501001305051497500100E780606C40
:1097400097B7FF1F238A07AC17850100130545143F
:109750007DBF03C7250095476319F702C16717C787
:10976000FF1F0357A761F91703D5A5006309F70287
:10977000B7E7040083A7C717829717850100130571
:10978000251297500100E780A07F854717B7FF1F7C
:109790002304F7A817850100130505138DBF97C78C
:1097A000FF1F239DA75C83D7E50097C6FF1F239863
:1097B000F65C83D7050197C6FF1F2393F65C83D71A
:1097C000250197C6FF1F239EF65A97C7FF1F2385C3
:1097D000075A631BE502B7E70400BC4F096613068E
:1097E0000690894517A5FF1F034585C48297035638
:1097F000E4008355A400178501001305A50B9750BD
:109800000100E780006051B79307700F2316F10045
:10981000B7E7040083A7870D17A6FF1F034646C1BD
:109820006C0082974DF9854717C7FF1F2306F75431
:109830005DB7178501001305E509D1BD83C5250076
:1098400091476392F502178501001305250A975089
:109850000100E780E07297000000E78040C9F24015
:1098600062440561828099476392F50222859700E0
:109870000000E780A0E2834564001785010013051E
:1098800065FF97500100E780C057D1BF9547639AA5
:10989000F50083471400E1F3178501001305450720
:1098A000BDB51785010013052507E1BF8280375735
:1098B000315F97A7FF1F9387E7B8130777D598C342
:1098C0009356C50017870100130787F4BA9683C51E
:1098D000060093568500BD8ABA9603C606009356C5
:1098E0004500BD8A3D89BA962A9783C6060003477C
:1098F0000700238407002383D700A383E700238284
:10990000B700A382C70097A7FF1F9387A7B423833D
:10991000B700A383C7002384D700A384E700828015
:10992000411106C697000000E780A0F8B7E70400E1
:1099300083A7871417A6FF1F1306C6B0D545014598
:109940008297B2404D4697A5FF1F9385A5B013059A
:1099500070304101170300006700A3BE617123242A
:10996000811A37E40400832704082326111A2322CE
:10997000911A2320211B232E3119170500001305EE
:1099800025C3829717A9FF1F130989AA9947854400
:109990002300A900231CF10097850100938545E66B
:1099A00093074006177501001305C5A5231CF10890
:1099B0002308910097C9FF1F9389A9D697500100EA
:1099C000E780204483D5090017850100130545E28F
:1099D00097500100E780E042294597500100E78059
:1099E000204703D5090097000000E78080EC83271B
:1099F0004417100885451305503082978327441774
:109A000017A6FF1F130606A5CD45130570308297D4
:109A10008327441717A6FF1F1306C6A1B5451305D4
:109A20006030829783274417300889451305103129
:109A3000829783274417300989451305203182977F
:109A4000832744159305000A0D4582978327441503
:109A50009305000A11458297A30591002306910002
:109A600002CD23080100230C01008327841630094E
:109A70009145130570408297832784161306B10021
:109A8000854513050040829783278416700085451D
:109A900013051040829783278416300885451305E7
:109AA000204082978327841610088545130550406F
:109AB0008297832704157D558297832744137D550C
:109AC00082977D5597A0FFFFE78020BC8327440C39
:109AD000829797A0FFFFE78080978327841417A6BB
:109AE000FF1F13062696D545014582978947130621
:109AF000700F814528092306F1009780FFFFE7805A
:109B000000618D471306000881452808230CF108E1
:109B10009780FFFFE780A05F9147230CF1009767D4
:109B200001009387A77F984383C747003AC8230A59
:109B3000F10097D0FFFFE7806093700085450545F1
:109B400097A0FFFFE78080BB30099305700F0945A0
:109B500097A0FFFFE78080BA3008930500080D4505
:109B600097A0FFFFE78080B910089545114597A0A1
:109B7000FFFFE780A0B8C16717C7FF1F13070720C3
:109B8000F9171CC32322070017A5FF1F1305058A19
:109B900097A0FFFFE78060B58327C41D17C5FF1F8F
:109BA0001305451C82973C4803450900854582976B
:109BB0008320C11A0324811A8324411A0329011A1C
:109BC0008329C1195D618280C16717C8FF1F0358CF
:109BD000E81AF9176301F8083DCDB5CD011126CA81
:109BE000B7E4040083A7841222CC2E862315B1008B
:109BF00006CE2A8401478146ED45428582972AC6D2
:109C000011ED178501001305E5C197500100E780AC
:109C10002037F2406244D24405618280FC440356FE
:109C2000A100A28582972C0017C5FF1F03550515BB
:109C300097A0FFFFE78020B869DD178501001305B5
:109C4000A5BF97500100E780A03383A7C412ED455C
:109C5000280082977DBF82800DC585471797FF1F1B
:109C6000A30FF77C9797FF1F238C077C35469795AA
:109C7000FF1F9385257C13056030170300006700E4
:109C8000438C9797FF1FA38C077AE9BF97C7FF1FE5
:109C900083C7470FA9EFC16717C7FF1F0357070EF9
:109CA000F9176306F7044111854722C417C7FF1F40
:109CB000230AF70C37E404007C4C06C68945179547
:109CC000FF1F0345E57682970323841A2244B2409E
:109CD0009797FF1F83C7C77517C5FF1F0355050A51
:109CE0001307401F81463146994541010283828016
:109CF0006D712324811023261110232291103284A8
:109D000001CD8947630AF5028320C1100324811025
:109D1000832441105161828017850100130585C09D
:109D2000AE8497500100E780A025A285268597C0C4
:109D3000FFFFE7806082C9BFB7E70400FC47280047
:109D40008297178501001305A5BE97500100E78093
:109D500020238347810039C41307000B6380E70287
:109D60001387A7051377F70F8D4663EDE602A285EB
:109D7000280097C0FFFFE78060F079B78547E3F5DB
:109D800087F883459100177501001305E598B335F1
:109D9000B00097A7FF1F2389B73097500100E780D5
:109DA00040069DB703479100A207B966D98F138774
:109DB000E6556384E70C636DF7042D671307B75509
:109DC000638FE708636AF70029671307A755638F56
:109DD000E708A2852800A1BF31671307C75563882C
:109DE000E70635671307D755E395E7FE8947E3FD97
:109DF00087F097000000E780A0E99305E4FFC20523
:109E0000C1811305A1009790FFFFE780603DEDBD84
:109E10003D671306F7556389C706636DF6009386A1
:109E2000E665E398D7FAA285280097C0FFFFE78090
:109E30004028D9BD9306F766638DD7041307F777DB
:109E4000E399E7F897C0FFFFE780E05375BD01464F
:109E5000A285280097C0FFFFE780E00D75B5A285B9
:109E6000280097C0FFFFE780001979BDA285280070
:109E700097C0FFFFE780E01941BDA285280097C089
:109E8000FFFFE780001A49B597C0FFFFE780802BEE
:109E9000A5BD97C0FFFFE7802031BDB5C16717C5DD
:109EA000FF1F0355A5EDF9176307F500B7E7040099
:109EB00003A3C7170283828017F3FFFF67002363A2
:109EC0001783FFFFE70203202A8408452E89B28901
:109ED00019C900C1971500009385A58661059730C3
:109EE0000100E780200581447D5A97100000E7803B
:109EF000E03963C7A404814497100000E780003A6A
:109F000063C8A40497C7FF1F938707E89C43DC47F7
:109F1000B307F94091872302F40063830904832780
:109F2000C900B307F4409587A302F4001C4C89C70D
:109F30009C4799C3228582971783FFFF6700C31B45
:109F40005C44139714008504BA972390470171BFAE
:109F50001C48139714008504BA972390070069BF23
:109F6000832789000547B307F4409587A302F400CF
:109F700083570400638EE7028DC309476384E704B7
:109F80000D47E395E7FA97870100938727ED1CCCEF
:109F900097870100938787ED11A897870100938722
:109FA00067B31CCC978701009387C7B35CC8BDBF5C
:109FB000978701009387079F1CCC978701009387A1
:109FC000679FEDB797870100938707EE1CCC9787B3
:109FD0000100938767EED9BF95E51783FFFFE7027E
:109FE0000310004618448347940075839D8B6317C4
:109FF000F70097100000E78060B448C41783FFFFA4
:10A000006700231082801783FFFFE702A30B1389E9
:10A010003500C16442094111AA890144F114135960
:10A020000901054A2EC697100000E7802026B24598
:10A030006348A400014541011783FFFF6700C30B7C
:10A0400083A7090013171400BA9783D70700638802
:10A05000B7006394970063742A010504E1B70545CE
:10A06000D9BF1783FFFFE7020305AA892E89328B28
:10A07000B6843A8ABE8A97A00000E780C0FE71C904
:10A08000268597200000E780C00C8D4763E7A70076
:10A090007D551783FFFF6700830583DB440097101E
:10A0A0000000E780A0242A8497100000E780402564
:10A0B0009307740031443305850263CDA7029710DE
:10A0C0000000E780A02297100000E78020222A8469
:10A0D00097100000E780C0229307740031443305D5
:10A0E000850263C3A70497100000E7802020930730
:10A0F000450029A897100000E780802033058502DD
:10A100001307F0179307C017E35FA7FA2D55E3C2B3
:10A1100077F963040B02D6865286A6854A85972076
:10A120000100E780C0BDB5B797100000E780401D73
:10A13000330585029307C5FFD1BF832749001385E7
:10A14000C90083D5270097000000E78000EC61F587
:10A1500081B769553DBF97C7FF1F2399A7C297C70E
:10A16000FF1F938767C2904381470C463307F50072
:10A17000420741836393B700828054461398470097
:10A180008507C2962390E600D5B797C7FF1F938730
:10A19000A7BF9C4303C58700828017C5FF1F0355D7
:10A1A000E5BE82801783FFFFE70263F3C167138771
:10A1B000D7FF630BE502636AA700F1176300F5029E
:10A1C00001451783FFFF6700C3F31387E7FF6302AF
:10A1D000E502FD171D8D13351500E5B797500000FA
:10A1E000E780602A7D15C5BF97500000E780E0FE3C
:10A1F000D5BF97500000E78000FDEDB71783FFFF44
:10A20000E702E3ED4111AA8401442EC69710000035
:10A21000E780C008B2456348A400014541011783A7
:10A22000FFFF670003EE9C48131514003E9583570B
:10A230000500E385B7FE0504C9BF03485500814604
:10A2400093F7F60F63E5070181473E858280584505
:10A2500093975600BA9703D727006316B70003D722
:10A260000700E304C7FE8506E1BF834645000147BA
:10A270009377F70F63E4D700814711A81C451316A5
:10A2800057000507B29703D60700E313B6FE3E85D5
:10A2900082801783FFFFE702E3E293170501C1877E
:10A2A00097CAFF1F938A4AAE635BF00883A70A0030
:10A2B000C0479C4703570400198D420541816368DC
:10A2C000F500014422851783FFFF6700E3E21205D2
:10A2D0002A94CDBFDC4713944900014A3E9483473A
:10A2E00044006341FA02014A834754006349FA0279
:10A2F0008509C20993D9090183A70A009847E3EBAE
:10A30000E9FCC1B71C4413195A00A6853E994A8539
:10A3100097000000E780C0EE05E1050AC9B75C447C
:10A3200013195A00A6853E994A8597000000E780D8
:10A3300020ED19E1050A4DBFE30C09FA61B7AA84C3
:10A3400081495DBF1783FFFFE70263D91C452A845B
:10A3500081E79307C5001CC51C44231204001CC0E0
:10A360009307F00F63EDB70093F5F50F2285972063
:10A370000000E780C0E51783FFFF670083D8939450
:10A380000501C167C18063F9F500A6852285972084
:10A390000000E780E0E8C5B7C18193F5F50F22859D
:10A3A00097200000E780A0E2A68522859720000084
:10A3B000E780E0E3C9B797C7FF1F9387E79C88430F
:10A3C00082801C4599C797C7FF1F23AFA79A0145F5
:10A3D00082807D55828097C7FF1F9387E79A9843B5
:10A3E00083474500484792073E9582801783FFFFC9
:10A3F000E702E3CE617100451C183EC6B707800135
:10A400003EC81C183ECA8357440002CE02D002CC7C
:10A41000231EF100834784002A8902D22301F1021E
:10A420003C083ED402D697000000E78000FB83572B
:10A4300005002316F10297500000E78000C82307AB
:10A44000A1025C4003556400F18313F717008347B2
:10A45000F10252055181F99BD98FA307F1029710A0
:10A460000100E780207939CDAA840355050097A023
:10A470000000E78020C083D704002AD26800231C94
:10A48000F10083D72400231DF1001C4803D64700A8
:10A490008C4397200000E780A0D08347B400CA8691
:10A4A00017760100130686498117A305F4006C0096
:10A4B000481097200100E78080845D611783FFFFCB
:10A4C000670023C42155D5BF1C45B1CF03C5A700E4
:10A4D000894613576500630BD7028D46630ED7027A
:10A4E00085466300D702130740063305E50203C71C
:10A4F000B700418B15CB83C7B700BD8B3355F540F3
:10A5000082801375F5031307803EC5B7096713757D
:10A51000F50313070771D1BF372709001375F5033A
:10A520001307077CD9B7014582801783FFFFE70235
:10A5300003BB03A98500630C09048347B900AE84FB
:10A5400093F7070E85C303459900930520030D81FA
:10A550000505B305B5028844610597300100E78021
:10A5600080AD35A02E8597000000E78020F62A8474
:10A5700019CD97000000E780605C8325C900B30710
:10A58000B54063FA87002E94B305A440E9F517831C
:10A59000FFFF670003B785457DBF1783FFFFE70215
:10A5A00003B42A8403D50500011132C636C43AC269
:10A5B0002EC002CA02CC02CE97A00000E78080AB7A
:10A5C00082452ACA22852ECC97000000E780E0E071
:10A5D00003570500231EE10097500000E780E0AD1F
:10A5E000A24632469247230FA10036874C08B28616
:10A5F0002285014697000000E780E0A605611783E9
:10A60000FFFF670003B01783FFFFE70243AD6171EF
:10A610001C183EC6B70780013EC81C183ECA3C083D
:10A6200000453ED4AA8402CC02CE02D002D202D689
:10A6300097000000E78060DA83570500355923163C
:10A64000F10297500000E78040A72307A10209C448
:10A650008357440081EB21594A855D611783FFFFD1
:10A66000670023AA03556400520551819710010029
:10A67000E78040582A8965D18347B40093F7070ED5
:10A6800099C71305840197300100E780009D835727
:10A690004400231EF100834784002301F1025C4043
:10A6A00003550900D98313F7070883471102231CB8
:10A6B000A10093F7F707D98FA300F1028357290070
:10A6C000231DF1005C40F18313F717008347F1026B
:10A6D000F99BD98FA307F10297A00000E78080992A
:10A6E0002AD235D9834794006800139757008347CF
:10A6F000B400FD8BD98FA305F4001C4803D6470096
:10A700008C4397200000E780A0A9A6871777010057
:10A710001307C722740005464C10268597000000D9
:10A72000E78060942A890DD98347B400A685FD8B04
:10A73000A305F40097000000E78060DF31BF1783B6
:10A74000FFFFE702C399832485FE2A8441112685F1
:10A7500097000000E78080D7834734FF93F7070E08
:10A760008DCB2AC6268597000000E78060C809CDFA
:10A77000834734FFB245FD8BA309F4FE91C52285C2
:10A7800097300100E780208B41011783FFFF6700AE
:10A7900043977DD98327C4FF2685829775F5834724
:10A7A00034FF93F7070E91C7228597300100E780A9
:10A7B000C08A032584FE97000000E78000E5E9B722
:10A7C0001783FFFFE702A38E9C4141112A8903C72B
:10A7D000070089472E84935667006380F6040D4670
:10A7E0006388C6049307F0076304F7022E85972059
:10A7F0000000E78060ABAA848149C16B130C49005B
:10A8000097B7FF1F938747589C43984763E4E90431
:10A8100041011783FFFF6700438D03D7450085473C
:10A82000E3F8E7FE2E8597200000E78040ADE1B712
:10A8300003D74500E3FEE7FC2E8597200000E78064
:10A84000A0A6AA84228597200000E78000A8C20461
:10A85000C98C5DB7DC470355A900139A49003E9A9D
:10A8600093170501C187635DF00083570A00639762
:10A87000A70263E774038327CA00034D5A002DA083
:10A88000A1672167A98F1307F7EFE374F7FE6397BA
:10A89000090097000000E780209161FD85098DB7D0
:10A8A00083278A00034D4A00835DA900035769008E
:10A8B000216A138BC7003AC6814A33CA4D01631E11
:10A8C0005D0197B7FF1F9387A74C9C43E1DBA286EE
:10A8D0006286814526858297D1B7A1679387F7EF76
:10A8E000930C4BFF63F24703B2455A8597F0FFFF85
:10A8F000E780A0710DC103278B00104709CE1043DC
:10A900006382C4023107D5BFEE85668597000000DB
:10A91000E780008F71F993861A0093FAF60F130BF4
:10A920000B0271BF835644005C43E3E9F6F62285CF
:10A930003AC697200000E7802081A1679387D7045B
:10A940002A8A035D4400324763E897008347D900B1
:10A9500093E707F8A306F9001C4766852286E2857F
:10A960008297C1670844FD17337AFA00529508C0F0
:10A970002312A40125B797B7FF1F9387E740984399
:10A98000814715C31447814763FFD500939745005E
:10A990004C47BE9519C903C7550081476375E6004A
:10A9A000DC451606B2973E85828003C74500814785
:10A9B000E37BE6FE16069C45F5B71773FFFFE7023B
:10A9C0006370AA892E8A814497BAFF1F938ACA3B73
:10A9D00083A70A00984763E6E4001773FFFF670048
:10A9E000A371DC471394440001493E9413BB140047
:10A9F00083474400634BF900014913BB14008347AC
:10AA00005400634FF9008504E1B7084493175900D7
:10AA10005287DA860146A2853E9582990509C9BF0B
:10AA20004844931759005287DA860546A2853E9519
:10AA300082990509E9B71773FFFFE702436A814569
:10AA400017F5FFFF1305054897B7FF1F239007343D
:10AA500097000000E780A0F61773FFFF6700636AA6
:10AA600097B7FF1F938747329C4395C31773FFFF28
:10AA7000E702E366814517F5FFFF1305A54497003C
:10AA80000000E780C0F31773FFFF670083678280D1
:10AA90001773FFFFE702036337E404008327841280
:10AAA00041112315E100AE893289368A3A86814602
:10AAB0000147ED45AA8482972AC621C90356A10001
:10AAC000D28597400100E78060288327C413CE8594
:10AAD00026858297058905C98327440D2314210102
:10AAE00001462C00268582972A8401C9B7E7040015
:10AAF00083A7C712ED45280082972285410117736D
:10AB0000FFFF6700635F4944D5B76554FDB75C41FB
:10AB1000FD175CC182801773FFFFE702435CB7E754
:10AB20000400FC5F829795473305F50281450D814E
:10AB30001773FFFF6700E35C1773FFFFE702235AF9
:10AB4000B7E70400FC5F829795473305F5020D8156
:10AB50001773FFFF6700E35A1773FFFFE7022358DD
:10AB6000B7E7040083A7870B035505008297177387
:10AB7000FFFF670003591773FFFFE70243560355B2
:10AB800005003287AE861796FF1F0356C69297B50B
:10AB9000FF1F9385252097000000E780A0EF177323
:10ABA000FFFF670003561773FFFFE7024353B7E742
:10ABB000040083A7C71782971773FFFF67006354CA
:10ABC0001773FFFFE702A351B7E7040083A78713BA
:10ABD00097B5FF1F9385051C829701451773FFFFEB
:10ABE000670023521773FFFFE702634FB7E70400C4
:10ABF00083A7C71F81451795FF1F0355C5878297F8
:10AC00001773FFFF6700E34F1773FFFFE702234D42
:10AC1000B7E7040083A7871397B5FF1F93858518AF
:10AC2000829701451773FFFF6700A34D1773FFFF5E
:10AC3000E702E34AB7E7040083A7C71F81451795DA
:10AC4000FF1F0355458982971773FFFF6700634B0A
:10AC50001773FFFFE702A3482E8597800000E78067
:10AC600080B397800000E78080F01773FFFF6700D4
:10AC700043491773FFFFE702834697800000E78090
:10AC800080FA1773FFFF6700C3475C49E1175CC98F
:10AC90005CC583572501A1072319F50083570501DA
:10ACA000A1072318F5008280F1473305F50297B715
:10ACB000FF1F938727119C433E9582808D47631524
:10ACC000F60803D74600854763F0E7081773FFFFD0
:10ACD000E702E340368536842E8997100000E7802E
:10ACE000A05C29C98357440093140501C18063E324
:10ACF0009704228597100000E780005BFD14231263
:10AD000094009307A0026300F5029307B002630763
:10AD1000F50293079002631FF5002285970001005A
:10AD2000E780608901A80146CA85228597A00000B6
:10AD3000E78000B41773FFFF6700A33C22859710DC
:10AD40000000E7806007FDB7828097B6FF1F9386FB
:10AD5000A6079C42014599CF9843D44217B6FF1FDE
:10AD60002324E6066396D70097B6FF1F23A0E606C6
:10AD70001385C7FE82801773FFFFE70243369700F3
:10AD80000000E780A04B7144330585029145979000
:10AD90000000E780C0EC11E565551773FFFF670001
:10ADA000433697B7FF1F23ADA70097000000E78049
:10ADB000E04833058502914597900000E78020EA3E
:10ADC00061DD97B7FF1F23AFA7FE97000000E78064
:10ADD000E04697B7FF1F239FA7FC97000000E7807E
:10ADE000E04597B7FF1F2398A7FC9777010093874B
:10ADF00027BA17B7FF1F2323F7FC97070000938795
:10AE000007E917B7FF1F2329F7FA014579B7177329
:10AE1000FFFFE702C32CAA8517B5FF1F130585F9AD
:10AE200097100000E780605F1773FFFF6700632DD6
:10AE30001773FFFFE702A32A97000000E78060FD79
:10AE400097100000E780E05E97B7FF1F9387C7F772
:10AE50009C4391CF1387C7FE19CB83D5C7FF17B586
:10AE6000FF1F1305E5F697200100E780C01C17734C
:10AE7000FFFF670003291773FFFFE70243269700D0
:10AE80000000E780C0EC09CD834785002A8493F752
:10AE9000070499EB0355E50097000000E78080F96F
:10AEA0001773FFFF6700E3258347C500930445013F
:10AEB00017B9FF1F130949F185E3832709005CC90E
:10AEC00097B7FF1F23A297F083274900F1FB97B79D
:10AED000FF1F23AD97EEE9B7FD172306F5006105C7
:10AEE00097800000E78060DA8307840063CB070463
:10AEF0008347840093E707F82304F400B7E70400CE
:10AF00009C5F82974205A94741813375F5028347CB
:10AF1000840093F707FCC98F2304F4008347D4000F
:10AF20003E951C402318A40089CF984319CB834732
:10AF3000C4005040814585073305F5024205418133
:10AF40000297832709005CC897B7FF1F23AE97E6D7
:10AF50008327490089E797B7FF1F23A997E683470F
:10AF6000C4009DDF8355040117B5FF1F130545E697
:10AF700097200100E780200C25B71773FFFFE70239
:10AF8000031697B7FF1F9387E7099C470144858302
:10AF9000858B85E3AE84B2853A8697100000E78002
:10AFA000204F2A8419C597100000E78060458294DD
:10AFB00008CC22851773FFFF6700A3141773FFFFE8
:10AFC000E702431041112E8932C6AA89970000007A
:10AFD000E780C031324713060502CA869705000094
:10AFE0009385C5CC17B5FF1F1305C5DC970000007E
:10AFF000E780E0F82A8425C99304C5009700000083
:10B00000E780E0411946AA85268597100000E78071
:10B0100020198545268597100000E78000151775D3
:10B0200001001305A5944E958345050026859710CC
:10B030000000E780C0195C4831468145A1075CC823
:10B040005CC483572401E1172319F40083570401DA
:10B05000E1172318F4001C4C3E859770FFFFE78032
:10B06000000BA3042501228541011773FFFF670030
:10B07000A3081773FFFFE70283064111AA842EC6B7
:10B0800032C497100000E780003A004DB2452246D6
:10B09000834784000CC050C093F7F70393E707047D
:10B0A0002304F40023180400268597100000E7808D
:10B0B000203583479400A9462317A40013D73700EF
:10B0C00005073307D7029D8B85072306F400A306E7
:10B0D000E40083C70401D8488507230FF7FE17B79C
:10B0E000FF1F130767CE5843232A04009307440128
:10B0F00029E317B7FF1F232BF7CC17B7FF1F232513
:10B10000F7CC17B4FF1F1304A4CC228597200100AD
:10B11000E780A0E41C44858B5D8D19E5814522857F
:10B1200097200100E78020F141011773FFFF6700BE
:10B1300043FD1CC317B7FF1F232AF7C8D9B71773DE
:10B14000FFFFE702C3F997050000938565B7014546
:10B1500097000000E78000B001451773FFFF67000C
:10B1600043FA1773FFFFE70283F797000000E780B9
:10B1700080B01773FFFF6700C3F88347C500A5E3DE
:10B180001773FFFFE702A3F52A840355E500970034
:10B190000000E78000C821C18347840093F7F7FBD4
:10B1A0002304F4001C4091C7DC4381C74C40014597
:10B1B000829797000000E78080B917B5FF1F13053D
:10B1C00025C197200100E78040E90355E40097007E
:10B1D0000000E78020C61773FFFF670083F28280BC
:10B1E0001773FFFFE702A3EF97B7FF1F9387C7BD52
:10B1F00097050000938565C817B5FF1F130545BD6A
:10B2000023A0070023A2070097200100E78080D237
:10B210001773FFFF6700E3EE1C4D91CFDC4381CF36
:10B220001773FFFFE702A3EB8345070082971773AD
:10B23000FFFF670003ED828097B7FF1F938787BBEF
:10B240009C4303C50700828097B7FF1F938787BA87
:10B250009C4303C51700828097B7FF1F938787B968
:10B260009C4303C52700828097B7FF1F938787B849
:10B270009C4303C54700828097B7FF1F938787B71A
:10B280009C4303C53700828097B7FF1F938787B61B
:10B290009C4303C55700828097B7FF1F938787B5EC
:10B2A0009C4303C56700828097B7FF1F938787B4CD
:10B2B0009C4303C57700828097B7FF1F938787B3AE
:10B2C0009C4303C58700828097B7FF1F938787B28F
:10B2D0009C4303C59700828097B7FF1F938787B170
:10B2E0009C4303C5A700828097B7FF1F938787B051
:10B2F0009C4303C5B70011E11D45828097B7FF1F2E
:10B30000938747AF9C4303C5C700828097B7FF1F51
:10B31000938747AE9C4303C5D700828097B7FF1F32
:10B32000938747AD9C4303C5E700828097B7FF1F13
:10B33000938747AC9C4303D50701828097B7FF1FD3
:10B34000938747AB9C4303C52701828097B7FF1FB4
:10B35000938747AA9C4303D54701828097B7FF1F75
:10B36000938747A99C4303D56701828097B7FF1F46
:10B37000938747A89C4303D58701828097B7FF1F17
:10B38000938747A79C4303C5A701828097B7FF1FF8
:10B39000938747A69C4303C5B701828097B7FF1FD9
:10B3A000938747A59C4303C5C701828097B7FF1FBA
:10B3B000938747A49C4303C5D701828097B7FF1F9B
:10B3C000938747A39C438857828097B7FF1F938733
:10B3D00067A29C4303D5C702828097B7FF1F93875C
:10B3E00067A19C4303D5E70219E11305800C828015
:10B3F00097B7FF1F938707A09C4303C5070382806D
:10B4000097B7FF1F9387079F9C43C85B828097B7BE
:10B41000FF1F9387A79D8843828097B7FF1F93875D
:10B42000279D8843828019E17D558280F5DE984210
:10B4300065DFFDD917B7FF1F1307C7BE1847AA87D7
:10B440007155058B631D072403C507001547E37D70
:10B45000A7FC03C737001305F0057D171377F70F17
:10B46000E364E5FC03C35700E30003FC83C8670003
:10B47000E38C08FA03C77700494579171377F70F6C
:10B48000E364E5FA03C7A70011481305F7FF137536
:10B49000F50FE36BA8F803CE97000D481305FEFFE8
:10B4A0001375F50FE362A8F803C8B7006309080035
:10B4B00065181378F80F1305600DE36705F703C5EA
:10B4C000C700794879151375F50FE36FA8F403C821
:10B4D000D7000D457D181378F80FE36705F503D8FD
:10B4E0000701930E40175118420813580801E3ED65
:10B4F0000EF303C8E7007D181378F80FE36605F331
:10B5000003C827017D181378F80FE36F05F103C80E
:10B510008700C54E75181378F80FE3E70EF103D8CE
:10B520006701856E938EBEE06D18420813580801BE
:10B53000E3EC0EEF03D847016D18420813580801D9
:10B54000E3E40EEF03D88701791842081358080185
:10B55000E36C05ED03C8A7017D181378F80FE365C8
:10B5600005ED03C5B7011D487D151375F50FE36D96
:10B57000A8EA03C5D701714879151375F50FE3657E
:10B58000A8EA03D5E7011308E00F7D1542054181C4
:10B59000E36CA8E803C50702494879151375F50F50
:10B5A000E364A8E8C85301C937C834005915130823
:10B5B00058BFE36BA8E603A8870237C5340013051C
:10B5C00055BF5918E36205E717B5FF1F2322C5824F
:10B5D00003C6050117B5FF1F232EF5800545E3754A
:10B5E000C5E403D82501D04933760603E31E06E2FD
:10B5F00003C61501E30A06E217A6FF1F2328B67E3D
:10B6000083C5270001466387A50003C61700F145DF
:10B610003306B60283C707039305C00272971A0761
:10B620001307C70516031A9796084697B387B702FC
:10B6300041553E973297420741836362E80617738C
:10B64000FFFFE702C3A9368597800000E780406CC2
:10B6500097000100E780C04B2A8497A00000E78094
:10B66000205E2A9497F00000E780002A2A949790A1
:10B670000000E78040852A9497F0FFFFE780E06FA5
:10B680002A9497400000E78000972A949770000062
:10B69000E78040A022951773FFFF670083A6828092
:10B6A0001773FFFFE702A3A34111A307A10097A00F
:10B6B0000000E78040C99305F1001705000013055D
:10B6C000E5B597F0FFFFE780802F01454101177333
:10B6D000FFFF670003A31773FFFFE702C39D17B4C3
:10B6E000FF1F1304249403288400795993681800D9
:10B6F00097B4FF1F23AC149313781800631008024B
:10B70000BA84BE89368B328A2E89AA8A97F0FFFFC7
:10B71000E780E0A77D15269519E531594A8517730D
:10B72000FFFF6700C39C97F0FFFFE78040A67D15F1
:10B730002695A167E353F5FE97B7FF1F938787C54B
:10B7400098433E8C814B01CB014597F00000E78088
:10B75000C047933B15004A85DA865686D285979076
:10B760000000E78060512A8911CD1C44F99B17B76E
:10B77000FF1F232DF78A83270C00CDD3E3800BFA1C
:10B78000829769BF268597B7FF1F23AF078897F079
:10B79000FFFFE780809C4146CE8517B5FF1F13054C
:10B7A000E59197300100E780605A97D00000E7806C
:10B7B000E09C0325040B97D00000E780A0A005457E
:10B7C00097D00000E780A0A7054597000000E7801C
:10B7D00060EDA9B797B7FF1F9387C7849C47858BF8
:10B7E000EDC71773FFFFE702838F17B5FF1F130520
:10B7F000258B97B7FF1F23A7078297B7FF1F23A5A6
:10B80000078297B7FF1F23A3078297200100E780D5
:10B81000C08497500000E78080F997100100E7800E
:10B82000405097100100E780405697A7FF1F93876D
:10B83000E77D9C4391C7054597800000E780E023A2
:10B8400097A7FF1F938747669C4399C741657D155E
:10B8500097700000E780E0A597F00000E780804146
:10B8600097D00000E780209397B7FF1F93878790BA
:10B870009C43139717016356070097F00000E78079
:10B88000A0B097B7FF1F23AB078297B7FF1F23A96D
:10B89000078297B7FF1F23A7078297B7FF1F23A52C
:10B8A000078297000000E780008C97000000E78087
:10B8B000A07597F0FFFFE780401897F00000E78041
:10B8C000E0D91773FFFF6700C383828097A7FF1F2C
:10B8D000938747758843828097A7FF1F9387877454
:10B8E000C8438280B7E7B0009387075063E1A7029F
:10B8F00097A7FF1F93870773D843FD576367E5003A
:10B9000097A7FF1F23A2A77281473E858280B95760
:10B91000EDBF1763FFFFE702837C97800000E7809D
:10B92000607597800000E780C0771763FFFF6700AE
:10B93000437D1763FFFFE702E3782A849304140230
:10B9400001112E85B289A685214636C63A899730DF
:10B950000100E780403D0DE9B24638082686CE85D5
:10B960001305940497500000E780604121462C089D
:10B970004A8597300100E780003B133515000561CB
:10B980001763FFFF670043770145D5BF1763FFFFCC
:10B99000E702E3749305450617A5FF1F1305C54588
:10B9A00097100100E78020691763FFFF6700637548
:10B9B0001763FFFFE702A37241112EC697F0FFFF46
:10B9C000E780C017B24588C141011763FFFF6700D8
:10B9D00043731763FFFFE702E36EAA842E84978008
:10B9E0000000E780006CAA89854522859700000049
:10B9F000E780E07D83C7E4011389940899E3138904
:10BA00000403CE85228597000000E780407C214614
:10BA100093051902228597000000E780607897A7B8
:10BA2000FF1F938727608C43228597100000E780D3
:10BA3000C082214693858402228597000000E7801A
:10BA400020761763FFFF6700236B1763FFFFE70292
:10BA50008366397197F00000E780E0B493054006F3
:10BA600061E997800000E78000606302051497A7F2
:10BA7000FF1F83C7273A13B7170097A6FF1F238B13
:10BA8000E638014499CFC16417A9FF1F13098959EA
:10BA90009309400EFD1497000000E7802083634265
:10BAA000A40A97F0FFFFE78060094169B729090000
:10BAB000096AFD7A2A8B81447D199389F97B130ADF
:10BAC0000A71938A8AC797000000E780208063D7B5
:10BAD000A4041304400EB387840217A7FF1F1307A3
:10BAE00067540324070B3E948357C4016382270BDA
:10BAF00018403307EB4063EAE900834744008507B9
:10BB0000B3874703D6976365F70801468145094522
:10BB100097F0FFFFE780C04AAA8B29E59740000015
:10BB2000E780808385476317F506896593850571EE
:10BB300017A5FF1F1305452C97100100E780A04FA4
:10BB400095A0B30734030327090BBA9703D7C7019E
:10BB50006308970003C75700A38207002382E7000A
:10BB6000050415BF9305C500228597000000E780F6
:10BB700080E65E85228697650100938565E097F0F3
:10BB8000FFFFE780404F5E8597100000E780608AE6
:10BB9000850415BF97A7FF1F9387C7489C478D83D0
:10BBA000858BC1F721611763FFFF6700435401468E
:10BBB0008545094502D002D202D402D697F0FFFF94
:10BBC000E7800040AA8479DD97F00000E780E09CE0
:10BBD0001389C4002A8481454A8597000000E780C4
:10BBE000005F0C4041464A8597000000E780405BBB
:10BBF000832944006385090C4E8502D802DA02DCF1
:10BC000002DE97300100E780E0382ACE14100546A6
:10BC10002C0808184ECC97500000E780E00A1375F6
:10BC2000F50F51ED8355840093E525004A85970073
:10BC30000000E780E05E11460C104A859700000086
:10BC4000E78000560146976501009385E5D3268578
:10BC500097F0FFFFE7802042268597000000E780ED
:10BC6000407D5C40A1D3014685450D4597F0FFFF1F
:10BC7000E7800035AA841DD548401389C400973059
:10BC80000100E78020312AC64A8597000000E7803E
:10BC9000404C3246636FC5004C404A859700000017
:10BCA000E780005001468145268597F0FFFFE78039
:10BCB000803C268597000000E780A077E5B5835596
:10BCC0008400ADB71763FFFFE702634197A7FF1F2B
:10BCD000938747359C471DC193E7870017A5FF1F32
:10BCE0001305851117A7FF1F2322F73497100100B2
:10BCF000E78040321763FFFF6700A340DD9B17A773
:10BD0000FF1F2325F73297300000E780E0647DF1C4
:10BD100017A5FF1F1305450E97100100E780E033BC
:10BD2000D1BF1763FFFFE70203394169AA892E8A51
:10BD3000B28A368BBA8B814417ACFF1F130C8C2E42
:10BD4000930C400E7D1997F0FFFFE780205863C4E5
:10BD5000A40001443DA03384940383270C0B3E943C
:10BD60008357C401638627055A87D6865286CE85B7
:10BD70001305040397000000E780E0BB01C923809E
:10BD80000B0022851763FFFF670063368347F401CA
:10BD900085C35A87D6865286CE85130594089700A8
:10BDA0000000E78040B909C585472380FB00D1BF6B
:10BDB000850451BF835745006380071E1763FFFF4B
:10BDC000E702433001112A8497000000E780C04D4C
:10BDD00009C985476309F50605611763FFFF670019
:10BDE000A33197E00000E780007C7DF58357440095
:10BDF0004947ED9BE392E7FEC1452285970000008D
:10BE0000E7804033AA84228597000000E780204F16
:10BE10000357440002CE91472A89631AF70022850E
:10BE200097000000E780A0513C082ACC3ECE97E066
:10BE30000000E78080765C55C5D374084A86A685E5
:10BE40000545829751BF03574400D147E3F6E7F811
:10BE5000032A0400C169014997AAFF1F938A8A1C1B
:10BE6000130B400EFD1997F0FFFFE7802046634F4C
:10BE7000A90E2285032A040097000000E780C04233
:10BE8000A1452A89228597000000E780A02AAA847C
:10BE9000228597000000E780804A14402A86AA89FC
:10BEA00078082685CA8597000000E780C0E7AA8445
:10BEB00005D503C7F40189476315F7008347C1011E
:10BEC00081DF5546D2851385640097300100E780F5
:10BED000E0E7014597800000E780C01901C583D7DE
:10BEE000C401A5E797A7FF1F9387C7139C479355E6
:10BEF0001900858913D73700058B01CF8983858B7E
:10BF00006399B70001452EC697000000E780C0DBAB
:10BF1000B2454E8597800000E780601F0346C1014F
:10BF20002A8493751900268597900000E780E039F0
:10BF300035C1268597800000E780E018268511C06E
:10BF4000014597800000E780004C97300000E780B3
:10BF5000A0408547E312F5E883C754001307F00FAC
:10BF6000E38CE7E68507A382F400BDB5B30469035B
:10BF700083A70A0BBE9483D7C401638B3701554650
:10BF8000D2851385640097300100E780C0D955DD64
:10BF90000509D1BD5DD86DB782801763FFFFE70249
:10BFA000631297800000E780000C05C1C164014462
:10BFB00017A9FF1F130909079309400EFD1497F0F5
:10BFC000FFFFE780A030634EA40017A5FF1F1305F5
:10BFD000A5E297100100E780E0031763FFFF670009
:10BFE000A311330534038327090B3E958357C501FD
:10BFF000638897002312050097800000E780A00C5B
:10C00000050475BF97A7FF1F9387C7019C478D83C2
:10C01000858B8DE31763FFFFE702630C17A5FF1FF6
:10C02000130585DD97100100E78020031763FFFFEC
:10C030006700230D82801763FFFFE702430A97051D
:10C0400000009385C5A017A5FF1F1305E5DA97101B
:10C050000100E78020EE1763FFFF6700830A176384
:10C06000FFFFE702C3078841B7E70400BC5B050593
:10C0700042054181829709C585472300F5000505E2
:10C080001763FFFF6700E30783C7F5FF2E8585076A
:10C09000A38FF5FE828083C7F5FFFD1793F7F70F97
:10C0A000A38FF5FE99EF1763FFFFE7024303B7E79E
:10C0B0000400BC571385F5FF82971763FFFF6700E5
:10C0C000430482801C41035745008D8FBA951CC1E3
:10C0D0002312B5003E85828093D78500A2051441C6
:10C0E000DD8D835745001387E6FF18C189072312AA
:10C0F000F50013D685004111238FB6FEA38FC6FE2F
:10C100004101828018419307F7FF1CC18357450006
:10C1100085072312F500A30FB7FE828083574500E1
:10C120008D8F2312F5001C41BE950CC12E85828097
:10C13000AA8703D7470008410D8FAA952392E700ED
:10C140008CC38280184108453305A74082808357FD
:10C150004500035765001D8F1C4108453385A740E6
:10C160003305A74082801763FFFFE70243F74111C1
:10C170002EC62A8497000000E780A0FDB2456373B5
:10C18000B50001A0835744000840BE952312B400B7
:10C190003E9541011763FFFF6700A3F61763FFFF9A
:10C1A000E702E3F341112E84B28532C69700000006
:10C1B000E780A0FB3246A28597300100E78000B9F6
:10C1C00041011763FFFF6700C3F31763FFFFE70237
:10C1D00003F12E84854597000000E78000F92300D5
:10C1E00085001763FFFF6700C3F11763FFFFE702D6
:10C1F00003EF41112317B100894597000000E78044
:10C20000C0F68347E1002300F5008347F100A30057
:10C21000F50041011763FFFF6700A3EE1763FFFFFF
:10C22000E702E3EB93D78500A2054111DD8D2317CB
:10C23000B100894597000000E78020F38347E100C3
:10C240002300F5008347F100A300F50041011763C7
:10C25000FFFF670003EB1763FFFFE70243E8139755
:10C26000850193D78501C166938606F0D98F13D7D0
:10C270008500758FD98FA2053707FF00F98D411111
:10C28000DD8D2EC6914597000000E78000EE6C0022
:10C29000114697300100E78060AB41011763FFFF53
:10C2A000670023E61763FFFFE70263E31C41854550
:10C2B00003C4070097000000E78080E6228517632B
:10C2C000FFFF670003E41763FFFFE70243E11C4140
:10C2D0004111894503C7070083C717002307E10001
:10C2E000A307F10097000000E78080E30355E10019
:10C2F00041011763FFFF6700C3E01763FFFFE70219
:10C3000003DE1C414111894503C7070083C717009D
:10C310002307E100A307F10097000000E78040E059
:10C320008357E100410113D58700A2075D8D4205C7
:10C3300041811763FFFF6700C3DC1763FFFFE7025C
:10C3400003DA0C4141112A8411466800973001003C
:10C35000E780C09F9145228597000000E78040DC80
:10C36000B247C166938606F01397870113D58701FC
:10C37000598D13D78700758F598DA2073707FF0096
:10C38000F98F5D8D41011763FFFF670083D71C455F
:10C39000BE950CC18280AE87944391E6584101EF6F
:10C3A0000CC15CC1828003C7570013671700A382CA
:10C3B000E700B687D5B70CC3EDB7AA87084119CDFA
:10C3C0001841D44398C36313D500D8C32A870346C2
:10C3D00057009376160081E623200700828094435D
:10C3E00081CA8C4203A847008CC363930601CCC367
:10C3F000799A14C3A302C7003687D1BF1C45DC4716
:10C400001D8DB777DBB6938777DB09853305F5029A
:10C41000420541818280F147B385F50248452E955A
:10C4200082808347450085072302F50082801763D9
:10C43000FFFFE702C3CA2A8409E41763FFFF67000E
:10C4400043CC83474400F5DBFD1793F7F70F230236
:10C45000F400E5F71C4403D7270005072391E70004
:10C46000DC4399C3228582974C4889CD8347540089
:10C47000898B99E71C4422859C479C439C47829763
:10C48000232A04000040232004007DB71763FFFF28
:10C49000E702E3C48357250041112EC681EB014416
:10C4A000228541011763FFFF6700A3C503570500FD
:10C4B0008147F146E305F7FEB385D702404585077E
:10C4C0002E948345440008C4F5F5B247AA8481E759
:10C4D000232A040009A81C456C0022859C439C4328
:10C4E000829748C84DDD85472312F400B2472320C8
:10C4F0000400231804002319F4005C485CC483D7AB
:10C500002400FD172391F40061BF1763FFFFE702CA
:10C5100003BD97A7FF1F9387279088432326050015
:10C5200023240500410597100100E78000B317633D
:10C53000FFFF670003BD1763FFFFE70243BA17A4BD
:10C54000FF1F1304648D1C40411199CF9C472300A9
:10C55000B5002AC65CC197000000E78040FB1C4084
:10C56000DC4399C33245829741011763FFFF67009F
:10C5700043B90347450029E3584DAA877D551DCF90
:10C580001763FFFFE702A3B51CC3DC4797A6FF1F95
:10C5900023A4E688F156130507012390D7009705D9
:10C5A00000009385050297100100E780A0980145DF
:10C5B0001763FFFF6700E3B47D55828082801763B5
:10C5C000FFFFE702C3B10111614681452800976072
:10C5D000FFFFE780C0B397A7FF1F9387E7839C43C4
:10C5E00028009305F00FDC473EC697000000E78067
:10C5F000C0F405611763FFFF6700A3B097A7FF1F93
:10C60000938787819C43D847A1679387C702631E9E
:10C61000F70A397106DE22DC26DA80004AD84ED6C7
:10C6200052D456D23285B28497000000E780C0C74A
:10C63000AA89268597000000E78020C92318A4FC5A
:10C64000268597000000E78040C82319A4FC2685B2
:10C6500097000000E78060C783D744000A8A231A46
:10C66000A4FC858393F7F70F230EF4FC8607BD0720
:10C6700093F7073F3301F1408A8A01498347C4FD9C
:10C680006367F902CE85130584FC232C54FD9700C3
:10C690000000E78080EA5281130104FCF2506254EA
:10C6A000D2544259B259225A925A21618280268527
:10C6B00097000000E78060C193171900D69705091D
:10C6C0002390A7001379F90F55BF82809797FF1F1A
:10C6D000938787749C43D847A1679387A702631AFF
:10C6E000F70A397106DE22DC26DA80004AD84ED6F7
:10C6F00052D456D23285B28497000000E780C0BA87
:10C70000AA89268597000000E78020BCFD572318E2
:10C71000A4FC26852319F4FC97000000E780E0BA0A
:10C7200083D744000A8A231AA4FC858393F7F70F62
:10C73000230EF4FC8607BD0793F7073F3301F14052
:10C740008A8A01498347C4FD6367F902CE851305D0
:10C7500084FC232C54FD97000000E78000DE52810A
:10C76000130104FCF2506254D2544259B259225A75
:10C77000925A21618280268597000000E780E0B40C
:10C7800093171900D69705092390A7001379F90F7D
:10C7900055BF82809797FF1F938707689C43D847B0
:10C7A000A16789076310F70A397106DE22DC26DAF1
:10C7B00080004AD84ED652D456D23285328997005C
:10C7C0000000E78060AEAA894A8597000000E780F4
:10C7D000C0AF835749000A8A2318A4FC858393F7C6
:10C7E000F70F230CF4FC8607BD0793F7073F3301CF
:10C7F000F1408A8A8144834784FD63E7F402CE8551
:10C80000130584FC232A54FD97000000E780E0D242
:10C810005281130104FCF2506254D2544259B2596D
:10C82000225A925A216182804A8597000000E7804F
:10C83000C0A993971400D69785042390A70093F47A
:10C84000F40F55BF82809797FF1F9387E75C9C4347
:10C85000D847A1679387E704631EF70A397106DE9C
:10C8600022DC26DA80004AD84ED652D456D23285FF
:10C87000B28497000000E78020A3AA89268597004C
:10C880000000E78080A42318A4FC26859700000000
:10C89000E780A0A3231AA4FC268597000000E78068
:10C8A000C0A283D744000A8A2319A4FC858393F786
:10C8B000F70F230EF4FC8607BD0793F7073F3301FC
:10C8C000F1408A8A01498347C4FD6367F902CE8536
:10C8D000130584FC232C54FD97000000E780E0C57D
:10C8E0005281130104FCF2506254D2544259B2599D
:10C8F000225A925A21618280268597000000E780A3
:10C90000C09C93171900D69705092390A7001379A7
:10C91000F90F55BF82809797FF1F9387E74F9C437E
:10C92000D847A1679387C704631AF70A397106DEEF
:10C9300022DC26DA80004AD84ED652D456D232852E
:10C94000B28497000000E7802096AA892685970088
:10C950000000E7808097FD572318A4FC2685231A42
:10C96000F4FC97000000E780409683D744000A8AD1
:10C970002319A4FC858393F7F70F230EF4FC860795
:10C98000BD0793F7073F3301F1408A8A0149834786
:10C99000C4FD6367F902CE85130584FC232C54FD86
:10C9A00097000000E78060B95281130104FCF25047
:10C9B0006254D2544259B259225A925A2161828009
:10C9C000268597000000E780409093171900D697BE
:10C9D00005092390A7001379F90F55BF8280979717
:10C9E000FF1F938767439C43D847A167DD07631701
:10C9F000F7041753FFFFE702836E797132853284A3
:10CA000097000000E780408A2AC622859700000030
:10CA1000E780A08B2311A102228597000000E78008
:10CA2000A088B2452300A102280897000000E780F3
:10CA3000C0B045611753FFFF6700A36C82809797D2
:10CA4000FF1F9387673D9C43D847A167938787045F
:10CA50006317F7041753FFFFE702636879713285A4
:10CA6000328497000000E78020842AC62285970040
:10CA70000000E78080852311A10222859700000035
:10CA8000E7808082B2452300A102280897000000B9
:10CA9000E780A0AA45611753FFFF67008366828085
:10CAA0009797FF1F938747379C43D847A167938782
:10CAB000A7046312F7021753FFFFE7024362011155
:10CAC0002800814597000000E78020A705611753E3
:10CAD000FFFF6700036382809797FF1F9387C73329
:10CAE0009C43D847A167938757026319F7021753EE
:10CAF000FFFFE702C35E0111328597F0FFFFE78079
:10CB0000A07A2308A1008145280097000000E78053
:10CB1000C0A205611753FFFF6700A35E828097974D
:10CB2000FF1F9387672F9C43D847A1679387E7022E
:10CB3000631BF7041753FFFFE702635A01113285A5
:10CB4000328497F0FFFFE7804078AA84228597F02F
:10CB5000FFFFE7808077854709E9228597F0FFFF8F
:10CB6000E78080744205B337A00028008145231870
:10CB700091003ECA97000000E780209C0561175392
:10CB8000FFFF6700035882809797FF1F9387C7288E
:10CB90009C43D84799476313F7081753FFFFE702F1
:10CBA000035479713285328497F0FFFFE780C06FBC
:10CBB0002AC6228597F0FFFFE78020712310A1028B
:10CBC000228597F0FFFFE780206E2301A1022285D6
:10CBD00097F0FFFFE780406DA301A102228597F047
:10CBE000FFFFE780606C2302A102228597F0FFFF20
:10CBF000E780806B2313A102228597F0FFFFE78077
:10CC0000A06AB2452314A102280897000000E7801B
:10CC1000C09245611753FFFF6700A34E828097972C
:10CC2000FF1F9387671F9C43D847A1679387C7035C
:10CC30006313F7081753FFFFE702634A79713285E0
:10CC4000328497F0FFFFE78020662AC6228597F09E
:10CC5000FFFFE78080672310A102228597F0FFFF86
:10CC6000E780A0662311A102228597F0FFFFE780ED
:10CC7000A0632302A102228597F0FFFFE780C06234
:10CC8000A302A102228597F0FFFFE780E061230362
:10CC9000A102228597F0FFFFE7800061B245A30360
:10CCA000A102280897000000E780208945611753FA
:10CCB000FFFF6700034582801753FFFFE70223420F
:10CCC00001112A8497F0FFFFE780005EAA84228585
:10CCD00097F0FFFFE780605F228597F0FFFFE78016
:10CCE000C05E035744008D4763F7E700228597F045
:10CCF000FFFFE780805D228597F0FFFFE780E05C23
:10CD00002800A68597000000E7802083056117535F
:10CD1000FFFF6700033F9797FF1F9387E70F9C4331
:10CD2000D847A167FD07631FF7001753FFFFE7020E
:10CD3000033B328597000000E78040F81753FFFF60
:10CD40006700233C82809797FF1F9387E70C9C43E3
:10CD5000D847A167E5076315F7081753FFFFE702F8
:10CD6000033879713285328497F0FFFFE780C05332
:10CD70002AC6228597F0FFFFE7802055228597F08D
:10CD8000FFFFE78080542310A102228597F0FFFF68
:10CD9000E780A053520551812311A102228523026D
:10CDA000010297F0FFFFE7802050A302A102228535
:10CDB00097F0FFFFE780404F2303A102228597F001
:10CDC000FFFFE780604EB245A303A102280897F059
:10CDD000FFFFE780807645611753FFFF67006332EE
:10CDE00082809797FF1F938727039C43D847A167AB
:10CDF0009387E703631FF7001753FFFFE702232E14
:10CE0000328597000000E78060EB1753FFFF670053
:10CE1000432F82809797FF1F938707009C43D84733
:10CE2000A16793874704631EF7021753FFFFE702CA
:10CE3000032B79713285328497F0FFFFE780C0467B
:10CE40002AC6228597F0FFFFE7802048B2452808D0
:10CE500097F0FFFFE780606E45611753FFFF6700A3
:10CE6000432A82809797FF1F938707FB9C43D847ED
:10CE7000A167938787026310F7041753FFFFE70248
:10CE8000032679713285328497F0FFFFE780C04135
:10CE90002AC6228597F0FFFFE7800041B2452300B4
:10CEA000A102280897F0FFFFE7802069456117532A
:10CEB000FFFF6700032582801753FFFFE70223224D
:10CEC000011197F0FFFFE780203EAA85280097F028
:10CED000FFFFE780806605611753FFFF670063224D
:10CEE0009797FF1F938747F39C43D847A167D107C4
:10CEF000631FF7001753FFFFE702631E3285970099
:10CF00000000E780A0FB1753FFFF6700831F8280AC
:10CF10009797FF1F938747F09C43D847A167C507A2
:10CF2000631FF7001753FFFFE702631B328597006B
:10CF30000000E780A0F81753FFFF6700831C828082
:10CF40009797FF1F938747ED9C43D847A167B90781
:10CF5000631FF7001753FFFFE7026318328597003E
:10CF60000000E780A0F51753FFFF67008319828058
:10CF70009797FF1F938747EA9C43D847A167AD0760
:10CF8000631FF7001753FFFFE70263153285970011
:10CF90000000E780A0F21753FFFF6700831682802E
:10CFA0009797FF1F938747E79C43D84789476318A4
:10CFB000F7021753FFFFE70283120111328532C8CF
:10CFC00097F0FFFFE780402EAA85280097F0FFFF2B
:10CFD000E780A05605611753FFFF67008312828028
:10CFE0009797FF1F938747E39C43D847A1678D0717
:10CFF0006311F7041753FFFFE702630E0111328537
:10D00000328497F0FFFFE780202A13066100AA848C
:10D010004C00228597300000E780C0232800A685B9
:10D0200097F0FFFFE780605105611753FFFF67002E
:10D03000430D82809797FF1F938747DE9C4381CFE4
:10D04000DC4391CB1753FFFFE70263098297175325
:10D05000FFFF6700030B82801753FFFFE7022308DF
:10D0600079713C08AE843ED2A165B7070A002A84D4
:10D070003ED448103C08DD053ED636C432C63AC21E
:10D0800097D0FFFFE780402C12474810BA8597F0F1
:10D09000FFFFE780C01332464810B28597F0FFFFCC
:10D0A000E780E014A2464810B68597F0FFFFE780BE
:10D0B0000012501001478146A685228597D0FFFFB8
:10D0C000E780E04D45611753FFFF67008303175367
:10D0D000FFFFE702C30001117C000329C501AE84F4
:10D0E0003ECAA165B70707002A843ECC48087C00E9
:10D0F000C5053ECE97D0FFFFE78000258345D900C8
:10D10000480897F0FFFFE780800C500801478146F0
:10D11000A685228597D0FFFFE780604805611753F9
:10D12000FFFF670003FE1753FFFFE70243FB83C7C0
:10D13000950093F7F707A384F50097000000E780B8
:10D1400040F91753FFFF6700C3FB1753FFFFE702C8
:10D1500003F979713C08AE843ED2A165B707090096
:10D160002A843ED448103C08938545043ED632C6F6
:10D1700036C497D0FFFFE780201DA2464810B68531
:10D1800097F0FFFFE780A00432464810B28597F081
:10D19000FFFFE780C005501001478146A685228524
:10D1A00097D0FFFFE780A03F45611753FFFF67005F
:10D1B00043F51753FFFFE70283F283C79500411140
:10D1C0002A8493F7F707A384F50032852EC697F0DB
:10D1D000FFFFE780800F85672AC46370F5029770B0
:10D1E0000000E78020E92246B24509ED114781465B
:10D1F000228597000000E78060E641011753FFFF9A
:10D20000670023F001478346F501DDB71753FFFFA1
:10D21000E70243EB01113C003ECAB7070A003ECCCF
:10D220003C003ECE83C79500AA89328593F7F70765
:10D23000A384F5002E8497F0FFFFE780000985673F
:10D24000637DF504A165AA8493858504480897D079
:10D25000FFFFE780600F268597700000E78080E180
:10D260002A8929E19145480897F0FFFFE78020F6D9
:10D27000A685480897F0FFFFE78060F7CA85480851
:10D2800097F0FFFFE780A0F4014781465008A28590
:10D290004E8597D0FFFFE780803005611753FFFF71
:10D2A000670083E58145480897F0FFFFE78020F29B
:10D2B0000349090275BF1753FFFFE702A3E0797125
:10D2C0001C103ECAB7070F003ECC404D1C10AA846C
:10D2D000AE894808994532C636893ECE97D0FFFFC1
:10D2E000E780800632464808B28597F0FFFFE78066
:10D2F00000EE630C0902A545480897F0FFFFE780A0
:10D30000C0E62546CA8597200100E78020A4500882
:10D3100001478146CE85268597D0FFFFE7802028EC
:10D3200045611753FFFF670023DD8355C40248089A
:10D3300097F0FFFFE780A0EB0355E402814505C5A8
:10D34000854785456301F502C167FD179305F00F19
:10D35000630BF5007D1597700000E780208E930524
:10D36000150093F5F50F480897F0FFFFE78020E6DA
:10D3700083450403480897F0FFFFE78040E58345B5
:10D380001403480897F0FFFFE78060E48355240307
:10D39000480897F0FFFFE78080E58355440348087D
:10D3A00097F0FFFFE780A0E49DB71753FFFFE70268
:10D3B00003D383C795008146014693F7F707A384FB
:10D3C000F50097000000E78040EF1753FFFF67006C
:10D3D00043D31753FFFFE70283D079713E841C10BB
:10D3E0003ECA2E89B7070F00A1653ECCFD051C1073
:10D3F000AA84480842C03AC23ECE36C432C697D04C
:10D40000FFFFE78060F432464808B28597F0FFFFDF
:10D41000E780E0DBA2464808B68597F0FFFFE7808B
:10D4200000DD12474808BA8597F0FFFFE78020DC4F
:10D430000248630C08029145480897F0FFFFE78017
:10D44000C0D21146A28597200100E78020905008A5
:10D4500001478146CA85268597D0FFFFE7802014C3
:10D4600045611753FFFF6700C3C98945480897F016
:10D47000FFFFE78080CF834704002300F500834748
:10D480001400A300F500E1B71753FFFFE70283C3C1
:10D4900083C7950001112A8A93F7F707A384F50043
:10D4A0003285AE8432C697F0FFFFE78000E2324655
:10D4B0002A89328597F0FFFFE78000DF8567637375
:10D4C000F902AA894A8597700000E780A0BA2A84E9
:10D4D00019ED114781464A86A685528597000000BE
:10D4E000E780C0B705611753FFFF6700E3C093876C
:10D4F000E9FF93F7F70F0547E366F7FE8347F5016A
:10D5000095EB8947E380F9FE8346F4015285014794
:10D510004A86A68597000000E78040B4A167D90736
:10D5200048083ECC230A010002CE97000000E780A5
:10D53000A0B04DBF639EE7008947639EF900930743
:10D540001020231FF50097700000E780C0B76DBF63
:10D550000947E39BE7FA8D47E398F9FA228597702C
:10D560000000E78080DF9797FF1F938727AA9C43DF
:10D5700099E79797FF1F938727939C4399C703D5F4
:10D58000040097800000E780A0CE231F04002285BE
:10D590005DBF1753FFFFE70283B401113C003ECA91
:10D5A000B7070B003ECC3C003ECE83C795002A89CE
:10D5B000328593F7F707A384F500AE8497F0FFFF59
:10D5C000E780A0D093170501C187635AF006A165D3
:10D5D0002A849385E502480897D0FFFFE780C0D6EC
:10D5E000A285480897F0FFFFE78060C09797FF1F6C
:10D5F0009387878B9C43A9EB01449375F40F4808EC
:10D6000097F0FFFFE780A0BC9355844093F5F50F9A
:10D61000480897F0FFFFE78080BB9355044193F5DE
:10D62000F50F480897F0FFFFE78060BA0147814691
:10D630005008A6854A8597D0FFFFE78040F6056130
:10D640001753FFFF6700E3AB416585460546A2859A
:10D650007D1597500000E78060BD59DD51059700AA
:10D660000100E780808F130440063344850271B7C0
:10D670001753FFFFE702A3A60111B70706003EC636
:10D6800083C7950021642A8993F7F707A384F500DF
:10D69000AE8428009305A4040AC40AC897D0FFFFEB
:10D6A000E78080CA300001478146A6854A8597D029
:10D6B000FFFFE780C0EE97E0FFFFE780E011130473
:10D6C0009404480822CC230A010002CE97000000EF
:10D6D000E780809605611753FFFF670083A2175309
:10D6E000FFFFE702239EC1642A8901449799FF1F27
:10D6F00093894993130A8002FD1497E0FFFFE780A6
:10D70000E0BD6347A40001451753FFFF6700C39EB8
:10D71000B307440303A7C90ABA9703D707006306F0
:10D72000970083D72700638427010504F9B70545CF
:10D73000E1BF1753FFFFE702E3982A8A2E8999C1B8
:10D7400023A0050081498144978AFF1F938A4A6D6F
:10D75000614B97E0FFFFE780A0BE63C7A4004E8542
:10D760001753FFFF670043993384640383A70A00BC
:10D770003E948357040099E763040900232089003D
:10D780008504C1BF4146D2851305440097100100AE
:10D79000E780605975F5A289E5B71753FFFFE702E7
:10D7A000639239717C083ED4B7070A003ED67C08E4
:10D7B0003ED883C795002A8A328593F7F707A3845A
:10D7C000F5002E8932C697F0FFFFE78000B085672D
:10D7D0006373F5083246AA84328597F0FFFFE7802D
:10D7E000A0AC8547AA8963E8A706A165938585044F
:10D7F000281097D0FFFFE78020B52685977000009E
:10D80000E78040872A8429ED9145281097F0FFFF93
:10D81000E780E09BA685281097F0FFFFE780209D1A
:10D82000CE85281097F0FFFFE780609A0147814678
:10D830003010CA85528597D0FFFFE78040D6A16798
:10D840009387770448183EDC230A010202DE97F032
:10D85000FFFFE780607E21611753FFFF6700C389E8
:10D860008145281097F0FFFFE7806096A685281075
:10D8700097F0FFFFE780A0979797FF1F938747B127
:10D880009C4381CB22856389090097D00000E78003
:10D8900040248345040271B797D00000E780C0227E
:10D8A000CDBF1753FFFFE702E38183C79500411106
:10D8B000AA8993F7F707A384F5003285AE84328AEC
:10D8C00097F0FFFFE78060A08567637FF5022A89F4
:10D8D00097600000E780007A2A84914631C583472B
:10D8E000F50105476387E70291C70D476366F704B3
:10D8F000AD461DA89305050303250A004146971070
:10D900000100E78040420DE941011743FFFF670036
:10D91000A37E9305950803250A0041469710010050
:10D92000E7806040814669F54A86A6854E85970066
:10D930000000E780C081C9BF83250A001305940851
:10D9400097700000E780A02919C1C146F1BF9787F1
:10D95000FF1F9387A76B9C4399E79787FF1F9387C8
:10D96000A7549C4399C7228597800000E780208AAE
:10D9700069FD8547A30FF400228597B00000E7807A
:10D980006084228597600000E780E0734E858146C1
:10D990004A86A68597F0FFFFE780607BA1679387A3
:10D9A000570448003EC42302010002C697F0FFFF5F
:10D9B000E780806891BF1743FFFFE702C36F83C70B
:10D9C00095004111AA8993F7F707A384F5003285E2
:10D9D0002E89B28A97F0FFFFE780208F85676374F6
:10D9E000F50EAA8497600000E780C0682A840DEDD8
:10D9F000416B014A978BFF1F938BCB62130C400E38
:10DA00007D1B19A833048A0383A70B0B3E9483570D
:10DA1000C40163836705050A97E0FFFFE780008B79
:10DA2000E342AAFE95460DA08357C501639697026F
:10DA30009305050303A50A00414697100100E780FE
:10DA4000802E994611E181462686CA854E8597F03B
:10DA5000FFFFE780C06F85A883A50A0013050403B4
:10DA600097700000E780A017C14679FD2285231E2C
:10DA7000940097A00000E780E07422859760000082
:10DA8000E78060649797FF1F938787909C43A9C3A3
:10DA900023000402228597D00000E78040F04E85E5
:10DAA00081462686CA8597F0FFFFE780406AA16716
:10DAB0009387070448003EC42302010002C697F082
:10DAC000FFFFE780605741011743FFFF67002362B4
:10DAD00089472300F402E1B7397106DE22DC4AD817
:10DAE000800052D456D25AD026DA4ED65ECE2E8A36
:10DAF00032892A8B97D0FFFFE780407A06057105AF
:10DB000041998A8A3301A140232224FC231404FC76
:10DB100097D0FFFFE780807883479A000605350598
:10DB200093F7F7072315A4FCA304FA004A852326DC
:10DB300024FC97E0FFFFE780407993170501C18738
:10DB40006340F0025681130104FCF2506254D25437
:10DB50004259B259225A925A025BF24B2161828099
:10DB6000AA844A8597E0FFFFE7802076AA894A8544
:10DB700097E0FFFFE7806075A1659385C5022A895C
:10DB8000130544FC97C0FFFFE780007C268597C003
:10DB9000FFFFE7804070854511C94A86CE8597C052
:10DBA000FFFFE780C069AA8B21E98945130544FC82
:10DBB00097E0FFFFE780A061A685130544FC97E08E
:10DBC000FFFFE780C062CE85130544FC97E0FFFFAE
:10DBD000E780E061CA85130544FC97E0FFFFE7801A
:10DBE000006101478146130644FCD2855A8597D0CF
:10DBF000FFFFE780C09AB9B78145130544FC97E061
:10DC0000FFFFE780C05CA685130544FC97E0FFFF9B
:10DC1000E780E05DCE85130544FC97E0FFFFE780D9
:10DC2000005DCA85130544FC97E0FFFFE780205C98
:10DC3000814497D0FFFFE7806066E3D4A4FA83A70E
:10DC40000B0113971400BA9783D5070099C51305E4
:10DC500044FC97E0FFFFE78080598504D9BF7971C4
:10DC600006D622D44AD000184ECE52CC56CA26D25E
:10DC70005AC8AE893289AA8A97D0FFFFE78000622E
:10DC80000605690541990A8A3301A140232A24FC2B
:10DC9000231C04FC97D0FFFFE780406083C79900F6
:10DCA00006052D0593F7F707231DA4FCA384F900AF
:10DCB0004A85232E24FC97E0FFFFE780006193173D
:10DCC0000501C187634FF0005281130104FDB2507A
:10DCD000225492540259F249624AD24A424B456157
:10DCE0008280AA844A8597E0FFFFE780005EA165F5
:10DCF0009385A5022A89130544FD97C0FFFFE7809D
:10DD0000A064268597C0FFFFE780E058854509C9D4
:10DD1000CA8597C0FFFFE78080552A8B29E1894596
:10DD2000130544FD97E0FFFFE780604AA6851305D1
:10DD300044FD97E0FFFFE780804BCA85130544FD53
:10DD400097E0FFFFE780A04A01478146130644FDA4
:10DD5000CE85568597D0FFFFE7806084B5B78145B3
:10DD6000130544FD97E0FFFFE7806046A685130595
:10DD700044FD97E0FFFFE7808047CA85130544FD17
:10DD800097E0FFFFE780A046814497D0FFFFE78040
:10DD9000E050E3DBA4FA83270B0113971400BA9732
:10DDA00083D5070099C5130544FD97E0FFFFE78081
:10DDB00000448504D9BF1743FFFFE702433283477E
:10DDC0004500404DD5EFFD575DC48346940009479B
:10DDD0006363D70A0346B400854663EEC60883062C
:10DDE000E40063CA06085C45F9562390D70097877C
:10DDF000FF1F83C7270399E3A304E4009787FF1F4E
:10DE00009387870A9C4381E78947A306F400978795
:10DE1000FF1F9387E7579C4381E789472306F40058
:10DE20009705000093854506AA841305040197F021
:10DE30000000E7802010FD57231AF40281471CDC04
:10DE400001489787FF1F23AB87FC9787FF1F9387A6
:10DE500027FD232E040304C0804397D0FFFFE780F3
:10DE6000204E61463306C502814522859740FFFF5B
:10DE7000E780E02981473E851743FFFF670063285D
:10DE8000FD57D5BF1743FFFFE70263252A840355DB
:10DE9000450297600000E780E01D19E5231E04009D
:10DEA0001743FFFF6700E3258357E401F5DB930584
:10DEB00004FF174501001305E5E697E00000E78041
:10DEC000E014F9BF1743FFFFE70263212E89A16524
:10DED00041119385E5032A8436C432C6BE843AC212
:10DEE00097C0FFFFE780404612472285BA8597E03A
:10DEF000FFFFE780C02D32462285B28597E0FFFF05
:10DF0000E780E02EA2462285B68597E0FFFFE780F6
:10DF1000002E630309029145228597E0FFFFE78009
:10DF2000C0241146A68597100100E78020E2410138
:10DF30001743FFFF6700E31C8945228597E0FFFF39
:10DF4000E780A02283C704002300F50083C71400E4
:10DF5000A300F500E9BF1743FFFFE702431883C79B
:10DF60009500444D054793F7F707A384F5001C423D
:10DF7000411183C707006367F7062E842A89B1C061
:10DF800003C7D400630FF7021787FF1F1307C7F1FA
:10DF9000184305C3A386F40097A00000E780404A19
:10DFA00083C7D40099E741657D1597400000E7805D
:10DFB000403083D72403918B89C797E00000E78026
:10DFC000C0134A85A28597F0FFFFE7808010A16704
:10DFD000C10748003EC42302010002C697F0FFFFBC
:10DFE000E780800541011743FFFF67008311174356
:10DFF000FFFFE702C30E03D745008D47AA844111F6
:10E000002E8432892E8563E3E70297E0FFFFE780E5
:10E01000C02BAA8523000900268597C0FFFFE78053
:10E02000002541011743FFFF6700A30D97E0FFFFA5
:10E03000E780A0292AC6228597E0FFFFE780E02835
:10E04000B24585472A862300F900268597C0FFFF41
:10E05000E780E01EF9B7397106DE22DC26DA80009F
:10E060004ED652D456D24AD85AD05ECEAE89B28459
:10E07000AA8A97D0FFFFE7806021060513052502D5
:10E0800041990A8A3301A140232224FC231404FC71
:10E0900097D0FFFFE780801F83C7990006054D05D5
:10E0A00093F7F7072315A4FCA384F90026852326FC
:10E0B00024FC97E0FFFFE780402193170501C1870B
:10E0C0006340F0025281130104FCF2506254D254B6
:10E0D0004259B259225A925A025BF24B2161828014
:10E0E000AA8B03AB040097C0FFFFE780C01A51E57D
:10E0F00083D7440001498544F11793B71700A30162
:10E10000F4FC834734FCA165C9C79385E504130576
:10E1100044FC97C0FFFFE7802023A685130544FC3D
:10E1200097E0FFFFE780A00ADE85130544FC97E037
:10E13000FFFFE780C00B834734FC114691E309469B
:10E14000DA85130544FC97E0FFFFE7806005814412
:10E15000630A0900416B7D1B97D0FFFFE780001326
:10E1600063CCA40201478146130644FCCE85568544
:10E1700097C0FFFFE780A042B1B7A685130634FC25
:10E1800097000000E780E0E6933415002A898604B2
:10E190008DBF9385C504A5BF8327C90013971400BD
:10E1A000BA9783D5070063886501130544FC97E09F
:10E1B000FFFFE780C003850445B71743FFFFE70271
:10E1C00083EF79711C103EC4B7070F003EC61C10C8
:10E1D0003EC883C79500AA8A328593F7F707A384C0
:10E1E000F500AE89328497E0FFFFE780000E9317B9
:10E1F0000501C187635AF0062A8A228597E0FFFF4E
:10E20000E780A00C2A895285032B040097C0FFFFEA
:10E21000E780600839ED8357440081440544F117D5
:10E2200093B71700A303F10083457100DA872287B3
:10E23000CA865286280097000000E780E0C80147A0
:10E2400081463000CE85568597C0FFFFE780203598
:10E25000A1679387D70348083ECC230A810026CEC6
:10E2600097F0FFFFE78040DD45611743FFFF670040
:10E2700003E8A2851306710097000000E78060D7CD
:10E28000AA84094455D13544E30055FB4A8597F0EB
:10E29000FFFFE78000450D4441D9014497D0FFFFBF
:10E2A000E780C0FE634DA400C16B0144FD1B97D005
:10E2B000FFFFE780A0FD634EA4001544B5B7DC4422
:10E2C00013171400BA9783D7070063832703050445
:10E2D000F1B7D84493171400BA9703D70700631B0C
:10E2E000770123902701268597A00000E78080DB37
:10E2F00001441DBF050465BF1743FFFFE70283DC30
:10E3000083C7950041112A8A93F7F707A384F50084
:10E3100032852E89328497E0FFFFE78000FB931758
:10E320000501C1876353F006AA89228597E0FFFFA4
:10E33000E780A0F92311A1004E85832A040097C02D
:10E34000FFFFE78040F539E58357440085440144E9
:10E35000F11793B71700A300F1000348110003570A
:10E360002100D6875285CE862686CA8597F0FFFF84
:10E37000E7806006A167F10748003EC423029100D0
:10E3800022C697F0FFFFE78020CB41011743FFFF34
:10E39000670083D6A2851306110097000000E7806E
:10E3A00040C52A84894455D9835721001167854483
:10E3B000BA97C2071167C1831307F7EFE36FF7F846
:10E3C0009787FF1F938787C49C4381CB854513059F
:10E3D000210097500000E780207583552100228599
:10E3E000814497C0FFFFE780A0E125D923100500F5
:10E3F000228597A00000E78040CD85B71743FFFF37
:10E40000E70263CB83C7950041112A8B93F7F70787
:10E41000A384F50032852E8A328497E0FFFFE780DF
:10E42000C0EA93170501C1876351F006AA8A2285C5
:10E4300097E0FFFFE78060E92A895685832B040077
:10E4400097C0FFFFE78020E531E583574400814412
:10E450000544F11793B71700A301F10003483100F9
:10E46000DE875A854A87D6862286D28597F0FFFFB7
:10E47000E78060F6A167ED0748003EC423028100F3
:10E4800026C697F0FFFFE78020BB41011743FFFF3F
:10E490006700E3C5A2851306310097000000E780FE
:10E4A00040B5AA8409445DD99167CA97C20711672C
:10E4B000C1831307F7EF0544E362F7FACA8597C0F3
:10E4C000FFFFE780E0D3014451F9814997D0FFFF76
:10E4D000E780C0DC63DBA900984893971900BA97DE
:10E4E00003D7070005EF2390270197D0FFFFE780B0
:10E4F000E0DA1544E384A9F6268597A00000E780BA
:10E50000C0BC9787FF1F938767B09C430144B9D76E
:10E510004A8597500000E780C05889B785097DB7C4
:10E520001743FFFFE70203BA79713E847C083EC8B7
:10E530002E8AB7071400A1653ECAE5057C08AA89A2
:10E54000080836C4428932C6BA8AC6843ECC97C00F
:10E55000FFFFE78060DFCA85080897E0FFFFE780DC
:10E5600000C732460808B28597E0FFFFE78020C861
:10E57000A246630A09049D45080897E0FFFFE7806B
:10E58000C0BE1D4681459740FFFFE78040B86389C4
:10E590000A089145080897E0FFFFE78000BD114693
:10E5A000A68597000100E780607A10080147814640
:10E5B000D2854E8597C0FFFFE78060FE4561174317
:10E5C000FFFF670063B3B685080897E0FFFFE780A9
:10E5D00000C21C400808D8439355C701858912071B
:10E5E0005183B205D98D97E0FFFFE78040C01C4002
:10E5F000080883C5870097E0FFFFE78040BD1C4007
:10E60000080883C5A70097E0FFFFE78040BC1C40D7
:10E61000080883C5970097E0FFFFE78040BB85BFF0
:10E620008945080897E0FFFFE78020B483C704000E
:10E630002300F50083C71400A300F500BDB71743FE
:10E64000FFFFE70223A883C795004111AA8993F72A
:10E65000F707A384F5003285AE84328497E0FFFF8C
:10E66000E780A0C693170501C187635DF0042A897E
:10E67000032A040097C0FFFFE780E0C119E9835730
:10E6800044000548F11793B71700A307F10081462E
:10E6900031A81306F100A28597000000E78060957D
:10E6A0001DC51C459DC783D6470001480347F1009F
:10E6B00093078500D2884A86A6854E85970000007C
:10E6C000E78040E641011743FFFF6700E3A20948E6
:10E6D0007DBF1D486DBF1743FFFFE702A39E657115
:10E6E0005C083EC4B7077B013EC65C083EC883C7D2
:10E6F00095002A8A328593F7F707A384F500AE893F
:10E7000097E0FFFFE78040BA8357E100E1C7894502
:10E71000280097C0FFFFE78020C38145280097E0CD
:10E72000FFFFE780C0AA97C0FFFFE78000C9978777
:10E73000FF1F9387E7C59C431774FF1F0344846E34
:10E74000AA843334800099C3136424009777FF1F91
:10E75000938787759C4399C3136444009787FF1F71
:10E760009387C78A9C4399C31364840083D50400AC
:10E770002800014997E0FFFFE78060A783D52400C8
:10E78000280097E0FFFFE78080A683D5440028009B
:10E7900097E0FFFFE780A0A597D0FFFFE78000ABE1
:10E7A00093150501C181280097E0FFFFE78020A4B1
:10E7B000A285280097E0FFFFE78060A39C44636088
:10E7C000F902014781463000CE85528597C0FFFF90
:10E7D000E780E0DC59611743FFFF6700E391DC4409
:10E7E0001314490028003E9497E0FFFFE7806096ED
:10E7F000834744000347540089070607BA978607F2
:10E80000E36AF5FC835524002800814A97E0FFFF66
:10E81000E780E09D83454400280097E0FFFFE78004
:10E82000009B83455400280097E0FFFFE780209A73
:10E830008347440063C9FA00814A8347540063C197
:10E84000FA020509A5BF1C4413975A002800BA977D
:10E8500083D50700850A97E0FFFFE7804099C9BF8D
:10E86000032BC40093975A0028003E9B83552B002E
:10E87000850A97E0FFFFE780809783550B0028000B
:10E8800097E0FFFFE780A0964DBF1743FFFFE70229
:10E8900003855C4993E717005CC997A00000E780F7
:10E8A00020B61743FFFF6700C3851743FFFFE7024A
:10E8B00003832E84814597F0FFFFE780C0E705C5FD
:10E8C00083570500FD172310F50009C48357250061
:10E8D0002310F40097000000E78060FB0145174318
:10E8E000FFFF6700038231457DD823100400C5BFB8
:10E8F0001733FFFFE702037D83C7950041112A8A82
:10E9000093F7F707A384F50032852E89328497E0C8
:10E91000FFFFE780809B93170501C1876356F006D0
:10E92000AA89C145228597E0FFFFE780A0802A8B56
:10E930004E85832A040097C0FFFFE780C09531E928
:10E9400083574400231101000544F11793B71700C2
:10E95000A300F10081440348110003572100D6872A
:10E960005285CE862286CA8597F0FFFFE780A0A653
:10E97000A1679387170248003EC42302810026C680
:10E9800097E0FFFFE780406B41011733FFFF67000F
:10E99000A37613061100A28597F0FFFFE78060655C
:10E9A000AA8409E523110100094475B793052100E4
:10E9B0005A8597000000E78080EF835721002A8462
:10E9C000D9DB9777FF1F938767649C4381CB85458D
:10E9D0001305210097500000E780001583552100A2
:10E9E0002685314497C0FFFFE78080812DD5231015
:10E9F0000500268597900000E780206D0144A1BFA7
:10EA00001733FFFFE702A36D41112E896C00AA8422
:10EA100002C697F0FFFFE78000D20DC10357050043
:10EA200005072310E50097000000E78040E68147D6
:10EA30003E8541011733FFFF6700A36C32479547BE
:10EA400065DBCA85268597300000E780400DC14709
:10EA5000E34005FE3244854741462310F4008357C6
:10EA60000900A685130544002311F4009700010056
:10EA7000E780C02D228545BF1733FFFFE70283647F
:10EA800083C795004111AA8A93F7F707A384F5007D
:10EA90003285AE89328497E0FFFFE78000839317C9
:10EAA0000501C1876356F0062A8AC145228597D0A1
:10EAB000FFFFE7802068AA845285032B040097B0EB
:10EAC000FFFFE780407D31E98357440023110100B7
:10EAD0008544F11793B71700A300F10001440348E0
:10EAE000110003572100DA875685D2862686CE8507
:10EAF00097F0FFFFE780208EA16793870702480009
:10EB00003EC42302910022C697E0FFFFE780C05277
:10EB100041011733FFFF6700235EA2851306110032
:10EB200097F0FFFFE780E04C2A8409E523110100FC
:10EB3000894475B726859305210097000000E7807A
:10EB400060ECAA8449FD83552100228597B0FFFF20
:10EB5000E780006B49F5014997C0FFFFE78000742B
:10EB6000635DA900184893171900BA9703D70700E7
:10EB70000DEF035721002390E70097C0FFFFE780C8
:10EB8000E071630625039777FF1F938727489C430F
:10EB900099C70355210097500000E78080F0228537
:10EBA00097900000E78060521DBF050975B7954436
:10EBB0003DB705C19307F00F630FF500C547630C20
:10EBC000F5009307F5FF05453315F5004205418132
:10EBD00082800145828041657D158280B9E91733C5
:10EBE000FFFFE702C34F034506033284970000008E
:10EBF000E78060FC9305803EB305B502C205C18184
:10EC000081CD0357E402854763F8E700130504014B
:10EC100097E00000E78020428357E40241677D17B8
:10EC20006385E700FD172317F4021733FFFF670022
:10EC3000434D82801733FFFFE702E347004283C75B
:10EC40009500444D0349140093F7F707A384F5009A
:10EC500083470400220911673369F900A167B347AC
:10EC6000F90041112A8BAE8A63ECE70E834724003A
:10EC70001307C00EB91793F7F70F6373F710034725
:10EC80003400C14763EEE70E834744001307E007F3
:10EC900093C707086371F70C8349840083477400A6
:10ECA000A209B3E9F900856763F7F90A034A64002A
:10ECB000834754004E85220A336AFA0097500000B9
:10ECC000E780403B61C123962403834B3400137AD1
:10ECD000FA00239A34032388740323994403938905
:10ECE0000401631C090023A60402239804024E8534
:10ECF00097E00000E78060363DA0034924004A8584
:10ED000097000000E78020EB2397A402834744008C
:10ED10004E85A388F402E38D0BFCE30B09FC97E01E
:10ED20000000E780202F97900000E7800073814665
:10ED30000146D6855A8597E0FFFFE7800058A16716
:10ED4000938797033EC423020100480002C697E060
:10ED5000FFFFE780602E41011733FFFF6700233973
:10ED60008544A2862686D6855A8597E0FFFFE780F0
:10ED7000C054A167938797033EC423029100F1B763
:10ED8000BD44C5B79144F1BF1733FFFFE70283339A
:10ED900001111C08404D3EC2B7070F003EC41C08BD
:10EDA0003EC62A89AE8997C0FFFFE78000D7585C2E
:10EDB0001C5C6346B70E6394E50063E2A70E3385DF
:10EDC000A740B3B7A700B305B7401306803E8146FE
:10EDD0009D8D97000100E78080B793140501C180E5
:10EDE000A1659385C503480097B0FFFFE780C05534
:10EDF0008145480097D0FFFFE780603D83550404BC
:10EE0000480097D0FFFFE780803E835524044800E8
:10EE100097D0FFFFE780A03D814589CCC167FD17F2
:10EE20009305F00F6388F400268597500000E78073
:10EE3000E0E0AA85480097D0FFFFE78040390355FE
:10EE40004404814501CDC167FD179305F00F6307A9
:10EE5000F50097500000E78060DEAA85480097D053
:10EE6000FFFFE780C03683456404480097D0FFFF6A
:10EE7000E780E03583457404480097D0FFFFE780C2
:10EE80000035500001478146CE854A8597B0FFFF87
:10EE9000E780E07005611733FFFF6700E3258144D9
:10EEA00081B71733FFFFE702832383C7950093F7EA
:10EEB000F707A384F50097000000E78020ED1733E3
:10EEC000FFFF670003241733FFFFE702A31F83C779
:10EED00095004111404D93F7F707A384F5002A8A66
:10EEE0003285B284AE8997D0FFFFE780003E2A8B3F
:10EEF000268597D0FFFFE780403D2A89268597D059
:10EF0000FFFFE780603A93170B0163CA0702E177BE
:10EF1000CA97C207C183116763E3E7029307091029
:10EF2000C207C1831307B00F637BF7009317090172
:10EF3000C187AA8A634AF000C54763FE57014101B1
:10EF40001733FFFF6700431B97B0FFFFE7802025C3
:10EF5000E31725FFD5B763080B0263060902814456
:10EF600063890A02B7077F00231064052311240573
:10EF70007CC0568597000000E780E0C39304803E84
:10EF8000B304950239A0B7077F00232004047CC096
:10EF900081440355240497E00000E780A0A3A1C4A6
:10EFA00097C0FFFFE78060B7269593D7F4413337CA
:10EFB0009500AE97BA9708DC5CDCCE855285970049
:10EFC0000000E780A0DC99E023220404A167938776
:10EFD000B70348003EC42302010002C697E0FFFFCA
:10EFE000E7808005A9BF814701481CDC232E04036C
:10EFF000E9B71733FFFFE702830E97C0FFFFE780F3
:10F000002034E1473305F502914597500000E78031
:10F0100000C5E55711C59777FF1F23A3A7E08147D8
:10F020003E851733FFFF6700C30D85471777FF1F26
:10F03000230AF7DE82801733FFFFE702430A977740
:10F04000FF1F9387A7DD80433DC08357040463906F
:10F05000A70683572404639CB7043689B28497C0FB
:10F06000FFFFE78080AB5C5C63C3B7046395B700C8
:10F070001C5C63EEA7028347640463F3F400A68775
:10F080002303F4048347740463F39700A687A30360
:10F09000F4048357440441677D176385E7008507BF
:10F0A0002312F4043C4481C7CA852685829717330E
:10F0B000FFFF670003059777FF1F938727D69C43C1
:10F0C000014599C303C5870082801733FFFFE7021C
:10F0D00003010111B70707003EC683C79500584DCD
:10F0E0000AC493F7F7070AC8A384F5002A89AE84F7
:10F0F00011CB1C4283C707002304F7009790000040
:10F10000E7800034216493055402280097B0FFFF84
:10F11000E780802397000000E78020FAAA85280076
:10F1200097D0FFFFE780A00A300001478146A685FF
:10F130004A8597B0FFFFE7808046130444024808E1
:10F1400022CC230A010002CE97E0FFFFE780C0EE49
:10F1500005611733FFFF6700C3FA1733FFFFE702AC
:10F1600003F801117C003ECAB70707003ECC7C00C3
:10F170003ECE83C795002E84AA8493F7F707A38415
:10F18000F500A16593855502480897B0FFFFE78019
:10F19000A01B97000000E78040F2AA85480897D09E
:10F1A000FFFFE780C002500801478146A2852685FF
:10F1B00097B0FFFFE780A03E05611733FFFF6700B0
:10F1C00043F49777FF1F938767C59C43094599C30D
:10F1D00003C5970082809777FF1F938727C49C43BE
:10F1E000094599C303C5D70082809777FF1F93878E
:10F1F000E7C29C43014599C303C5A700828017332A
:10F20000FFFFE70223EC0111B70708003EC683C7E2
:10F210009500404D0AC493F7F7070AC8A384F50088
:10F220002A89AE8429C41442854703C7060063E0D7
:10F23000E70A83479400094681496380C702B30700
:10F24000F740A304E400B339F00083C71600230598
:10F25000F40097900000E780A01E03572403058B5D
:10F2600019C76386090097D00000E78000E9216490
:10F2700093058402280097B0FFFFE780E00C970019
:10F280000000E78040F4AA85280097D0FFFFE780C0
:10F2900000F497000000E78080F5AA85280097D049
:10F2A000FFFFE780C0F2014781463000A6854A850E
:10F2B00097B0FFFFE780A02E13047402480822CC09
:10F2C000230A010002CE97E0FFFFE780E0D6056148
:10F2D0001733FFFF670043E21733FFFFE70223E026
:10F2E00001117C003ECAB70708003ECC7C003ECE30
:10F2F00083C795002E84AA8493F7F707A384F500AB
:10F30000A16593858502480897B0FFFFE780C00399
:10F3100097000000E78020EBAA85480897D0FFFF00
:10F32000E780E0EA97000000E78060ECAA854808E3
:10F3300097D0FFFFE780A0E9500801478146A285EA
:10F34000268597B0FFFFE780802505611733FFFF13
:10F35000670023DB9777FF1F938747AC9C430145EA
:10F3600099C303C5B70082801733FFFFE70223D795
:10F370000111B70707003EC683C79500404D0AC478
:10F3800093F7F7070AC8A384F5002A89AE8405C855
:10F390001C42054783C707006368F7060347B400AC
:10F3A000630FF700A305F40097900000E780400981
:10F3B0008347B400B9CF97D0FFFFE78040BE2164F8
:10F3C0009305B400280097B0FFFFE780E0F79700AF
:10F3D0000000E78060F8AA85280097D0FFFFE7804B
:10F3E00000DF014781463000A6854A8597B0FFFFC0
:10F3F000E780E01A2904480822CC230A010002CE43
:10F4000097E0FFFFE78040C305611733FFFF670008
:10F4100043CF97D0FFFFE78020BF55B71733FFFFDB
:10F42000E702E3CB01117C003ECAB70707003ECCE0
:10F430007C003ECE83C795002E84AA8493F7F707FD
:10F44000A384F500A165AD05480897B0FFFFE780EC
:10F45000A0EF97000000E78020F0AA85480897D029
:10F46000FFFFE780C0D6500801478146A285268568
:10F4700097B0FFFFE780A01205611733FFFF670019
:10F4800043C89777FF1F938767999C43094599C3A2
:10F4900003C5C70082801733FFFFE70243C4011191
:10F4A0007C00AE843ECAA165B70707002A843ECC23
:10F4B000D1057C0048083ECE97B0FFFFE780C0E84A
:10F4C00097000000E78020FCAA85480897D0FFFF3E
:10F4D000E780E0CF500801478146A685228597B096
:10F4E000FFFFE780C00B05611733FFFF670063C1B3
:10F4F0001733FFFFE702A3BE83C7950093F7F70713
:10F50000A384F50097000000E78020F91733FFFF80
:10F51000670023BF1733FFFFE702C3BA83C7950015
:10F520000329C501411193F7F707A384F5001C4295
:10F5300083C90700854763E637079777FF1F9387DF
:10F5400027E59C432E84AA8485CF97000000E7809E
:10F5500080F389476306F502630409028347C90003
:10F56000638037032306390197900000E78040ED60
:10F5700083572903898B89C797D00000E780E0B7BC
:10F580002685A28597000000E78020F1A167CD07BE
:10F5900048003EC42302010002C697E0FFFFE78057
:10F5A000A0A941011733FFFF670003B59777FF1F3D
:10F5B0009387C7869C431D4599C303C5E700828096
:10F5C0001733FFFFE702A3B10111B70707003EC6DB
:10F5D00083C79500584D0AC493F7F7070AC8A38458
:10F5E000F5002A89AE8415C71C4283C7070093968D
:10F5F0008701E18663C4060685466381D706834694
:10F60000E7006388F6002307F70097900000E78083
:10F6100020E321649305E400280097B0FFFFE78012
:10F62000A0D297000000E780A0F8AA85280097D014
:10F63000FFFFE780C0B9014781463000A6854A85B3
:10F6400097B0FFFFE780A0F53504480822CC230AD5
:10F65000010002CE97E0FFFFE780009E05611733AF
:10F66000FFFF670003AA1733FFFFE70243A701115B
:10F670007C003ECAB70707003ECC7C003ECE83C765
:10F6800095002E84AA8493F7F707A384F500A1655B
:10F69000B905480897B0FFFFE78000CB970000004E
:10F6A000E78000F1AA85480897D0FFFFE78020B2E5
:10F6B000500801478146A285268597B0FFFFE78065
:10F6C00000EE05611733FFFF6700A3A31733FFFFA9
:10F6D000E702439FAA8401441769FF1F1309497475
:10F6E000E14997C0FFFFE780A0C56344A40001453E
:10F6F00019A833053403832709003E958357250055
:10F700006397970011051733FFFF6700E39E050419
:10F71000C9BF032E8500630A0E121773FF1F130360
:10F72000E38E03230300631503002943639006124D
:10F7300003234E01631503001D436399071017331C
:10F74000FFFFE7024397C689428A3E89BA8AB68498
:10F75000328BAE8B2A84B5E103554E0019E5014387
:10F760001A851733FFFF67008398A167A98F116778
:10F7700063FBE70097000000E78080F5814597F084
:10F78000FFFFE780C0120844B70700E05841F98F37
:10F7900018455CC1B707001FF98F1CC55C4991C7AC
:10F7A000610597E00000E780408BE38A09FA228533
:10F7B00097900000E78060C65DB7328597C0000073
:10F7C000E78040430D4349DD1C44116703D54700E2
:10F7D000A167A98F63FBE70097000000E78040EF77
:10F7E000814597F0FFFFE780800C03238400931688
:10F7F0004B01D1828347B300035663008588FD8B9C
:10F80000A305F300FD777D8E558EFD76FD16B204BF
:10F81000F18E83274301C58E231273012313D30076
:10F820002304530123052301A3044301BDDF2285E3
:10F8300097B0FFFFE78080C9AA850844B5D161056C
:10F8400097D00000E780207F8DB71D431A85828006
:10F850001733FFFFE70203870569AA84AE89328A5E
:10F860000144FD5A7D1997C0FFFFE78020A263473E
:10F87000A40001451733FFFF67000388D84493179E
:10F880001400BA9703D70700631F3703239057016B
:10F8900063070A00268597900000E780A0809C44BB
:10F8A0009DC383D76700B3F72701639E3701D288D2
:10F8B00001488147014781460146814526859700D9
:10F8C0000000E78040E5050479BF1723FFFFE7024A
:10F8D000637F79711C103EC4B7070F003EC61C1031
:10F8E0003EC883C79500AA8A328593F7F707A38499
:10F8F000F5002E89328497D0FFFFE780009D931793
:10F900000501C187635AF006AA89228597D0FFFFB7
:10F91000E780A09B2A8A4E85032B040097B0FFFF47
:10F92000E780609739ED8357440081440544F1171F
:10F9300093B71700A303F10083457100DA8722878C
:10F94000D2864E86280097E0FFFFE780E057014708
:10F9500081463000CA85568597B0FFFFE78020C4F6
:10F96000A1679387F70348083ECC230A810026CE7F
:10F9700097D0FFFFE780406C45611723FFFF6700CA
:10F98000A377A2851306710097E0FFFFE78060660A
:10F99000AA84094455D1528597E0FFFFE78060D4DF
:10F9A0000D4459D90546D285268597000000E78089
:10F9B00060EA2A8451B71723FFFFE7024372835599
:10F9C00007000346270041112A842E8532C62EC423
:10F9D00097E0FFFFE780E0D001C93246A2452285CB
:10F9E00097000000E78000E741011723FFFF670051
:10F9F00043711723FFFFE702036C83C79500411192
:10FA0000AA8A93F7F707A384F5003285AE8932847A
:10FA100097D0FFFFE780608B93170501C18763577D
:10FA2000F00AC1452A8A228597C0FFFFE7808070CF
:10FA30002A8D228597D0FFFFE78020892A89228599
:10FA400097D0FFFFE7804086930705F893F7F70FFD
:10FA50001307E007AA8B637BF706228597D0FFFF89
:10FA6000E78080842A8C228597D0FFFFE780C083BF
:10FA7000AA8C5285032B040097B0FFFFE780A0817A
:10FA800039E983574400231101008144F11793B7EA
:10FA90001700A300F100054403471100835621001D
:10FAA000938784005685DA8822885286CE8597F01F
:10FAB000FFFFE78020A7A167E90748003EC42302B3
:10FAC000810026C697D0FFFFE7800057410117232A
:10FAD000FFFF6700C36113061100A28597E0FFFFD7
:10FAE000E7802051AA8409E52311010009446DB77C
:10FAF000930521006A8597F0FFFFE780A0F02A8434
:10FB000041FD835521009356C900131649018548CC
:10FB10006688E2875E87858A518226859700000085
:10FB2000E78060BF2A848DBF1723FFFFE702A35839
:10FB300083C7950041112A8B93F7F707A384F5003B
:10FB40003285AE89328497C0FFFFE7800078931733
:10FB50000501C1876352F00A2A8A228597C0FFFFF8
:10FB6000E780A076AA8A228597C0FFFFE780E0752C
:10FB70002A89228597C0FFFFE7800073930705F865
:10FB800093F7F70F1307E0072A8C6377F7062285B0
:10FB900097C0FFFFE7804071AA8C228597C0FFFFC6
:10FBA000E78080702A8D5285832B040097A0FFFF89
:10FBB000E780606E39E58357440085440144F117BE
:10FBC00093B71700A301F1000347310093078400A6
:10FBD0005A85DE882688D6865286CE8597F0FFFF26
:10FBE000E78040948D4748003EC42302910022C61E
:10FBF00097D0FFFFE780404441011723FFFF6700D4
:10FC0000034FA2851306310097E0FFFFE780603EB7
:10FC10002A84894455D99356C90013164901854849
:10FC20006A88E6876287858A5182D68597000000B8
:10FC3000E78060AEAA8449BF1723FFFFE70283482D
:10FC40002A8981440144617A916A176BFF1F130B63
:10FC5000EB3B97B0FFFFE780606463C7A400228599
:10FC60001723FFFF67004349832709009399140076
:10FC7000CE9703D5070033074501420741836364EC
:10FC8000570305C103270B0019C785453E859740DB
:10FC90000000E78060E9832709000504CE972390E0
:10FCA000070085047DB797000000E78060A28327E6
:10FCB00009000504CE972390070065D5814597F08C
:10FCC000FFFFE780C0BEF1BF1723FFFFE702833FBE
:10FCD00083C7950041112A8A93F7F707A384F5009B
:10FCE00032852E89328497C0FFFFE780005E93172C
:10FCF0000501C187635AF004AA89832A040097A0EA
:10FD0000FFFFE780405931E58357440085440144B3
:10FD1000F11793B71700A301F10003483100D6870C
:10FD200052850147CE862686CA8597D0FFFFE78099
:10FD3000806AA167F50748003EC42302910022C6ED
:10FD400097D0FFFFE780402F41011723FFFF670097
:10FD5000A33AA2851306310097E0FFFFE7806029F0
:10FD60002A8489445DD99767FF1F9387272A9C437C
:10FD700081CF044997B0FFFFE7804052AA852685CE
:10FD800097400000E78040DA130504019700000067
:10FD9000E780C0EA228597800000E7800033814435
:10FDA000ADBF1723FFFFE702033183C79500411161
:10FDB000AA8A93F7F707A384F5003285AE893284C7
:10FDC0002311010097C0FFFFE78020509317050122
:10FDD000C1876354F0062A8AC145228597C0FFFF78
:10FDE000E7804035AA8B5285032B040097A0FFFFC4
:10FDF000E780604A21E98357440085440144F117B4
:10FE000093B71700A300F100034811000357210026
:10FE1000DA875685D2862686CE8597D0FFFFE78083
:10FE2000805BA1679387270248003EC423029100AC
:10FE300022C697D0FFFFE780202041011723FFFF54
:10FE40006700E32AA2851306110097E0FFFFE78011
:10FE5000401A2A8489444DD99767FF1F9387071B4F
:10FE600098433E8901CF044997B0FFFFE7800043E4
:10FE7000AA85268597400000E78000CB1305040182
:10FE800097000000E78080DB97B0FFFFE78000412C
:10FE900095443DD9930521005E8597F0FFFFE780EB
:10FEA00060B6AA8435F11C480357210022852390AF
:10FEB000E70097800000E780402183270900A9D749
:10FEC0000355210097400000E780A0BD35BF1723F0
:10FED000FFFFE702431E83C795004111AA8A93F7EB
:10FEE000F707A384F5003285AE89328497C0FFFFFF
:10FEF000E780A03D93170501C1876351F0062A8A68
:10FF0000228597C0FFFFE780403C2A895285032B5A
:10FF1000040097A0FFFFE780003831E583574400D5
:10FF200085440144F11793B71700A301F10003487A
:10FF30003100DA8756854A87D2862686CE8597D0C5
:10FF4000FFFFE7804049A167F90748003EC423024C
:10FF5000910022C697D0FFFFE780000E41011723D2
:10FF6000FFFF6700C318A2851306310097E0FFFF6B
:10FF7000E78020082A8489445DD99167CA97C2071F
:10FF80001167C1831307F7EF8544E362F7FA9767B8
:10FF9000FF1F9387A7079843BE8B01CF044997B0F3
:10FFA000FFFFE780A02FAA85268597400000E78005
:10FFB000A0B71305040197000000E78020C897B0A0
:10FFC000FFFFE780A02D95443DD11C482285814448
:10FFD0002390270197800000E780200F83A70B0064
:10FFE000B9D74A8597400000E780A0AB89B71723AF
:10FFF000FFFFE702C30E2A844105B2849700000088
:020000040001F9
:10000000E780C0C311C5228597800000E780E00B20
:1000100081460146A685228597800000E780C04E74
:100020001C4C89C7DC4799C3228582971723FFFFA1
:100030006700230D9767FF1F938747DE9C430145A9
:1000400099C31385070182809767FF1F938707DD98
:10005000884382801723FFFFE70263089317C600D7
:10006000DD8DC2054111C1812A8432C697C0FFFFD0
:10007000E780E0173246228511829375F60F97C00C
:10008000FFFFE780C01441011723FFFF67006307EC
:100090001723FFFFE702030379713C083ED2B7073D
:1000A0000C003ED43C083ED683C79500AE842A8916
:1000B00093F7F707A384F500A165938535044810ED
:1000C00097A0FFFFE7804028C165FD150144176A2E
:1000D000FF1F130A2AF5930A400EAE892E8B2EC6F7
:1000E00097B0FFFFE780801E42059317040141810E
:1000F000C183B24563E9A702C167FD176387F500B5
:10010000481097C0FFFFE780800E501001478146DE
:10011000A6854A8597A0FFFFE780604845611723C1
:10012000FFFF670063FD3307540383270A0BBA9769
:1001300003D6C701630A3601638A35014810970068
:100140000000E78060F1DA85050451BFB285EDBF9C
:100150001723FFFFE70223F679717C083EC8B70733
:1001600011003ECA7C083ECC83C79500AA8932851F
:1001700093F7F707A384F5002E8997C0FFFFE78068
:10018000C01485676378F504A165AA848905080809
:1001900097A0FFFFE780401B268597400000E7807F
:1001A00060ED133415000A04A285080897C0FFFF0C
:1001B000E780E001A685080897C0FFFFE7802003DD
:1001C00025CC014781461008CA854E8597A0FFFFC0
:1001D000E780E03C45611723FFFF670043F1B30769
:1001E00054030327CA0ABA9703D70700631C970072
:1001F00003D6270063806505080897000000E780A4
:10020000A0E5DE8505042EC697B0FFFFE780000D50
:100210004205931704014181C183B245E3E1A7FC84
:10022000C167FD17E38FF5F8080897C0FFFFE78067
:1002300000FC41BFB285F9B7C165FD150144176ADD
:10024000FF1F130A2ADE930A80022E8BAE8B65BF36
:100250001723FFFFE702A3E81841834717008346EF
:100260000700A207D58FD207D1832390F5008347DB
:100270002700034717008D45A207D98F91832310CC
:10028000F60097C0FFFFE780A0E91723FFFF670094
:1002900043E71723FFFFE702E3E2C1640144176964
:1002A000FF1F130929D893098002FD1497B0FFFF9F
:1002B000E780C0026347A40001451723FFFF6700E2
:1002C000A3E3330534038327C90A3E95835705000A
:1002D000E38597FE0504D9BF1723FFFFE70283DEFE
:1002E0002A8AAE89B284B68A97400000E78080D817
:1002F00019E591473E851723FFFF6700E3DF2A8951
:100300004E8597C00000E780E08E2A84638E0A0441
:100310008D476DD103570500C547E31D47FD0347D2
:10032000F9018546AD47E317D7FC8347450081CFE8
:100330004146A6855D0597F00000E780C09E814795
:1003400055D9AD4745BF130965012302E500CA85AC
:10035000268597100000E780606231C1A547E38BD6
:100360000AF82302040079B705C183570500E39218
:1003700047F94146A685190597F00000E780A09A45
:1003800081472DD99947BDB74E8597000000E7807A
:1003900080F02A84954739DD130955004DBF414649
:1003A000A68523104401231134011305190097F089
:1003B0000000E780A099228597800000E780A0EAEE
:1003C00081470DBF1723FFFFE70263D179717C00DE
:1003D0003ECCB7070A003ECE7C003ED083C79500D6
:1003E000B2842E8493F7F707A384F5001306A100C7
:1003F0002A892C00268597000000E780A0E5A165EA
:1004000028088D0597A0FFFFE78000F490408355F2
:10041000A10003558100854697000000E78000ECAD
:10042000AA84AA85280897C0FFFFE78040DA035610
:10043000A10083558100280897000000E780C0C113
:10044000300801478146A2854A8597A0FFFFE780D3
:100450000015854748103ED42302910202D697D05A
:10046000FFFFE78060BD45611723FFFF670063C999
:100470001723FFFFE702A3C679717C003ECCB707C4
:100480000A003ECE7C003ED083C79500B2842E8405
:1004900093F7F707A384F5001306A1002A892C001F
:1004A000268597000000E780E0DAA16528088D0521
:1004B00097A0FFFFE78040E990408355A1000355D6
:1004C0008100814697000000E78040E1AA84AA8568
:1004D000280897C0FFFFE78080CF0356A10083550F
:1004E0008100280897000000E78000B73008014726
:1004F0008146A2854A8597A0FFFFE780400A481001
:100500002302910202D402D697D0FFFFE780C0B247
:1005100045611723FFFF6700C3BE1723FFFFE702F4
:1005200003BC97000000E78060DB1723FFFF670034
:1005300043BD9767FF1F9387A78E88438280172349
:10054000FFFFE702C3B9835725004111AE842A8417
:100550002307B10017F5FFFF130525466C0023168E
:10056000F10097A0FFFFE780804591C42285978026
:100570000000E780E0D6FD572310F40013062002A8
:100580008145130554009720FFFFE78040B84101E3
:100590001723FFFF6700E3B61723FFFFE70283B2CD
:1005A00079717C003ECCB7070A003ECE7C003ED07D
:1005B00083C79500AA89AE8493F7F7073285A38491
:1005C000F5001306A1002C0097000000E78080C80A
:1005D00003558100114497400000E780A0A915C58C
:1005E0000355A100014497B00000E780A06011CD41
:1005F000035705008357810045446318F70085457C
:1006000097000000E780E0F3014421699305390079
:10061000280897A0FFFFE78020D3A285280897C06D
:10062000FFFFE780C0BA0356A10083558100280868
:1006300097000000E78040A2300801478146A68568
:100640004E8597A0FFFFE78080F548104AD423022B
:10065000810202D697D0FFFFE780009E45611723F5
:10066000FFFF670063A91723FFFFE702A3A59757C2
:10067000FF1F9387A77A2A8488432E8915C50357BD
:1006800045038357C4016311F7022326050223188B
:100690000502410597D00000E780209C6306090011
:1006A00097800000E78060DB81449769FF1F938992
:1006B0006997130A800297B0FFFFE78020C263C4E6
:1006C000A4049757FF1F9387277E9C4399C7035520
:1006D000C40197200000E780C0BD630709002285A0
:1006E00097800000E780C0A01306400E8145228558
:1006F0009720FFFFE780A0A1FD57231EF4001723DA
:10070000FFFF6700639F3385440383A7C90A3E95B3
:10071000035705008357C4016317F700CA85970084
:100720000000E78000E2850479B71723FFFFE702A6
:10073000639983C795004111AA8993F7F707A384AA
:10074000F5003285AE8497C0FFFFE78000B885676B
:100750006378F5042A8997400000E780A09101445E
:1007600001CD83D704003144638827018545970074
:100770000000E78080EF01444E85A2864A86A68568
:1007800097D0FFFFE780A09CA167938717044800DC
:100790003EC42302810002C697D0FFFFE780C089D4
:1007A00041011723FFFF670023951723FFFFE7028F
:1007B00063919757FF1F93876766804329C401455C
:1007C00097C00000E780002181470148C1641CDC1C
:1007D000232E0403232004041769FF1F13098984AF
:1007E00001449309400EFD1497B0FFFFE78000AE6F
:1007F000634FA400814517F5FFFF1305857F97A080
:10080000FFFFE780C01B1723FFFF6700E38E330560
:1008100034038327090B3E958357C50163879700EF
:10082000854597000000E78040E4050475BF9357B5
:10083000050113D78700A380F50093170501C18335
:10084000A1832380E5002381F500A381A500828098
:100850001723FFFFE702A3882300050083C71500C5
:10086000A300F50083C725002301F50083C73500E9
:10087000A301F50083C745002302F50083C7550097
:10088000A302F50083C7650093059500A303050047
:100890002303F50023040500328597000000E7805C
:1008A00040F91723FFFF6700C3851723FFFFE70207
:1008B00063814111E9540DCD85CD93F9C5FF2E8497
:1008C0002A89AA84338AA900B7EA040063189A0225
:1008D0000D88854411CCB7E704009C5F82972AC637
:1008E00022866C003305390197E00000E78000465E
:1008F000268541011723FFFF6700038083A78A0332
:100900009104829793170501C183A183A38EF4FEFE
:1009100093570501238FF4FEA183238EA4FEA38F9A
:10092000F4FE6DB763E6D5021713FFFFE702237BE2
:10093000B28741113686BE8536C697E00000E78053
:10094000E040B246410136851713FFFF6700637B25
:10095000814636858280838705001387F5003D0533
:10096000FD8793F77708834607007D158606B58FC8
:10097000A300F5006307B7007D17834717009D8329
:10098000DDB782801713FFFFE7026375B7E7040046
:1009900083A7070932872A863A858297133515007F
:1009A0001713FFFF6700E37515C181478DC117134A
:1009B000FFFFE702C372414697E00000E78000397D
:1009C00085473E851713FFFF6700A37381473E8568
:1009D00082801DCD1713FFFFE702637041468145FA
:1009E0002A849710FFFFE7808072414681451305F6
:1009F00004039710FFFFE78080710147C16723223E
:100A0000040438C87CC805451713FFFF6700636FEF
:100A10000145828081473DCDB5CD1713FFFFE70229
:100A2000036CB2842E891306800581452A849710B1
:100A3000FFFFE780C06DCA8524C4268597000000AB
:100A4000E780C0F64146814522859710FFFFE78089
:100A5000006C3044A285228597000000E780C0F238
:100A600093040401A285268597000000E780E0EE4C
:100A7000A6851305040297000000E78000EE22859A
:100A800097000000E78020F585473E851713FFFF9C
:100A9000670023673E8582801713FFFFE7028362AA
:100AA0004111E9540DCD85CD93F9C5FF2E842A89D6
:100AB000AA84338AA900B7EA0400639844030D8826
:100AC000814411CCB7E704009C5F82972AC6228636
:100AD0006C003305390197E00000E7802027268568
:100AE00041011713FFFF6700236183A78A03910465
:100AF000829793170501C183A183A38EF4FE9357B8
:100B00000501238FF4FEA183238EA4FEA38FF4FEA0
:100B10006DB765CD1713FFFFE702C35AB28411E624
:100B200005451713FFFF6700235D2A842E890145C1
:100B3000EDD93C487848B3E6E700E5D69386F7FF61
:100B4000B3B7F6007D17032A4404BA9734C87CC8AB
:100B500063050A06C14913050A03B3894941229571
:100B6000637D3601B2862E86A68597000000E78059
:100B7000A0DB7C40BE9464C065B7CE862E86CE8551
:100B800097000000E78040DAC114D2944E992322E6
:100B90000404A2879306040103C7070003C60703E2
:100BA0008507318FA38FE7FEE398F6FE3044A285D8
:100BB000228597000000E78020DD2699C149330691
:100BC000994063EC9900A9DCA686A6851305040369
:100BD00097000000E78040D579BF8147B306F40055
:100BE0003307F6000347070083C5060085072D8FEE
:100BF0002380E600E39437FF3044A28522859700E6
:100C00000000E78060D8C1145DBF014582800DC13E
:100C10001713FFFFE702A34C1306800581459710C9
:100C2000FFFFE780C04E05451713FFFF6700634DC8
:100C300001458280814749C5C1C51713FFFFE702FF
:100C4000034AFC4141462E84AA846399C704138653
:100C50000501A2878146C14503C7070003C50703F5
:100C60008507298F3305D600034505008506298FA2
:100C7000A38FE7FEE392B6FE3044A2852685970057
:100C80000000E78060D0228597000000E78060F8D0
:100C900085473E851713FFFF6700A34613850703AB
:100CA0001D8E814522959710FFFFE78040467C40CE
:100CB000130700F813060402A2972388E70251BF26
:100CC0003E8582801713FFFFE70263416D712E841A
:100CD000B284AA8590102800368997000000E7802A
:100CE000A0D309EDD55725A050400C40280097000F
:100CF0000000E78040E27DD5FD142104F5F42C00CE
:100D00004A8597000000E78020F3814761DD3E853A
:100D100051611713FFFF6700C33E1713FFFFE70280
:100D2000033C41112EC432C62C000546970000003A
:100D3000E78080F941011713FFFF6700833C171319
:100D4000FFFFE702C33901112A842EC602C802CA76
:100D500002CC02CE97E00000E780C023B2462A868C
:100D6000A285080897000000E78060FB1375F50F67
:100D700005611713FFFF6700C3381713FFFFE70272
:100D800003367971B2872A8421462308B1001305FE
:100D90001101BE853AC436C697E00000E78000FB2B
:100DA000B24693059101368597000000E78060A860
:100DB0002285141035460C0897000000E78020F6C5
:100DC0002A84224701E921460C103A8597E0000069
:100DD000E780C0F7228545611713FFFF6700633284
:100DE0001713FFFFE702A32F7171AE84AA850A854E
:100DF000328497000000E78060BB11C90A86A6858F
:100E0000228597000000E78020B8814711E1C5479F
:100E10003E854D611713FFFF6700A32E1713FFFFD9
:100E2000E702E3281D712A8AB289BE8435468547C8
:100E3000130511012E8CB68A3A8BC28C468D23087D
:100E4000F10097E00000E78060F010100C08528578
:100E5000231F010097000000E780C0F82A843DEDC1
:100E6000A1476313FD089307900591E0E5473546D8
:100E7000E2851305110113990A012308F1001359A2
:100E8000090197E00000E78060EC13578900939711
:100E90008A00D98F90080C085285231FF100970013
:100EA0000000E78020F42A8415E9A1E49387FA0082
:100EB00091831379F9003EC6631309004149668B9B
:100EC0008144C14B854DB247639F970C6A868C0065
:100ED00033855C0197E00000E78040E722852561CB
:100EE0001713FFFF6700632093079004C9F0A5471D
:100EF000BDBF834701050947C14B2308F100834764
:100F00001105A58FA308F10093872400814463E1B4
:100F1000FB04014714083386E6008C08B386E4001E
:100F2000BA95DA9683C6060083C505000507AD8E1F
:100F30002300D600E390E7FE4147639CE704900856
:100F40000C08528597000000E780C0E925D181A0F8
:100F5000B3069B00BA871008B305F60090083E96CA
:100F600003C506000346060085078506298E2380F3
:100F7000C500E39277FF998F90080C085285BE94C4
:100F800097000000E78000E68947014749D12A849D
:100F9000B1B790083E96034606001408BE9623801B
:100FA000C600850759BFB2478504638797148147F8
:100FB0001808B306F70098083E973386F9000347F0
:100FC0000700034606008507318F2380E600E39182
:100FD00077FF90080C08528597000000E78080E0BA
:100FE0005DF53546E285130511012308B10197E04F
:100FF0000000E780A0D513970401418393978400F4
:101000002183D98F10180C085285231FF1009700F7
:101010000000E78020DD25FD814710183387F900A7
:101020003E960347070003460600B306FB0085070C
:10103000318F2380E600E39277FF65A81808B30696
:10104000F70098083E973386F900034707000346E8
:1010500006008507318F2380E600E3E127FFCA877A
:10106000639E770990080C08528597000000E7807E
:1010700060D711FD81479800B306F700900818105B
:101080003E973E9603470700034606008507318FCB
:101090002380E600E39177FF3546E28513051101D1
:1010A0002308B10197E00000E78040CA13970401CC
:1010B0004183939784002183D98F10180C0852859F
:1010C000231FF10097000000E780C0D1E31105EC79
:1010D000814710183387F9003E96034707000346FF
:1010E0000600B306FB008507318F2380E600E3E2AC
:1010F00027FFC109410BC1BB814785B79408BE9644
:1011000083C6060018083E972300D700850789BFCD
:10111000638006321713FFFFE70263F959712A84CF
:10112000BE89B28B85473546130511022E8B468C3E
:101130004289BA8A368A2300F10297E00000E780EC
:10114000E0C010180C102285231701029700000040
:10115000E78040C963180512A147631FFC06930787
:10116000900563930900E5473546DA8513051102BA
:1011700093140A012300F102C18097E00000E78088
:10118000E0BC93178A0013D78400D98F90080C1005
:1011900022852317F10297000000E780A0C47DE1BB
:1011A000639209049307FA00BD88918391E0C144DA
:1011B000C207C183DE8C814A3EC6414DB24763E21D
:1011C000FA0E6286B3854B01881097E00000E78035
:1011D00080B54DC93D557DA093079004E39609F86D
:1011E000A54759B7834701050947C14C2300F102C0
:1011F00083471105B3C7F900A300F10293872900C3
:10120000814963E1FC04814618103306D7008C083D
:101210003387D900B69556970347070083C5050065
:1012200085062D8F2300E600E390D7FE41476390AB
:10123000E70690080C10228597000000E78080BA2E
:1012400035D189A0B3863A01BA871010B305F600EC
:1012500090083E9603C506000346060085078506EE
:10126000298E2380C500E39297FF3387EC409008D6
:101270000C102285BA9997000000E780A0B6894734
:10128000014741D165611713FFFF670003E690082E
:101290003E96034606001410BE962380C6008507BE
:1012A00079B7B247850A93990A01939D8A0093D929
:1012B00009016391570F85473546DA8513051102F9
:1012C0002300F10293D9890097E00000E78000A88D
:1012D000B3ED3D0190000C1022852317B103970058
:1012E0000000E78020B059FD8147A68963EA970690
:1012F00026860C084A8597E00000E78020A58147F4
:101300001810B306F700100898083E973E9603475A
:101310000700034606008507318F2380E600E3E1DE
:1013200097FE639FA90590080C1022859700000086
:10133000E78040AB21F981479810B306F700900889
:1013400018183E973E960347070003460600850798
:10135000318F2380E600E391A7FF4109C10CB9BD9D
:1013600018089000B306F7003E963387FC00034749
:101370000700034606008507318F2380E600B5B7D6
:1013800098084E97034707001C10CE972380E7006C
:10139000850941BF85473546DA85130511022300CB
:1013A000F10293D9890097E00000E780209AB3ED1D
:1013B0003D0190000C1022852317B1039700000017
:1013C000E78040A2E31005EC814718089000B306BF
:1013D000F7003E963387FC000347070003460600EC
:1013E0008507318F2380E600E391A7FF41460C0873
:1013F0004A8597E00000E780609581471810B306A2
:10140000F700100898083E973E96034707000346EA
:1014100006008507318F2380E600E391A7FF90083F
:101420000C10228597000000E780C09B1DD599BD58
:101430007D5582801713FFFFE70263CA01112A84DA
:101440002E8593055100328902C002C202C402C631
:101450009304740097F0FFFFE780A03D1D46A6852A
:101460001305910097E00000E780408E10088A8500
:101470004A8597000000E780E09619ED9307140075
:10148000180883C607000346070085070507B18EC5
:10149000A38FD7FEE397F4FE05611713FFFF6700E4
:1014A00043C61713FFFFE702E3C12E848C414111AD
:1014B000AA89838715003289914463D30700A14428
:1014C0009757FF1F9387C7EC9C43A1C7C1CA8D479D
:1014D0002310F10083C725004A852301F10083C74B
:1014E0003500A301F10083C745002302F10083C743
:1014F0005500A302F10083C7650093059100A30383
:1015000001002303F1002304010097F0FFFFE780AF
:1015100040320C404A860A8597F0FFFFE78080330F
:101520000328040083564400A6881D08814701470C
:10153000E51642868A854E8597000000E780408E3A
:101540002A8919E5A685228597B0FFFFE780E0C1CB
:101550004A8541011713FFFF670003BA4A860A85CF
:1015600097F0FFFFE780002F6DB71713FFFFE7022B
:1015700063B52E848C414111AA8983871500328975
:10158000914463D30700A1449757FF1F938747E017
:101590009C43A1C7C1C68D472310F10083C7250016
:1015A0004A852301F10083C73500A301F10083C7F9
:1015B00045002302F10083C75500A302F10083C751
:1015C000650093059100A30301002303F1002304A8
:1015D000010097F0FFFFE780C0250C404A860A858E
:1015E00097F0FFFFE780002783564400032804009C
:1015F0008A85858EC2061D08C1822312D400A68862
:1016000081470147E51642864E8597000000E78036
:1016100060B041011713FFFF670003AE4A860A85D9
:1016200097F0FFFFE78000234DBF1713FFFFE7028E
:1016300003ABB335B000011185052A891315F601F6
:10164000336515012308B1009305110136843AC6AC
:1016500032C03EC442C297F0FFFFE780801DA24720
:101660001248425593D68700230BF1009305910150
:1016700093578800A30AD100A30BF100230C0101AA
:1016800097F0FFFFE780E01A324702460328040084
:10169000B337E000835644009207914411C2A1443D
:1016A0004A85A68842860C0897F0FFFFE7804077BE
:1016B0002A8919E5A685228597B0FFFFE780E0AA71
:1016C0004A8505611713FFFF6700A3A31713FFFFE8
:1016D000E702439F01113EC68647B335B00085053A
:1016E000AA891315F6015D8D2308B1009305110138
:1016F00036843A89B28442C446C297F0FFFFE7803D
:10170000401322489248164593578800A30AF100D7
:101710009305910193D78800230B0101A30BF100DE
:10172000230C110197F0FFFFE780A0103247104013
:1017300083564400B337E00092070328090091481C
:1017400091C0A1480C084E8597000000E780809C5E
:10175000AA8401E9835544004A8597B0FFFFE780DA
:10176000C0A0268505611713FFFF6700E398AA95BF
:101770009307F00F170701001307475E6317B500C3
:1017800013C5F7FF1375F50F828005058346F5FF36
:10179000B58FBA9783C70700D5B7035745001441E3
:1017A0009307F00F170601001306465B36974207B2
:1017B0004183139506014181631BE500AD8FB2970C
:1017C00003C50700130515F3133515008280850640
:1017D00003C5F6FFA98FB29783C70700D9BF1713B8
:1017E000FFFFE702C38FB28736842E86BA86AA85AA
:1017F0003E85BA8497F0FFFFE7806052634F050093
:10180000228597D00000E780E0782A86A686A28508
:10181000268597F0FFFFE78080501713FFFF6700D2
:10182000438E1713FFFFE702E3895D712A8BAE8AAF
:1018300017050100130505502C00B284368ABA89B9
:101840003E8997F0FFFFE780C04F2A845DE13410A6
:101850004146DA85280097F0FFFFE780404C2A8454
:1018600049E98547A303F100A6C293077100240844
:10187000BEC4A68685470D462C18281002DC02DE61
:10188000D6C0BEC697F0FFFFE78000442A8435E14A
:1018900083477102A6860D4693F7F7072300FA00E7
:1018A000C1473EDE2C188947281026DCA303F1002F
:1018B00097F0FFFFE78040412A8405ED4146A68569
:1018C0004E8597D00000E78060488D47A6860D467C
:1018D0002C182810A303F10097F0FFFFE780C03E0B
:1018E0002A8401E94146A6854A8597D00000E78011
:1018F000E045228561611703FFFF6700E37F17035F
:10190000FFFFE702C37D97F700009387A7A19843E5
:1019100083C7470079712A89AE8417050100130532
:10192000E5410C083AC42306F10097F0FFFFE78079
:1019300040412A8405ED14104146CA85080897F0F5
:10194000FFFFE780C03D2A8415E1140815462C00EE
:10195000081097F0FFFFE780803C2A8401E92146C8
:101960002C08268597D00000E780403E22854561FF
:101970001703FFFF6700E3781703FFFFE7022376F3
:1019800097F700009387079A9C477971AA842E8461
:10199000170501001305053B0C083EC697F0FFFF35
:1019A000E780203A0DE914104146A685080897F013
:1019B000FFFFE780C03605E1140811466C000810EF
:1019C00097F0FFFFE780A03519E58347F10193F712
:1019D000F7032300F40045611703FFFF67006372FC
:1019E0001703FFFFE702A36F3688A148814701472D
:1019F000E54697F0FFFFE780A0421703FFFF67006F
:101A000043701703FFFFE702836D3688A1488147C3
:101A10000147E54697F0FFFFE780C06F1703FFFF20
:101A20006700236E1703FFFFE702636B01112A842F
:101A30002E850C0832C697F0FFFFE780803009ED55
:101A40003247970601009386662E1008C14522850D
:101A500097000000E780E0D805611703FFFF6700EB
:101A6000436A1703FFFFE70283674111C1472EC096
:101A700032C48A8509463EC23EC697F0FFFFE78022
:101A8000A02441011703FFFF6700A3671703FFFFAF
:101A9000E702E3644111AE8613061009AA850A85A0
:101AA00002C002C202C402C697F0FFFFE7802027EF
:101AB00041011703FFFF6700C3641703FFFFE7023D
:101AC0000362328797060100938646282E86930587
:101AD000000297000000E780C0D01703FFFF6700F7
:101AE00043621703FFFFE702835F7971C1472ACC86
:101AF0002ED032D42C080D4628003ECE3ED23ED603
:101B000002C402C602C802CA97F0FFFFE780C01BEA
:101B100045611703FFFF6700C35E1703FFFFE7027E
:101B2000035C0111AA842E84170501001305852288
:101B30008A8597F0FFFFE780C02015E5140841462D
:101B4000A6850A8597F0FFFFE780601D09ED8347B2
:101B5000E1010347F101A207D98FCA07C983617761
:101B6000D98F2310F40005611703FFFF6700635945
:101B700015CD1703FFFFE70283569747FF1F938793
:101B8000A72E90439745FF1F9385452E1745FF1FAE
:101B90001305852997D00000E78000C51745FF1F72
:101BA000130585281703FFFF6700A3551745FF1F7F
:101BB0001305852782808DCD1703FFFFE70223528F
:101BC0009747FF1F9387472A944301112E840A8663
:101BD0009745FF1F9385852997D00000E78040C671
:101BE0000A850294014505611703FFFF67006351F1
:101BF0007D5582801703FFFFE702634E97D00000F8
:101C0000E78080D19747FF1F23A0A72617F5FFFF86
:101C10001305E5C997B00000E780C0741703FFFF04
:101C20006700234E1747FF1F13074726931715001A
:101C300008433E95FD572310F50082801703FFFFF0
:101C4000E702E3492A84084009E51703FFFF67001C
:101C5000434B1C4158401CC06313E5005CC08347E4
:101C6000550023200500F99BA302F50097A0FFFF74
:101C7000E780207CC9BF1703FFFFE702A344974713
:101C8000FF1F9387A72298432A8411CB83473500EF
:101C900093F7070289C70355050089450297130585
:101CA000440197B00000E780403B83550400035592
:101CB000E40097300000E780A00C485819C597A0B1
:101CC000FFFFE7800077232A0402130584039700AF
:101CD0000000E780E0F68144B1499790FFFFE7807C
:101CE000206A63CBA402834734002320040493F7C3
:101CF00027FCA301F40000489790FFFFE7804069AC
:101D000013161500814522859700FFFFE7802040CC
:101D10001703FFFF6700433EB3873403032904031F
:101D200085043E994A8597000000E78060F123040E
:101D3000090065B78347350093F7070299E301452A
:101D400082808357E500E39CB7FEC167FD176316E9
:101D5000F60005458280054599A81703FFFFE702B5
:101D6000033893170601C187B2842A840149635955
:101D7000F002835705009DCB01456367F6000345DC
:101D800084003E953325A6001375F50F0DA01C4861
:101D900013171900BA9783D70700E38E97FA05093E
:101DA0009790FFFFE780C05EE343A9FE014517035C
:101DB000FFFF670003351703FFFFE702A330AE897B
:101DC000AA849790FFFFE78060522A8497D0FFFF94
:101DD000E780A02EAA86014713068401970500001C
:101DE000938585E41745FF1F1305850A9790FFFF2C
:101DF000E780E0182A8925C98C441304C500228590
:101E00009E0593F5050897A0FFFFE780403CCC4076
:101E100083877400E18163DD070493E5050822856B
:101E200097A0FFFFE780A03A0D46938544002285E6
:101E300097A0FFFFE780C03683D50400228597A0D6
:101E4000FFFFE780E03D83D52400228597A0FFFFB8
:101E5000E780003D03D6490083A50900228597A0AD
:101E6000FFFFE780E0334A851703FFFF6700C328C1
:101E700093F5F5076DB71703FFFFE702432601113E
:101E80002A84328532C697A0FFFFE780E02797803B
:101E9000FFFFE780C030835704001747FF1F130779
:101EA00067183246231BF100930700F8A30DF100D9
:101EB0001C471843231AA1008983858BB307F74079
:101EC000B28548083ECE231C0100230D0100970077
:101ED0000000E78080EE05611703FFFF67006322C3
:101EE0001703FFFFE702031E004101453DC49304B1
:101EF000C40026853289AE8997A0FFFFE780C02401
:101F000095452A8A2685035B040197A0FFFFE78099
:101F10002021268597A0FFFFE780603E8D45AA8A95
:101F2000268597A0FFFFE780A01F268597A0FFFFCB
:101F3000E780E03C5C48420A135A0A01D2975CC42D
:101F400023186401814763983A0146054D813306A1
:101F500025419337160013F5F70F1703FFFF6700AE
:101F6000A3191703FFFFE702031589692A8BAE8BBC
:101F7000328AB68A81440144314CFD199790FFFFA3
:101F8000E780004063CDA4009790FFFFE7804042C8
:101F9000018D33B5AA001703FFFF6700431533898E
:101FA000840383270B003E9963170A008347890047
:101FB00085043E94E1B703560A00DE854A8533F670
:101FC000C90097000000E780E0F16DD10545E1B759
:101FD0001703FFFFE702A31001112A847C000355B9
:101FE000E5003ECAB70707003ECC7C003ECE9720F6
:101FF0000000E78020082A898545480897A0FFFF50
:10200000E78020399945480897A0FFFFE780E01551
:10201000AA844A8597200000E780A0082380A400B6
:102020009747FF1F938707009C434166130606F0FE
:102030009396870113D78701558F93D68700F18E2A
:10204000558FA207B706FF00F58FD98F11462C00D8
:10205000138514003EC497D00000E78020CF5008BD
:10206000A38204008945228597000000E780E0E014
:1020700019C9AA851305840397A0FFFFE780E03103
:102080003C4085073CC005611703FFFF67006307FD
:102090001703FFFFE702A3049790FFFFE78040319B
:1020A0002A8405049790FFFFE780802F3305A40260
:1020B000F14791453305F50297200000E78020BAEB
:1020C00011E565551703FFFF6700A3039747FF1F3F
:1020D00023A6A7DC9790FFFFE780802D2A840504C4
:1020E0009790FFFFE780C02B3305A40289450605C2
:1020F00097200000E780A0B669D59747FF1F23A768
:10210000A7D89790FFFFE780A02A2A84050497901C
:10211000FFFFE780E0283304A4029747FF1F2399BD
:1021200087D69790FFFFE780A0282A849790FFFF2B
:10213000E7800027930714003385A7029747FF1F06
:102140002399A7D497070100938787841747FF1F18
:102150002324F7D40145BDB71703FFFFE70283F639
:10216000AA842E8901449749FF1F9389A9EB130A7A
:1021700080069790FFFFE780A0226347A4000145F7
:102180001703FFFF670043F73305440383A70902E2
:102190004A86A6853E9597000000E780E0B919E1E0
:1021A0000504C1BF0545E9BF1703FFFFE702A3F020
:1021B000AA8A2E8BB28B368C3A8A8144014481499B
:1021C000974CFF1F938C0CE6130D80069790FFFF32
:1021D000E780001D63C9A40011E085494E851703FF
:1021E000FFFF6700C3F03389A40383A70C025E8658
:1021F000D6853E994A8597000000E780E0B31DC16F
:102200009790FFFFE780C01A0544636D4501D286B1
:102210006286DA851305090397000000E780A0D4E1
:1022200011C1854985045DB71703FFFFE70283E904
:10223000C16441112A8901449749FF1F938989DEAE
:10224000130A8006FD1436C632C42EC29790FFFFD3
:10225000E780001592452246B2466348A400014536
:1022600041011703FFFF670023E93305440383A7F8
:1022700009023E9509C683473500C18B9DC791C6AB
:102280008347350093F707028DC363069900835790
:10229000E500639C27010357050001CB63E7E500D8
:1022A00083478500BA97E3CDF5FA050469BF1703A4
:1022B000FFFFE70223E1C1642A8901449749FF1F18
:1022C000938949D6130A8006FD149790FFFFE78093
:1022D000200D6346A4001703FFFF6700E3E1330509
:1022E000440383A709023E958357E500638A97005C
:1022F000630499006396270197000000E780E09748
:102300000504E1B71703FFFFE70263DA89692A8A48
:10231000AE8A328BB68B8144174CFF1F130C8CD0C6
:10232000930C8006314DFD199790FFFFE780400721
:1023300063C6A4001703FFFF670023DB3389940300
:1023400083270C028355CA015A863E994A85970015
:102350000000E780609E31C1814D15A03384AD033C
:102360008327090303D60B00D68533F6C9003E94B4
:10237000228597000000E780E0B609E9850D979077
:10238000FFFFE780E0FFE3CBADFC01A822859700CB
:102390000000E780E08A23040400850471B7170376
:1023A000FFFFE70243D14169AA8A014A174BFF1F89
:1023B000130B4BC77D19C14B054C9790FFFFE7806E
:1023C00020FE6346AA001703FFFF670043D293096C
:1023D0008006B3073A0383290B02BE9983D7E9002D
:1023E000638E270163842A01639A570103A489033A
:1023F00001E84E8597000000E780C0BD050A75BF63
:1024000083570401639977099304C400268597A034
:10241000FFFFE78060D385452A8D2685835C040114
:1024200097A0FFFFE780C0CF268597A0FFFFE7803A
:10243000A0E762056185635905048D45268597A04F
:10244000FFFFE780E0CD8945268597A0FFFFE78065
:1024500020CD8945268597A0FFFFE78060CC854584
:10246000268597A0FFFFE780E0CC8347050009475A
:1024700093F7F707639AE7009945268597A0FFFF32
:10248000E78040CBA30285014848337D2D01231806
:1024900094016A9548C40040A1BF1703FFFFE702FB
:1024A00003C437E404008327041D82979747FF1F66
:1024B00083C747A41715FF1F13054507A300F500A1
:1024C0008327441C82978327841C81461306F00FC0
:1024D0008145014582971703FFFF670083C21747B5
:1024E000FF1F1307279118439745FF1F83C585A03A
:1024F0009747FF1F9387879E83468703034697036B
:102500006397D5009747FF1F2386C79E828083C5A8
:1025100087010347A7036317B6009747FF1F238B65
:10252000E79C828003C687016317C7009747FF1F98
:102530002382D79C828083C68701130750026319C8
:10254000D700930760021747FF1F2305F79A828081
:1025500083C68701130660026315D60093077002D5
:10256000DDB783C7870155BF9747FF1F938707973D
:10257000D44B0947638DE6081703FFFFE70223B634
:102580001749FF1F1309C9923E8483470900918BA5
:102590009DCFB7E4040083A7041D829783A7441C42
:1025A0001745FF1F13054591829783A7841C814619
:1025B0001746FF1F0346469281450145829721C574
:1025C00083470900ED9B1747FF1F2303F78E8347BF
:1025D000040093F7F70F85CB91471747FF1F232977
:1025E000F79097000000E78080EB97000000E780FD
:1025F00040EFB7E70400BC4F414691451745FF1F28
:102600000345458E82971703FFFF670083AF8280E3
:102610001703FFFFE702A3AC8D4741116306F504E2
:10262000C5476308F50285476310F5029747FF1F0A
:102630002384A78CB7E70400BC4B93050010174513
:10264000FF1F0345258A829741011703FFFF67009B
:1026500043AB85471747FF1F2300F78AB7E70400FE
:10266000BC4B93050020E1BF9747FF1F9387078767
:10267000D44B1147638DE600B7E7040083A7071D1D
:102680008297B7E70400BC4B930500044DBF054992
:102690001747FF1F232E278583C7070032C62E84C6
:1026A00093F7F70FD5D3B7E4040083A7041D7D1477
:1026B0001374F40F8297E37689FCB245994703C6F9
:1026C0001500E3F0C7FCFC4409061745FF1F13057E
:1026D000E5828297BC48930500081745FF1F034514
:1026E0006580829779BF1703FFFFE702439F173783
:1026F000FF1F1307A77E4047184B1C409736FF1F4C
:1027000023A4F67E6316E4001737FF1F2320F77E0D
:10271000130584FE9790FFFFE78060A6035564FFD2
:102720009780FFFFE780E06E97A0FFFFE78060D013
:102730001703FFFF6700E39C1703FFFFE702239ADD
:102740009737FF1F93878779D84BDC4789C7970056
:102750000000E78080F985471737FF1F232AF778A5
:102760009737FF1F938707699C439305000217352E
:10277000FF1F0345257783C787031737FF1F230BE9
:10278000F776B7E70400BC4B82971703FFFF67009B
:1027900043979737FF1F23A5A77482801703FFFF76
:1027A000E702439237E404007C4CA1451735FF1F34
:1027B0000345457382977C48A1451735FF1F0345A4
:1027C00065729734FF1F938464718297DC4489EBB0
:1027D00097000000E78080D91703FFFF6700C391CF
:1027E00003D567FF9780FFFFE780A062AA896DD1BC
:1027F000D84891476310F7027C4C91451735FF1F6D
:102800000345456E82977C4891451735FF1F034568
:10281000656D829703A9490103D409018947B7E986
:1028200004001737FF1F2325F76C83A7091D210418
:102830004204829783C784011715FF1F130505CF34
:1028400061191717FF1FA303F7CE83A7491C418007
:1028500082979737FF1F2381076A83A7C91C814688
:1028600009469375F40F4A85829711E99737FF1F40
:1028700083C7C77889C79700FF1FE780A037B7E7EE
:102880000400BC4F2146A1451735FF1F0345856550
:10289000829799B71703FFFFE702638493F7052038
:1028A00001112E8481CF97000000E78020E91345B5
:1028B000042005611703FFFF6700A38493F7051049
:1028C000A9CF9734FF1F93846461DC489700000010
:1028D000E78020C11737FF1F1307C751184383C76D
:1028E0008401034787036318F700DC4489C7970016
:1028F0000000E78080DF85471737FF1F232AF75E38
:10290000B7E70400BC4B930500021735FF1F0345D2
:10291000655D82971345041069BF93F70508BDC72D
:102920009737FF1F83C7975DE91719469735FF1F34
:102930009385E55C1305D10093F4F70F1739FF1F5A
:102940000349C95B97C00000E780404093970401AA
:10295000C1831737FF1F1307E75A231DF100231CFC
:10296000F1009737FF1F938767573ACE3ACAD8438B
:102970002306010009CBDC439315890154080D4659
:10298000E185680082971345040825B793F7250071
:10299000A5C39737FF1F93876754D84B89476306B2
:1029A000F7029737FF1F83C7A75013F7270011EFD0
:1029B000918B99CFB7E70400BC4F1306000A8945F5
:1029C0001735FF1F03450552829713452400D5B5DF
:1029D0009737FF1F938707429C4383C787031737A7
:1029E000FF1F2309F75097000000E78060DBF1BF6D
:1029F00093F7050281CB97000000E78060DA13456A
:102A0000040245BD93F7850081CB97000000E78065
:102A1000E0D21345840071BD93F7150081CB970078
:102A20000000E780A0B41345140061B593F745009A
:102A300081CB97000000E78060B31345440095BD4B
:102A400093F7050495C39737FF1F83C7274991CB99
:102A500097000000E780A0A491471737FF1F2329A4
:102A6000F74813450404B1B593F705010145E38226
:102A700007E49737FF1F93876746D84B914763104A
:102A8000F7049737FF1F9387A7429C4313D727006C
:102A90008583D98F858B91E7B7E7040083A7071D4E
:102AA0008297B7E70400FC4F91451735FF1F034598
:102AB0006543829785471737FF1F232BF74213453E
:102AC0000401C5BB9737FF1F238AA752828017F3E3
:102AD000FEFFE702C3609737FF1F23A70740973722
:102AE000FF1F23A5074085471734FF1F13048430B9
:102AF0001737FF1F232EF73E1C4083C78703173766
:102B0000FF1F2309F73E9790FFFFE780A08F29C59D
:102B10009717FF1F23A0A7A21C401705000013054D
:102B2000A5D783C787031737FF1F2305F73C171760
:102B3000FF1FA30DF79E9737FF1FA381073AB7E743
:102B4000040083A7070882979737FF1F238CA738B5
:102B500017F3FEFF6700E35AB7C7898E938767EDC7
:102B60001717FF1F2328F79C45BF1737FF1F034781
:102B7000E736795555E79737FF1F9387273603C701
:102B8000170005079736FF1FA38AE63403C717000F
:102B90008D463377D7029736FF1FA381E63483C66D
:102BA00017001737FF1F1307E724184393F6F60F94
:102BB000A9EE834787031737FF1F230DF732854799
:102BC0001737FF1F230CF7309737FF1F9387472EC8
:102BD0009C430145998BA9E717F3FEFFE7022350B9
:102BE00037E404007C48C1451735FF1F0345852F96
:102BF00082973C4885451735FF1F0345A52E8297D0
